 qagamex86

 Timestamp is 4839b8c7 (Sun May 25 23:06:47 2008)

 Preferred load address is 20000000

 Start         Length     Name                   Class
 0001:00000000 0003b186H .text                   CODE
 0002:00000000 000000e0H .idata$5                DATA
 0002:000000e0 00006d48H .rdata                  DATA
 0002:00006e30 00000008H .rdata$sxdata           DATA
 0002:00006e38 00000004H .rtc$IAA                DATA
 0002:00006e3c 00000004H .rtc$IZZ                DATA
 0002:00006e40 00000004H .rtc$TAA                DATA
 0002:00006e44 00000004H .rtc$TZZ                DATA
 0002:00006e48 00000014H .idata$2                DATA
 0002:00006e5c 00000014H .idata$3                DATA
 0002:00006e70 000000e0H .idata$4                DATA
 0002:00006f50 000003e4H .idata$6                DATA
 0002:00007340 0000005aH .edata                  DATA
 0003:00000000 00000004H .CRT$XCA                DATA
 0003:00000004 00000004H .CRT$XCAA               DATA
 0003:00000008 00000004H .CRT$XCZ                DATA
 0003:0000000c 00000004H .CRT$XIA                DATA
 0003:00000010 00000010H .CRT$XIC                DATA
 0003:00000020 00000004H .CRT$XIZ                DATA
 0003:00000024 00000004H .CRT$XPA                DATA
 0003:00000028 00000004H .CRT$XPX                DATA
 0003:0000002c 00000004H .CRT$XPZ                DATA
 0003:00000030 00000004H .CRT$XTA                DATA
 0003:00000034 00000004H .CRT$XTZ                DATA
 0003:00000040 00002684H .data                   DATA
 0003:000026e0 0014c6a0H .bss                    DATA

  Address         Publics by Value              Rva+Base     Lib:Object

 0000:00000000       __except_list              00000000     <absolute>
 0000:00000002       ___safe_se_handler_count   00000002     <absolute>
 0001:00000000       _BotNumActivePlayers       20001000 f   ai_chat.obj
 0001:000000d0       _BotIsFirstInRankings      200010d0 f   ai_chat.obj
 0001:000001e0       _BotIsLastInRankings       200011e0 f   ai_chat.obj
 0001:000002f0       _BotFirstClientInRankings  200012f0 f   ai_chat.obj
 0001:00000400       _BotLastClientInRankings   20001400 f   ai_chat.obj
 0001:00000510       _BotRandomOpponentName     20001510 f   ai_chat.obj
 0001:00000670       _BotMapTitle               20001670 f   ai_chat.obj
 0001:000006c0       _BotWeaponNameForMeansOfDeath 200016c0 f   ai_chat.obj
 0001:00000760       _BotRandomWeaponName       20001760 f   ai_chat.obj
 0001:000007f0       _BotVisibleEnemies         200017f0 f   ai_chat.obj
 0001:000008c0       _BotValidChatPosition      200018c0 f   ai_chat.obj
 0001:00000a50       _BotChat_EnterGame         20001a50 f   ai_chat.obj
 0001:00000b60       _BotChat_ExitGame          20001b60 f   ai_chat.obj
 0001:00000c60       _BotChat_StartLevel        20001c60 f   ai_chat.obj
 0001:00000d60       _BotChat_EndLevel          20001d60 f   ai_chat.obj
 0001:00000f30       _BotChat_Death             20001f30 f   ai_chat.obj
 0001:000012b0       _BotChat_Kill              200022b0 f   ai_chat.obj
 0001:000014b0       _BotChat_EnemySuicide      200024b0 f   ai_chat.obj
 0001:000015c0       _BotChat_HitTalking        200025c0 f   ai_chat.obj
 0001:00001740       _BotChat_HitNoDeath        20002740 f   ai_chat.obj
 0001:000018f0       _BotChat_HitNoKill         200028f0 f   ai_chat.obj
 0001:00001a60       _BotChat_Random            20002a60 f   ai_chat.obj
 0001:00001cb0       _BotChatTime               20002cb0 f   ai_chat.obj
 0001:00001ce0       _BotChatTest               20002ce0 f   ai_chat.obj
 0001:000027f0       _BotGetItemTeamGoal        200037f0 f   ai_cmd.obj
 0001:00002850       _BotGetMessageTeamGoal     20003850 f   ai_cmd.obj
 0001:000028a0       _BotGetTime                200038a0 f   ai_cmd.obj
 0001:000029b0       _FindClientByName          200039b0 f   ai_cmd.obj
 0001:00002a60       _FindEnemyByName           20003a60 f   ai_cmd.obj
 0001:00002b40       _NumPlayersOnSameTeam      20003b40 f   ai_cmd.obj
 0001:00002be0       _BotGetPatrolWaypoints     20003be0 f   ai_cmd.obj
 0001:00002e00       _BotAddressedToBot         20003e00 f   ai_cmd.obj
 0001:00003060       _BotMatch_HelpAccompany    20004060 f   ai_cmd.obj
 0001:000033d0       _BotMatch_DefendKeyArea    200043d0 f   ai_cmd.obj
 0001:00003500       _BotMatch_GetItem          20004500 f   ai_cmd.obj
 0001:00003600       _BotMatch_Camp             20004600 f   ai_cmd.obj
 0001:000038d0       _BotMatch_Patrol           200048d0 f   ai_cmd.obj
 0001:000039d0       _BotMatch_GetFlag          200049d0 f   ai_cmd.obj
 0001:00003ad0       _BotMatch_RushBase         20004ad0 f   ai_cmd.obj
 0001:00003bc0       _BotMatch_TaskPreference   20004bc0 f   ai_cmd.obj
 0001:00003cc0       _BotMatch_ReturnFlag       20004cc0 f   ai_cmd.obj
 0001:00003d90       _BotMatch_JoinSubteam      20004d90 f   ai_cmd.obj
 0001:00003e40       _BotMatch_LeaveSubteam     20004e40 f   ai_cmd.obj
 0001:00003ee0       _BotMatch_WhichTeam        20004ee0 f   ai_cmd.obj
 0001:00003f60       _BotMatch_CheckPoint       20004f60 f   ai_cmd.obj
 0001:00004150       _BotMatch_FormationSpace   20005150 f   ai_cmd.obj
 0001:00004200       _BotMatch_Dismiss          20005200 f   ai_cmd.obj
 0001:000042a0       _BotMatch_Suicide          200052a0 f   ai_cmd.obj
 0001:00004320       _BotMatch_StartTeamLeaderShip 20005320 f   ai_cmd.obj
 0001:000043d0       _BotMatch_StopTeamLeaderShip 200053d0 f   ai_cmd.obj
 0001:00004490       _BotMatch_WhoIsTeamLeader  20005490 f   ai_cmd.obj
 0001:000044f0       _BotMatch_WhatAreYouDoing  200054f0 f   ai_cmd.obj
 0001:000046d0       _BotMatch_WhatIsMyCommand  200056d0 f   ai_cmd.obj
 0001:00004710       _BotNearestVisibleItem     20005710 f   ai_cmd.obj
 0001:00004830       _BotMatch_WhereAreYou      20005830 f   ai_cmd.obj
 0001:00004a60       _BotMatch_LeadTheWay       20005a60 f   ai_cmd.obj
 0001:00004c80       _BotMatch_Kill             20005c80 f   ai_cmd.obj
 0001:00004d90       _BotMatch_CTF              20005d90 f   ai_cmd.obj
 0001:00004ef0       _BotMatch_EnterGame        20005ef0 f   ai_cmd.obj
 0001:00004f30       _BotMatch_NewLeader        20005f30 f   ai_cmd.obj
 0001:00004f80       _BotMatchMessage           20005f80 f   ai_cmd.obj
 0001:00005430       _BotResetNodeSwitches      20006430 f   ai_dmnet.obj
 0001:00005440       _BotDumpNodeSwitches       20006440 f   ai_dmnet.obj
 0001:000054c0       _BotRecordNodeSwitch       200064c0 f   ai_dmnet.obj
 0001:00005530       _BotGetAirGoal             20006530 f   ai_dmnet.obj
 0001:000056d0       _BotGoForAir               200066d0 f   ai_dmnet.obj
 0001:000057e0       _BotNearbyGoal             200067e0 f   ai_dmnet.obj
 0001:00005880       _BotReachedGoal            20006880 f   ai_dmnet.obj
 0001:000059c0       _BotGetItemLongTermGoal    200069c0 f   ai_dmnet.obj
 0001:00005a90       _BotGetLongTermGoal        20006a90 f   ai_dmnet.obj
 0001:000071f0       _BotLongTermGoal           200081f0 f   ai_dmnet.obj
 0001:00007620       _AINode_Observer           20008620 f   ai_dmnet.obj
 0001:00007670       _AINode_Respawn            20008670 f   ai_dmnet.obj
 0001:00007750       _BotSelectActivateWeapon   20008750 f   ai_dmnet.obj
 0001:00007810       _BotClearPath              20008810 f   ai_dmnet.obj
 0001:00007b80       _AIEnter_Battle_SuicidalFight 20008b80 f   ai_dmnet.obj
 0001:00007bd0       _AIEnter_Battle_NBG        20008bd0 f   ai_dmnet.obj
 0001:00007c00       _AIEnter_Respawn           20008c00 f   ai_dmnet.obj
 0001:00007ce0       _AINode_Battle_Retreat     20008ce0 f   ai_dmnet.obj
 0001:00008220       _AIEnter_Battle_Retreat    20009220 f   ai_dmnet.obj
 0001:00008250       _AINode_Battle_Chase       20009250 f   ai_dmnet.obj
 0001:00008720       _AIEnter_Battle_Chase      20009720 f   ai_dmnet.obj
 0001:00008760       _AINode_Battle_Fight       20009760 f   ai_dmnet.obj
 0001:00008c00       _AIEnter_Battle_Fight      20009c00 f   ai_dmnet.obj
 0001:00008c40       _AINode_Seek_NBG           20009c40 f   ai_dmnet.obj
 0001:00009020       _AIEnter_Seek_NBG          2000a020 f   ai_dmnet.obj
 0001:000090c0       _AINode_Seek_LTG           2000a0c0 f   ai_dmnet.obj
 0001:00009640       _AIEnter_Seek_LTG          2000a640 f   ai_dmnet.obj
 0001:000096e0       _AINode_Stand              2000a6e0 f   ai_dmnet.obj
 0001:000097f0       _AIEnter_Stand             2000a7f0 f   ai_dmnet.obj
 0001:00009830       _AINode_Intermission       2000a830 f   ai_dmnet.obj
 0001:000098b0       _AIEnter_Intermission      2000a8b0 f   ai_dmnet.obj
 0001:00009910       _AINode_Seek_ActivateEntity 2000a910 f   ai_dmnet.obj
 0001:00009ed0       _AINode_Battle_NBG         2000aed0 f   ai_dmnet.obj
 0001:0000a2e0       _AIEnter_Seek_ActivateEntity 2000b2e0 f   ai_dmnet.obj
 0001:0000a310       _BotSetUserInfo            2000b310 f   ai_dmq3.obj
 0001:0000a370       _BotCTFCarryingFlag        2000b370 f   ai_dmq3.obj
 0001:0000a3b0       _BotTeam                   2000b3b0 f   ai_dmq3.obj
 0001:0000a440       _BotOppositeTeam           2000b440 f   ai_dmq3.obj
 0001:0000a470       _EntityIsDead              2000b470 f   ai_dmq3.obj
 0001:0000a4b0       _EntityCarriesFlag         2000b4b0 f   ai_dmq3.obj
 0001:0000a4d0       _EntityIsInvisible         2000b4d0 f   ai_dmq3.obj
 0001:0000a4f0       _EntityIsShooting          2000b4f0 f   ai_dmq3.obj
 0001:0000a500       _BotRememberLastOrderedTask 2000b500 f   ai_dmq3.obj
 0001:0000a550       _BotRefuseOrder            2000b550 f   ai_dmq3.obj
 0001:0000a5c0       _BotCTFRetreatGoals        2000b5c0 f   ai_dmq3.obj
 0001:0000a630       _BotPointAreaNum           2000b630 f   ai_dmq3.obj
 0001:0000a690       _ClientName                2000b690 f   ai_dmq3.obj
 0001:0000a720       _ClientFromName            2000b720 f   ai_dmq3.obj
 0001:0000a7c0       _stristr                   2000b7c0 f   ai_dmq3.obj
 0001:0000a830       _EasyClientName            2000b830 f   ai_dmq3.obj
 0001:0000a9f0       _BotSynonymContext         2000b9f0 f   ai_dmq3.obj
 0001:0000aa20       _BotChooseWeapon           2000ba20 f   ai_dmq3.obj
 0001:0000aa90       _BotSetupForMovement       2000ba90 f   ai_dmq3.obj
 0001:0000aba0       _BotUpdateInventory        2000bba0 f   ai_dmq3.obj
 0001:0000ad70       _BotUpdateBattleInventory  2000bd70 f   ai_dmq3.obj
 0001:0000ade0       _BotBattleUseItems         2000bde0 f   ai_dmq3.obj
 0001:0000ae50       _BotIsDead                 2000be50 f   ai_dmq3.obj
 0001:0000ae60       _BotIsObserver             2000be60 f   ai_dmq3.obj
 0001:0000aec0       _BotIntermission           2000bec0 f   ai_dmq3.obj
 0001:0000aef0       _BotInLavaOrSlime          2000bef0 f   ai_dmq3.obj
 0001:0000af30       _BotCreateWayPoint         2000bf30 f   ai_dmq3.obj
 0001:0000afc0       _BotFindWayPoint           2000bfc0 f   ai_dmq3.obj
 0001:0000b000       _BotFreeWaypoints          2000c000 f   ai_dmq3.obj
 0001:0000b030       _TeamPlayIsOn              2000c030 f   ai_dmq3.obj
 0001:0000b040       _BotAggression             2000c040 f   ai_dmq3.obj
 0001:0000b160       _BotWantsToRetreat         2000c160 f   ai_dmq3.obj
 0001:0000b1f0       _BotWantsToChase           2000c1f0 f   ai_dmq3.obj
 0001:0000b280       _BotCanAndWantsToRocketJump 2000c280 f   ai_dmq3.obj
 0001:0000b300       _BotHasPersistantPowerupAndWeapon 2000c300 f   ai_dmq3.obj
 0001:0000b3d0       _BotGoCamp                 2000c3d0 f   ai_dmq3.obj
 0001:0000b4a0       _BotWantsToCamp            2000c4a0 f   ai_dmq3.obj
 0001:0000b670       _BotDontAvoid              2000c670 f   ai_dmq3.obj
 0001:0000b6d0       _BotGoForPowerups          2000c6d0 f   ai_dmq3.obj
 0001:0000b720       _BotRoamGoal               2000c720 f   ai_dmq3.obj
 0001:0000ba00       _BotAttackMove             2000ca00 f   ai_dmq3.obj
 0001:0000bf60       _BotSameTeam               2000cf60 f   ai_dmq3.obj
 0001:0000c020       _InFieldOfVision           2000d020 f   ai_dmq3.obj
 0001:0000c0f0       _BotEntityVisible          2000d0f0 f   ai_dmq3.obj
 0001:0000c4f0       _BotFindEnemy              2000d4f0 f   ai_dmq3.obj
 0001:0000c900       _BotTeamFlagCarrierVisible 2000d900 f   ai_dmq3.obj
 0001:0000c9b0       _BotTeamFlagCarrier        2000d9b0 f   ai_dmq3.obj
 0001:0000ca30       _BotEnemyFlagCarrierVisible 2000da30 f   ai_dmq3.obj
 0001:0000cae0       _BotAimAtEnemy             2000dae0 f   ai_dmq3.obj
 0001:0000da00       _BotCheckAttack            2000ea00 f   ai_dmq3.obj
 0001:0000de80       _BotMapScripts             2000ee80 f   ai_dmq3.obj
 0001:0000e1a0       _BotSetMovedir             2000f1a0 f   ai_dmq3.obj
 0001:0000e260       _BotModelMinsMaxs          2000f260 f   ai_dmq3.obj
 0001:0000e350       _BotFuncButtonActivateGoal 2000f350 f   ai_dmq3.obj
 0001:0000eb10       _BotFuncDoorActivateGoal   2000fb10 f   ai_dmq3.obj
 0001:0000ec30       _BotTriggerMultipleActivateGoal 2000fc30 f   ai_dmq3.obj
 0001:0000ede0       _BotPushOntoActivateGoalStack 2000fde0 f   ai_dmq3.obj
 0001:0000ef60       _BotEnableActivateGoalAreas 2000ff60 f   ai_dmq3.obj
 0001:0000efc0       _BotIsGoingToActivateEntity 2000ffc0 f   ai_dmq3.obj
 0001:0000f040       _BotGetActivateGoal        20010040 f   ai_dmq3.obj
 0001:0000f7e0       _BotGoForActivateGoal      200107e0 f   ai_dmq3.obj
 0001:0000f890       _BotRandomMove             20010890 f   ai_dmq3.obj
 0001:0000f920       _BotAIBlocked              20010920 f   ai_dmq3.obj
 0001:0000fbe0       _BotAIPredictObstacles     20010be0 f   ai_dmq3.obj
 0001:0000fd70       _BotCheckConsoleMessages   20010d70 f   ai_dmq3.obj
 0001:00010100       _BotCheckEvents            20011100 f   ai_dmq3.obj
 0001:00010440       _BotCheckSnapshot          20011440 f   ai_dmq3.obj
 0001:00010530       _BotAlternateRoute         20011530 f   ai_dmq3.obj
 0001:000105b0       _BotGetAlternateRouteGoal  200115b0 f   ai_dmq3.obj
 0001:00010690       _BotDeathmatchAI           20011690 f   ai_dmq3.obj
 0001:000109b0       _BotSetupDeathmatchAI      200119b0 f   ai_dmq3.obj
 0001:00010b80       _BotSetLastOrderedTask     20011b80 f   ai_dmq3.obj
 0001:00010cc0       _BotCTFSeekGoals           20011cc0 f   ai_dmq3.obj
 0001:000113d0       _BotTeamGoals              200123d0 f   ai_dmq3.obj
 0001:00011440       _ClientOnSameTeamFromName  20012440 f   ai_dmq3.obj
 0001:00011500       _BotPopFromActivateGoalStack 20012500 f   ai_dmq3.obj
 0001:00011550       _BotClearActivateGoalStack 20012550 f   ai_dmq3.obj
 0001:00011600       _BotAI_Print               20012600 f   ai_main.obj
 0001:000116e0       _BotAI_Trace               200126e0 f   ai_main.obj
 0001:00011780       _BotAI_GetClientState      20012780 f   ai_main.obj
 0001:000117c0       _BotAI_GetEntityState      200127c0 f   ai_main.obj
 0001:00011820       _BotAI_GetSnapshotEntity   20012820 f   ai_main.obj
 0001:00011860       _BotAI_BotInitialChat      20012860 f   ai_main.obj
 0001:00011900       _BotTestAAS                20012900 f   ai_main.obj
 0001:000119d0       _BotSetInfoConfigString    200129d0 f   ai_main.obj
 0001:00011ce0       _BotUpdateInfoConfigStrings 20012ce0 f   ai_main.obj
 0001:00011d90       _BotInterbreedBots         20012d90 f   ai_main.obj
 0001:00011ee0       _BotWriteInterbreeded      20012ee0 f   ai_main.obj
 0001:00012140       _BotInterbreedEndMatch     20013140 f   ai_main.obj
 0001:000121c0       _BotEntityInfo             200131c0 f   ai_main.obj
 0001:000121d0       _NumBots                   200131d0 f   ai_main.obj
 0001:000121e0       _BotTeamLeader             200131e0 f   ai_main.obj
 0001:00012210       _BotChangeViewAngle        20013210 f   ai_main.obj
 0001:000122e0       _BotChangeViewAngles       200132e0 f   ai_main.obj
 0001:00012570       _BotInputToUserCommand     20013570 f   ai_main.obj
 0001:000127e0       _BotUpdateInput            200137e0 f   ai_main.obj
 0001:000128c0       _RemoveColorEscapeSequences 200138c0 f   ai_main.obj
 0001:00012910       _BotAI                     20013910 f   ai_main.obj
 0001:00012c30       _BotScheduleBotThink       20013c30 f   ai_main.obj
 0001:00012cd0       _BotWriteSessionData       20013cd0 f   ai_main.obj
 0001:00012da0       _BotReadSessionData        20013da0 f   ai_main.obj
 0001:00012e60       _BotAISetupClient          20013e60 f   ai_main.obj
 0001:000131a0       _BotAIShutdownClient       200141a0 f   ai_main.obj
 0001:00013280       _BotResetState             20014280 f   ai_main.obj
 0001:00013400       _BotAILoadMap              20014400 f   ai_main.obj
 0001:00013480       _BotInitLibrary            20014480 f   ai_main.obj
 0001:000138e0       _BotAISetup                200148e0 f   ai_main.obj
 0001:00013a40       _BotAIShutdown             20014a40 f   ai_main.obj
 0001:00013a90       _BotInterbreeding          20014a90 f   ai_main.obj
 0001:00013b80       _BotAIStartFrame           20014b80 f   ai_main.obj
 0001:00014070       _BotNumTeamMates           20015070 f   ai_team.obj
 0001:00014150       _BotClientTravelTimeToGoal 20015150 f   ai_team.obj
 0001:000141b0       _BotSortTeamMatesByBaseTravelTime 200151b0 f   ai_team.obj
 0001:00014380       _BotSetTeamMateTaskPreference 20015380 f   ai_team.obj
 0001:000143d0       _BotGetTeamMateTaskPreference 200153d0 f   ai_team.obj
 0001:00014420       _BotSortTeamMatesByTaskPreference 20015420 f   ai_team.obj
 0001:00014530       _BotSayTeamOrderAlways     20015530 f   ai_team.obj
 0001:000145d0       _BotCTFOrders_BothFlagsNotAtBase 200155d0 f   ai_team.obj
 0001:000148c0       _BotCTFOrders_FlagNotAtBase 200158c0 f   ai_team.obj
 0001:00014cb0       _BotCTFOrders_EnemyFlagNotAtBase 20015cb0 f   ai_team.obj
 0001:00014f60       _BotCTFOrders_BothFlagsAtBase 20015f60 f   ai_team.obj
 0001:00015350       _BotCTFOrders              20016350 f   ai_team.obj
 0001:000153d0       _BotCreateGroup            200163d0 f   ai_team.obj
 0001:00015470       _BotTeamOrders             20016470 f   ai_team.obj
 0001:00015610       _FindHumanTeamLeader       20016610 f   ai_team.obj
 0001:00015690       _BotTeamAI                 20016690 f   ai_team.obj
 0001:00015a40       _BotVoiceChat_GetFlag      20016a40 f   ai_vcmd.obj
 0001:00015b00       _BotVoiceChat_Offense      20016b00 f   ai_vcmd.obj
 0001:00015ba0       _BotVoiceChat_Defend       20016ba0 f   ai_vcmd.obj
 0001:00015c70       _BotVoiceChat_DefendFlag   20016c70 f   ai_vcmd.obj
 0001:00015c80       _BotVoiceChat_Patrol       20016c80 f   ai_vcmd.obj
 0001:00015ce0       _BotVoiceChat_Camp         20016ce0 f   ai_vcmd.obj
 0001:00015e50       _BotVoiceChat_FollowMe     20016e50 f   ai_vcmd.obj
 0001:00015fe0       _BotVoiceChat_FollowFlagCarrier 20016fe0 f   ai_vcmd.obj
 0001:00016010       _BotVoiceChat_ReturnFlag   20017010 f   ai_vcmd.obj
 0001:000160a0       _BotVoiceChat_StartLeader  200170a0 f   ai_vcmd.obj
 0001:000160c0       _BotVoiceChat_StopLeader   200170c0 f   ai_vcmd.obj
 0001:00016110       _BotVoiceChat_WhoIsLeader  20017110 f   ai_vcmd.obj
 0001:00016190       _BotVoiceChat_WantOnDefense 20017190 f   ai_vcmd.obj
 0001:00016210       _BotVoiceChat_WantOnOffense 20017210 f   ai_vcmd.obj
 0001:00016290       _BotVoiceChat_Dummy        20017290 f   ai_vcmd.obj
 0001:00016290       _BotVoiceChat              20017290 f   ai_team.obj
 0001:00016290       _SP_team_CTF_redspawn      20017290 f   g_team.obj
 0001:00016290       _SP_team_CTF_blueplayer    20017290 f   g_team.obj
 0001:00016290       _SP_team_CTF_bluespawn     20017290 f   g_team.obj
 0001:00016290       _SP_misc_teleporter_dest   20017290 f   g_misc.obj
 0001:00016290       _SP_team_CTF_redplayer     20017290 f   g_team.obj
 0001:00016290       _SP_item_botroam           20017290 f   g_spawn.obj
 0001:00016290       _BotVoiceChatOnly          20017290 f   ai_team.obj
 0001:00016290       _SP_info_player_intermission 20017290 f   g_client.obj
 0001:00016290       _BotSetTeamStatus          20017290 f   ai_dmq3.obj
 0001:000162a0       _BG_FindItemForPowerup     200172a0 f   bg_misc.obj
 0001:000162f0       _BG_FindItemForWeapon      200172f0 f   bg_misc.obj
 0001:00016340       _BG_FindItem               20017340 f   bg_misc.obj
 0001:00016380       _BG_CanItemBeGrabbed       20017380 f   bg_misc.obj
 0001:00016510       _BG_EvaluateTrajectory     20017510 f   bg_misc.obj
 0001:00016650       _BG_EvaluateTrajectoryDelta 20017650 f   bg_misc.obj
 0001:00016740       _BG_AddPredictableEventToPlayerstate 20017740 f   bg_misc.obj
 0001:00016770       _BG_TouchJumpPad           20017770 f   bg_misc.obj
 0001:00016820       _BG_PlayerStateToEntityState 20017820 f   bg_misc.obj
 0001:00016a90       _BG_PlayerStateToEntityStateExtraPolate 20017a90 f   bg_misc.obj
 0001:00016d10       _BG_PlayerTouchesItem      20017d10 f   bg_misc.obj
 0001:00016db0       _PM_AddEvent               20017db0 f   bg_pmove.obj
 0001:00016dd0       _PM_AddTouchEnt            20017dd0 f   bg_pmove.obj
 0001:00016eb0       _PM_ClipVelocity           20017eb0 f   bg_pmove.obj
 0001:000192f0       _PM_UpdateViewAngles       2001a2f0 f   bg_pmove.obj
 0001:000193c0       _PmoveSingle               2001a3c0 f   bg_pmove.obj
 0001:00019720       _Pmove                     2001a720 f   bg_pmove.obj
 0001:000197b0       _PM_SlideMove              2001a7b0 f   bg_slidemove.obj
 0001:00019ea0       _PM_StepSlideMove          2001aea0 f   bg_slidemove.obj
 0001:0001a1f0       _P_DamageFeedback          2001b1f0 f   g_active.obj
 0001:0001a320       _P_WorldEffects            2001b320 f   g_active.obj
 0001:0001a4d0       _ClientImpacts             2001b4d0 f   g_active.obj
 0001:0001a570       _G_TouchTriggers           2001b570 f   g_active.obj
 0001:0001a780       _SpectatorThink            2001b780 f   g_active.obj
 0001:0001a870       _ClientInactivityTimer     2001b870 f   g_active.obj
 0001:0001a980       _ClientTimerActions        2001b980 f   g_active.obj
 0001:0001aaa0       _ClientIntermissionThink   2001baa0 f   g_active.obj
 0001:0001aae0       _ClientEvents              2001bae0 f   g_active.obj
 0001:0001acd0       _SendPendingPredictableEvents 2001bcd0 f   g_active.obj
 0001:0001ad80       _ClientThink_real          2001bd80 f   g_active.obj
 0001:0001b280       _ClientThink               2001c280 f   g_active.obj
 0001:0001b2e0       _G_RunClient               2001c2e0 f   g_active.obj
 0001:0001b320       _SpectatorClientEndFrame   2001c320 f   g_active.obj
 0001:0001b430       _ClientEndFrame            2001c430 f   g_active.obj
 0001:0001b5c0       _UpdateTournamentInfo      2001c5c0 f   g_arenas.obj
 0001:0001c070       _SpawnModelsOnVictoryPads  2001d070 f   g_arenas.obj
 0001:0001c190       _Svcmd_AbortPodium_f       2001d190 f   g_arenas.obj
 0001:0001c1c0       _G_ParseInfos              2001d1c0 f   g_bot.obj
 0001:0001c5b0       _G_GetArenaInfoByMap       2001d5b0 f   g_bot.obj
 0001:0001c670       _G_AddRandomBot            2001d670 f   g_bot.obj
 0001:0001c8e0       _G_RemoveRandomBot         2001d8e0 f   g_bot.obj
 0001:0001c980       _G_CountHumanPlayers       2001d980 f   g_bot.obj
 0001:0001c9e0       _G_CountBotPlayers         2001d9e0 f   g_bot.obj
 0001:0001ca80       _G_CheckMinimumPlayers     2001da80 f   g_bot.obj
 0001:0001cc00       _G_CheckBotSpawn           2001dc00 f   g_bot.obj
 0001:0001ccd0       _G_RemoveQueuedBotBegin    2001dcd0 f   g_bot.obj
 0001:0001cd00       _G_BotConnect              2001dd00 f   g_bot.obj
 0001:0001cde0       _Svcmd_BotList_f           2001dde0 f   g_bot.obj
 0001:0001d300       _G_GetBotInfoByName        2001e300 f   g_bot.obj
 0001:0001d350       _G_InitBots                2001e350 f   g_bot.obj
 0001:0001d880       _Svcmd_AddBot_f            2001e880 f   g_bot.obj
 0001:0001d9d0       _SP_info_player_deathmatch 2001e9d0 f   g_client.obj
 0001:0001da30       _SP_info_player_start      2001ea30 f   g_client.obj
 0001:0001da50       _SpotWouldTelefrag         2001ea50 f   g_client.obj
 0001:0001db10       _SelectRandomFurthestSpawnPoint 2001eb10 f   g_client.obj
 0001:0001ddd0       _SelectSpawnPoint          2001edd0 f   g_client.obj
 0001:0001dde0       _SelectInitialSpawnPoint   2001ede0 f   g_client.obj
 0001:0001de80       _InitBodyQue               2001ee80 f   g_client.obj
 0001:0001dec0       _BodySink                  2001eec0 f   g_client.obj
 0001:0001df10       _CopyToBodyQue             2001ef10 f   g_client.obj
 0001:0001e170       _SetClientViewAngle        2001f170 f   g_client.obj
 0001:0001e220       _TeamCount                 2001f220 f   g_client.obj
 0001:0001e270       _TeamLeader                2001f270 f   g_client.obj
 0001:0001e2c0       _PickTeam                  2001f2c0 f   g_client.obj
 0001:0001e3c0       _ClientUserinfoChanged     2001f3c0 f   g_client.obj
 0001:0001e8c0       _ClientConnect             2001f8c0 f   g_client.obj
 0001:0001eac0       _ClientSpawn               2001fac0 f   g_client.obj
 0001:0001f0f0       _ClientDisconnect          200200f0 f   g_client.obj
 0001:0001f290       _respawn                   20020290 f   g_client.obj
 0001:0001f2d0       _ClientBegin               200202d0 f   g_client.obj
 0001:0001f3c0       _DeathmatchScoreboardMessage 200203c0 f   g_cmds.obj
 0001:0001f590       _Cmd_Score_f               20020590 f   g_cmds.obj
 0001:0001f5a0       _CheatsOk                  200205a0 f   g_cmds.obj
 0001:0001f620       _ConcatArgs                20020620 f   g_cmds.obj
 0001:0001f6d0       _SanitizeString            200206d0 f   g_cmds.obj
 0001:0001f720       _ClientNumberFromString    20020720 f   g_cmds.obj
 0001:0001f8d0       _Cmd_Give_f                200208d0 f   g_cmds.obj
 0001:0001fb30       _Cmd_God_f                 20020b30 f   g_cmds.obj
 0001:0001fb90       _Cmd_Notarget_f            20020b90 f   g_cmds.obj
 0001:0001fbf0       _Cmd_Noclip_f              20020bf0 f   g_cmds.obj
 0001:0001fc60       _Cmd_LevelShot_f           20020c60 f   g_cmds.obj
 0001:0001fcd0       _Cmd_TeamTask_f            20020cd0 f   g_cmds.obj
 0001:0001fd70       _Cmd_Kill_f                20020d70 f   g_cmds.obj
 0001:0001fdc0       _BroadcastTeamChange       20020dc0 f   g_cmds.obj
 0001:0001fe40       _SetTeam                   20020e40 f   g_cmds.obj
 0001:00020170       _StopFollowing             20021170 f   g_cmds.obj
 0001:000201e0       _Cmd_Team_f                200211e0 f   g_cmds.obj
 0001:00020360       _Cmd_Follow_f              20021360 f   g_cmds.obj
 0001:00020460       _Cmd_FollowCycle_f         20021460 f   g_cmds.obj
 0001:00020600       _G_Say                     20021600 f   g_cmds.obj
 0001:000209e0       _G_Voice                   200219e0 f   g_cmds.obj
 0001:00020d70       _Cmd_GameCommand_f         20021d70 f   g_cmds.obj
 0001:00020e10       _Cmd_Where_f               20021e10 f   g_cmds.obj
 0001:00020e50       _Cmd_CallVote_f            20021e50 f   g_cmds.obj
 0001:00021410       _Cmd_Vote_f                20022410 f   g_cmds.obj
 0001:00021560       _Cmd_CallTeamVote_f        20022560 f   g_cmds.obj
 0001:00021b10       _Cmd_TeamVote_f            20022b10 f   g_cmds.obj
 0001:00021c70       _Cmd_SetViewpos_f          20022c70 f   g_cmds.obj
 0001:00021d90       _ClientCommand             20022d90 f   g_cmds.obj
 0001:00022450       _AddScore                  20023450 f   g_combat.obj
 0001:000224d0       _TossClientItems           200234d0 f   g_combat.obj
 0001:000225f0       _LookAtKiller              200235f0 f   g_combat.obj
 0001:00022680       _GibEntity                 20023680 f   g_combat.obj
 0001:00022710       _body_die                  20023710 f   g_combat.obj
 0001:00022740       _CheckAlmostCapture        20023740 f   g_combat.obj
 0001:00022830       _CheckAlmostScored         20023830 f   g_combat.obj
 0001:000228e0       _player_die                200238e0 f   g_combat.obj
 0001:00022dc0       _CheckArmor                20023dc0 f   g_combat.obj
 0001:00022e20       _G_Damage                  20023e20 f   g_combat.obj
 0001:00023280       _CanDamage                 20024280 f   g_combat.obj
 0001:000234c0       _G_RadiusDamage            200244c0 f   g_combat.obj
 0001:00023700       _Pickup_Powerup            20024700 f   g_items.obj
 0001:000238d0       _Pickup_Holdable           200248d0 f   g_items.obj
 0001:00023930       _Pickup_Ammo               20024930 f   g_items.obj
 0001:000239a0       _Pickup_Weapon             200249a0 f   g_items.obj
 0001:00023a90       _Pickup_Health             20024a90 f   g_items.obj
 0001:00023b10       _Pickup_Armor              20024b10 f   g_items.obj
 0001:00023b60       _RespawnItem               20024b60 f   g_items.obj
 0001:00023cc0       _Touch_Item                20024cc0 f   g_items.obj
 0001:00023fb0       _LaunchItem                20024fb0 f   g_items.obj
 0001:000240f0       _Drop_Item                 200250f0 f   g_items.obj
 0001:000241a0       _Use_Item                  200251a0 f   g_items.obj
 0001:000241b0       _FinishSpawningItem        200251b0 f   g_items.obj
 0001:000243a0       _G_CheckTeamItems          200253a0 f   g_items.obj
 0001:00024440       _RegisterItem              20025440 f   g_items.obj
 0001:00024480       _SaveRegisteredItems       20025480 f   g_items.obj
 0001:000244e0       _G_SpawnItem               200254e0 f   g_items.obj
 0001:000245e0       _G_BounceItem              200255e0 f   g_items.obj
 0001:00024760       _G_RunItem                 20025760 f   g_items.obj
 0001:000248a0       _ClearRegisteredItems      200258a0 f   g_items.obj
 0001:00024930       _G_Printf                  20025930 f   g_main.obj
 0001:00024960       _G_Error                   20025960 f   g_main.obj
 0001:00024990       _G_FindTeams               20025990 f   g_main.obj
 0001:00024b10       _G_RegisterCvars           20025b10 f   g_main.obj
 0001:00024ba0       _G_UpdateCvars             20025ba0 f   g_main.obj
 0001:00024c10       _Com_Error                 20025c10 f   g_main.obj
 0001:00024c50       _Com_Printf                20025c50 f   g_main.obj
 0001:00024c90       _AddTournamentPlayer       20025c90 f   g_main.obj
 0001:00024d50       _RemoveTournamentLoser     20025d50 f   g_main.obj
 0001:00024da0       _AdjustTournamentScores    20025da0 f   g_main.obj
 0001:00024e10       _SortRanks                 20025e10 f   g_main.obj
 0001:00024ef0       _SendScoreboardMessageToAllClients 20025ef0 f   g_main.obj
 0001:00024f50       _MoveClientToIntermission  20025f50 f   g_main.obj
 0001:00025040       _FindIntermissionPoint     20026040 f   g_main.obj
 0001:00025100       _BeginIntermission         20026100 f   g_main.obj
 0001:00025190       _ExitLevel                 20026190 f   g_main.obj
 0001:00025290       _G_LogPrintf               20026290 f   g_main.obj
 0001:00025360       _LogExit                   20026360 f   g_main.obj
 0001:00025440       _CheckIntermissionExit     20026440 f   g_main.obj
 0001:00025580       _ScoreIsTied               20026580 f   g_main.obj
 0001:000255e0       _CheckExitRules            200265e0 f   g_main.obj
 0001:00025790       _CheckTournament           20026790 f   g_main.obj
 0001:000259b0       _CheckVote                 200269b0 f   g_main.obj
 0001:00025a70       _PrintTeam                 20026a70 f   g_main.obj
 0001:00025ac0       _SetLeader                 20026ac0 f   g_main.obj
 0001:00025bc0       _CheckTeamLeader           20026bc0 f   g_main.obj
 0001:00025c80       _CheckTeamVote             20026c80 f   g_main.obj
 0001:00025d70       _G_RunThink                20026d70 f   g_main.obj
 0001:00025dd0       _G_RunFrame                20026dd0 f   g_main.obj
 0001:00026020       _G_InitGame                20027020 f   g_main.obj
 0001:00026260       _G_ShutdownGame            20027260 f   g_main.obj
 0001:000262c0       _CalculateRanks            200272c0 f   g_main.obj
 0001:000265e0       _vmMain                    200275e0 f   g_main.obj
 0001:000266e0       _G_Alloc                   200276e0 f   g_mem.obj
 0001:00026750       _G_InitMemory              20027750 f   g_mem.obj
 0001:00026760       _Svcmd_GameMem_f           20027760 f   g_mem.obj
 0001:00026780       _SP_target_position        20027780 f   g_target.obj
 0001:00026780       _SP_info_notnull           20027780 f   g_misc.obj
 0001:00026780       _SP_info_camp              20027780 f   g_misc.obj
 0001:000267a0       _TeleportPlayer            200277a0 f   g_misc.obj
 0001:00026900       _SP_misc_model             20027900 f   g_misc.obj
 0001:00026900       _SP_info_null              20027900 f   g_misc.obj
 0001:00026900       _SP_light                  20027900 f   g_misc.obj
 0001:00026910       _locateCamera              20027910 f   g_misc.obj
 0001:00026a20       _SP_misc_portal_surface    20027a20 f   g_misc.obj
 0001:00026aa0       _SP_misc_portal_camera     20027aa0 f   g_misc.obj
 0001:00026b00       _Use_Shooter               20027b00 f   g_misc.obj
 0001:00026d00       _InitShooter               20027d00 f   g_misc.obj
 0001:00026da0       _SP_shooter_rocket         20027da0 f   g_misc.obj
 0001:00026db0       _SP_shooter_plasma         20027db0 f   g_misc.obj
 0001:00026dc0       _SP_shooter_grenade        20027dc0 f   g_misc.obj
 0001:00026dd0       _G_ExplodeMissile          20027dd0 f   g_missile.obj
 0001:00026ee0       _fire_plasma               20027ee0 f   g_missile.obj
 0001:00027030       _fire_grenade              20028030 f   g_missile.obj
 0001:00027190       _fire_bfg                  20028190 f   g_missile.obj
 0001:000272f0       _fire_rocket               200282f0 f   g_missile.obj
 0001:00027450       _fire_grapple              20028450 f   g_missile.obj
 0001:000275a0       _G_BounceMissile           200285a0 f   g_missile.obj
 0001:00027700       _G_MissileImpact           20028700 f   g_missile.obj
 0001:00027ae0       _G_RunMissile              20028ae0 f   g_missile.obj
 0001:00027c30       _G_TestEntityPosition      20028c30 f   g_mover.obj
 0001:00027ca0       _SetMoverState             20028ca0 f   g_mover.obj
 0001:00027e10       _MatchTeam                 20028e10 f   g_mover.obj
 0001:00027e40       _ReturnToPos1              20028e40 f   g_mover.obj
 0001:00027f40       _Reached_BinaryMover       20028f40 f   g_mover.obj
 0001:000280b0       _Use_BinaryMover           200290b0 f   g_mover.obj
 0001:000281e0       _InitMover                 200291e0 f   g_mover.obj
 0001:00028420       _Blocked_Door              20029420 f   g_mover.obj
 0001:00028590       _Touch_DoorTrigger         20029590 f   g_mover.obj
 0001:000285f0       _Think_SpawnNewDoorTrigger 200295f0 f   g_mover.obj
 0001:000287a0       _Think_MatchTeam           200297a0 f   g_mover.obj
 0001:000287d0       _SP_func_door              200297d0 f   g_mover.obj
 0001:00028a30       _Touch_Plat                20029a30 f   g_mover.obj
 0001:00028a70       _Touch_PlatCenterTrigger   20029a70 f   g_mover.obj
 0001:00028ab0       _SpawnPlatTrigger          20029ab0 f   g_mover.obj
 0001:00028c00       _SP_func_plat              20029c00 f   g_mover.obj
 0001:00028d60       _Touch_Button              20029d60 f   g_mover.obj
 0001:00028d90       _SP_func_button            20029d90 f   g_mover.obj
 0001:00028f20       _Think_BeginMoving         20029f20 f   g_mover.obj
 0001:00028f40       _Reached_Train             20029f40 f   g_mover.obj
 0001:00029150       _Think_SetupTrainTargets   2002a150 f   g_mover.obj
 0001:00029230       _SP_path_corner            2002a230 f   g_mover.obj
 0001:00029260       _SP_func_train             2002a260 f   g_mover.obj
 0001:00029320       _SP_func_static            2002a320 f   g_mover.obj
 0001:00029370       _SP_func_rotating          2002a370 f   g_mover.obj
 0001:00029440       _SP_func_bobbing           2002a440 f   g_mover.obj
 0001:00029540       _SP_func_pendulum          2002a540 f   g_mover.obj
 0001:00029650       _G_TryPushingEntity        2002a650 f   g_mover.obj
 0001:00029a30       _G_MoverPush               2002aa30 f   g_mover.obj
 0001:00029f00       _G_MoverTeam               2002af00 f   g_mover.obj
 0001:0002a0a0       _G_RunMover                2002b0a0 f   g_mover.obj
 0001:0002a0e0       _G_WriteClientSessionData  2002b0e0 f   g_session.obj
 0001:0002a160       _G_ReadSessionData         2002b160 f   g_session.obj
 0001:0002a210       _G_InitSessionData         2002b210 f   g_session.obj
 0001:0002a2d0       _G_InitWorldSession        2002b2d0 f   g_session.obj
 0001:0002a320       _G_WriteSessionData        2002b320 f   g_session.obj
 0001:0002a380       _G_SpawnString             2002b380 f   g_spawn.obj
 0001:0002a3f0       _G_SpawnFloat              2002b3f0 f   g_spawn.obj
 0001:0002a420       _G_SpawnInt                2002b420 f   g_spawn.obj
 0001:0002a450       _G_SpawnVector             2002b450 f   g_spawn.obj
 0001:0002a490       _G_CallSpawn               2002b490 f   g_spawn.obj
 0001:0002a590       _G_NewString               2002b590 f   g_spawn.obj
 0001:0002a5f0       _G_ParseField              2002b5f0 f   g_spawn.obj
 0001:0002a730       _G_SpawnGEntityFromSpawnVars 2002b730 f   g_spawn.obj
 0001:0002a8b0       _G_AddSpawnVarToken        2002b8b0 f   g_spawn.obj
 0001:0002a920       _G_ParseSpawnVars          2002b920 f   g_spawn.obj
 0001:0002aa40       _SP_worldspawn             2002ba40 f   g_spawn.obj
 0001:0002abe0       _G_SpawnEntitiesFromString 2002bbe0 f   g_spawn.obj
 0001:0002ae20       _G_FilterPacket            2002be20 f   g_svcmds.obj
 0001:0002af40       _G_ProcessIPBans           2002bf40 f   g_svcmds.obj
 0001:0002afb0       _Svcmd_AddIP_f             2002bfb0 f   g_svcmds.obj
 0001:0002b000       _Svcmd_RemoveIP_f          2002c000 f   g_svcmds.obj
 0001:0002b0c0       _Svcmd_EntityList_f        2002c0c0 f   g_svcmds.obj
 0001:0002b250       _ClientForString           2002c250 f   g_svcmds.obj
 0001:0002b330       _Svcmd_ForceTeam_f         2002c330 f   g_svcmds.obj
 0001:0002b3b0       _ConsoleCommand            2002c3b0 f   g_svcmds.obj
 0001:0002b580       _dllEntry                  2002c580 f   g_syscalls.obj
 0001:0002b590       _trap_Printf               2002c590 f   g_syscalls.obj
 0001:0002b5b0       _trap_Error                2002c5b0 f   g_syscalls.obj
 0001:0002b5d0       _trap_Milliseconds         2002c5d0 f   g_syscalls.obj
 0001:0002b5e0       _trap_Argc                 2002c5e0 f   g_syscalls.obj
 0001:0002b5f0       _trap_Argv                 2002c5f0 f   g_syscalls.obj
 0001:0002b610       _trap_FS_FOpenFile         2002c610 f   g_syscalls.obj
 0001:0002b630       _trap_FS_Read              2002c630 f   g_syscalls.obj
 0001:0002b650       _trap_FS_Write             2002c650 f   g_syscalls.obj
 0001:0002b670       _trap_FS_FCloseFile        2002c670 f   g_syscalls.obj
 0001:0002b690       _trap_FS_GetFileList       2002c690 f   g_syscalls.obj
 0001:0002b6b0       _trap_SendConsoleCommand   2002c6b0 f   g_syscalls.obj
 0001:0002b6d0       _trap_Cvar_Register        2002c6d0 f   g_syscalls.obj
 0001:0002b6f0       _trap_Cvar_Update          2002c6f0 f   g_syscalls.obj
 0001:0002b710       _trap_Cvar_Set             2002c710 f   g_syscalls.obj
 0001:0002b730       _trap_Cvar_VariableIntegerValue 2002c730 f   g_syscalls.obj
 0001:0002b750       _trap_Cvar_VariableStringBuffer 2002c750 f   g_syscalls.obj
 0001:0002b770       _trap_LocateGameData       2002c770 f   g_syscalls.obj
 0001:0002b7a0       _trap_DropClient           2002c7a0 f   g_syscalls.obj
 0001:0002b7c0       _trap_SendServerCommand    2002c7c0 f   g_syscalls.obj
 0001:0002b7e0       _trap_SetConfigstring      2002c7e0 f   g_syscalls.obj
 0001:0002b800       _trap_GetConfigstring      2002c800 f   g_syscalls.obj
 0001:0002b820       _trap_GetUserinfo          2002c820 f   g_syscalls.obj
 0001:0002b840       _trap_SetUserinfo          2002c840 f   g_syscalls.obj
 0001:0002b860       _trap_GetServerinfo        2002c860 f   g_syscalls.obj
 0001:0002b880       _trap_SetBrushModel        2002c880 f   g_syscalls.obj
 0001:0002b8a0       _trap_Trace                2002c8a0 f   g_syscalls.obj
 0001:0002b8d0       _trap_PointContents        2002c8d0 f   g_syscalls.obj
 0001:0002b8f0       _trap_InPVS                2002c8f0 f   g_syscalls.obj
 0001:0002b910       _trap_AdjustAreaPortalState 2002c910 f   g_syscalls.obj
 0001:0002b930       _trap_LinkEntity           2002c930 f   g_syscalls.obj
 0001:0002b950       _trap_UnlinkEntity         2002c950 f   g_syscalls.obj
 0001:0002b970       _trap_EntitiesInBox        2002c970 f   g_syscalls.obj
 0001:0002b990       _trap_EntityContact        2002c990 f   g_syscalls.obj
 0001:0002b9b0       _trap_BotAllocateClient    2002c9b0 f   g_syscalls.obj
 0001:0002b9c0       _trap_GetUsercmd           2002c9c0 f   g_syscalls.obj
 0001:0002b9e0       _trap_GetEntityToken       2002c9e0 f   g_syscalls.obj
 0001:0002ba00       _trap_SnapVector           2002ca00 f   g_syscalls.obj
 0001:0002ba20       _trap_BotLibSetup          2002ca20 f   g_syscalls.obj
 0001:0002ba30       _trap_BotLibShutdown       2002ca30 f   g_syscalls.obj
 0001:0002ba40       _trap_BotLibVarSet         2002ca40 f   g_syscalls.obj
 0001:0002ba60       _trap_BotLibStartFrame     2002ca60 f   g_syscalls.obj
 0001:0002ba80       _trap_BotLibLoadMap        2002ca80 f   g_syscalls.obj
 0001:0002baa0       _trap_BotLibUpdateEntity   2002caa0 f   g_syscalls.obj
 0001:0002bac0       _trap_BotGetSnapshotEntity 2002cac0 f   g_syscalls.obj
 0001:0002bae0       _trap_BotGetServerCommand  2002cae0 f   g_syscalls.obj
 0001:0002bb00       _trap_BotUserCommand       2002cb00 f   g_syscalls.obj
 0001:0002bb20       _trap_AAS_EntityInfo       2002cb20 f   g_syscalls.obj
 0001:0002bb40       _trap_AAS_Initialized      2002cb40 f   g_syscalls.obj
 0001:0002bb50       _trap_AAS_PresenceTypeBoundingBox 2002cb50 f   g_syscalls.obj
 0001:0002bb70       _trap_AAS_Time             2002cb70 f   g_syscalls.obj
 0001:0002bb90       _trap_AAS_PointAreaNum     2002cb90 f   g_syscalls.obj
 0001:0002bbb0       _trap_AAS_TraceAreas       2002cbb0 f   g_syscalls.obj
 0001:0002bbe0       _trap_AAS_BBoxAreas        2002cbe0 f   g_syscalls.obj
 0001:0002bc10       _trap_AAS_AreaInfo         2002cc10 f   g_syscalls.obj
 0001:0002bc30       _trap_AAS_PointContents    2002cc30 f   g_syscalls.obj
 0001:0002bc50       _trap_AAS_NextBSPEntity    2002cc50 f   g_syscalls.obj
 0001:0002bc70       _trap_AAS_ValueForBSPEpairKey 2002cc70 f   g_syscalls.obj
 0001:0002bca0       _trap_AAS_VectorForBSPEpairKey 2002cca0 f   g_syscalls.obj
 0001:0002bcc0       _trap_AAS_FloatForBSPEpairKey 2002ccc0 f   g_syscalls.obj
 0001:0002bce0       _trap_AAS_IntForBSPEpairKey 2002cce0 f   g_syscalls.obj
 0001:0002bd00       _trap_AAS_AreaReachability 2002cd00 f   g_syscalls.obj
 0001:0002bd20       _trap_AAS_AreaTravelTimeToGoalArea 2002cd20 f   g_syscalls.obj
 0001:0002bd50       _trap_AAS_EnableRoutingArea 2002cd50 f   g_syscalls.obj
 0001:0002bd70       _trap_AAS_PredictRoute     2002cd70 f   g_syscalls.obj
 0001:0002bdc0       _trap_AAS_Swimming         2002cdc0 f   g_syscalls.obj
 0001:0002bde0       _trap_AAS_PredictClientMovement 2002cde0 f   g_syscalls.obj
 0001:0002be40       _trap_EA_SayTeam           2002ce40 f   g_syscalls.obj
 0001:0002be60       _trap_EA_Command           2002ce60 f   g_syscalls.obj
 0001:0002be80       _trap_EA_Action            2002ce80 f   g_syscalls.obj
 0001:0002bea0       _trap_EA_Gesture           2002cea0 f   g_syscalls.obj
 0001:0002bec0       _trap_EA_Talk              2002cec0 f   g_syscalls.obj
 0001:0002bee0       _trap_EA_Attack            2002cee0 f   g_syscalls.obj
 0001:0002bf00       _trap_EA_Use               2002cf00 f   g_syscalls.obj
 0001:0002bf20       _trap_EA_Respawn           2002cf20 f   g_syscalls.obj
 0001:0002bf40       _trap_EA_Crouch            2002cf40 f   g_syscalls.obj
 0001:0002bf60       _trap_EA_SelectWeapon      2002cf60 f   g_syscalls.obj
 0001:0002bf80       _trap_EA_View              2002cf80 f   g_syscalls.obj
 0001:0002bfa0       _trap_EA_GetInput          2002cfa0 f   g_syscalls.obj
 0001:0002bfd0       _trap_EA_ResetInput        2002cfd0 f   g_syscalls.obj
 0001:0002bff0       _trap_BotLoadCharacter     2002cff0 f   g_syscalls.obj
 0001:0002c010       _trap_BotFreeCharacter     2002d010 f   g_syscalls.obj
 0001:0002c030       _trap_Characteristic_BFloat 2002d030 f   g_syscalls.obj
 0001:0002c070       _trap_Characteristic_BInteger 2002d070 f   g_syscalls.obj
 0001:0002c0a0       _trap_Characteristic_String 2002d0a0 f   g_syscalls.obj
 0001:0002c0d0       _trap_BotAllocChatState    2002d0d0 f   g_syscalls.obj
 0001:0002c0e0       _trap_BotFreeChatState     2002d0e0 f   g_syscalls.obj
 0001:0002c100       _trap_BotQueueConsoleMessage 2002d100 f   g_syscalls.obj
 0001:0002c120       _trap_BotRemoveConsoleMessage 2002d120 f   g_syscalls.obj
 0001:0002c140       _trap_BotNextConsoleMessage 2002d140 f   g_syscalls.obj
 0001:0002c160       _trap_BotNumConsoleMessages 2002d160 f   g_syscalls.obj
 0001:0002c180       _trap_BotInitialChat       2002d180 f   g_syscalls.obj
 0001:0002c1d0       _trap_BotNumInitialChats   2002d1d0 f   g_syscalls.obj
 0001:0002c1f0       _trap_BotReplyChat         2002d1f0 f   g_syscalls.obj
 0001:0002c240       _trap_BotEnterChat         2002d240 f   g_syscalls.obj
 0001:0002c260       _trap_BotGetChatMessage    2002d260 f   g_syscalls.obj
 0001:0002c280       _trap_BotFindMatch         2002d280 f   g_syscalls.obj
 0001:0002c2a0       _trap_BotMatchVariable     2002d2a0 f   g_syscalls.obj
 0001:0002c2d0       _trap_UnifyWhiteSpaces     2002d2d0 f   g_syscalls.obj
 0001:0002c2f0       _trap_BotReplaceSynonyms   2002d2f0 f   g_syscalls.obj
 0001:0002c310       _trap_BotLoadChatFile      2002d310 f   g_syscalls.obj
 0001:0002c330       _trap_BotSetChatGender     2002d330 f   g_syscalls.obj
 0001:0002c350       _trap_BotSetChatName       2002d350 f   g_syscalls.obj
 0001:0002c370       _trap_BotResetGoalState    2002d370 f   g_syscalls.obj
 0001:0002c390       _trap_BotResetAvoidGoals   2002d390 f   g_syscalls.obj
 0001:0002c3b0       _trap_BotRemoveFromAvoidGoals 2002d3b0 f   g_syscalls.obj
 0001:0002c3d0       _trap_BotPushGoal          2002d3d0 f   g_syscalls.obj
 0001:0002c3f0       _trap_BotPopGoal           2002d3f0 f   g_syscalls.obj
 0001:0002c410       _trap_BotEmptyGoalStack    2002d410 f   g_syscalls.obj
 0001:0002c430       _trap_BotDumpAvoidGoals    2002d430 f   g_syscalls.obj
 0001:0002c450       _trap_BotDumpGoalStack     2002d450 f   g_syscalls.obj
 0001:0002c470       _trap_BotGoalName          2002d470 f   g_syscalls.obj
 0001:0002c490       _trap_BotGetTopGoal        2002d490 f   g_syscalls.obj
 0001:0002c4b0       _trap_BotGetSecondGoal     2002d4b0 f   g_syscalls.obj
 0001:0002c4d0       _trap_BotChooseLTGItem     2002d4d0 f   g_syscalls.obj
 0001:0002c500       _trap_BotChooseNBGItem     2002d500 f   g_syscalls.obj
 0001:0002c540       _trap_BotTouchingGoal      2002d540 f   g_syscalls.obj
 0001:0002c560       _trap_BotItemGoalInVisButNotVisible 2002d560 f   g_syscalls.obj
 0001:0002c590       _trap_BotGetLevelItemGoal  2002d590 f   g_syscalls.obj
 0001:0002c5b0       _trap_BotGetNextCampSpotGoal 2002d5b0 f   g_syscalls.obj
 0001:0002c5d0       _trap_BotSetAvoidGoalTime  2002d5d0 f   g_syscalls.obj
 0001:0002c600       _trap_BotUpdateEntityItems 2002d600 f   g_syscalls.obj
 0001:0002c610       _trap_BotLoadItemWeights   2002d610 f   g_syscalls.obj
 0001:0002c630       _trap_BotInterbreedGoalFuzzyLogic 2002d630 f   g_syscalls.obj
 0001:0002c650       _trap_BotSaveGoalFuzzyLogic 2002d650 f   g_syscalls.obj
 0001:0002c670       _trap_BotMutateGoalFuzzyLogic 2002d670 f   g_syscalls.obj
 0001:0002c690       _trap_BotAllocGoalState    2002d690 f   g_syscalls.obj
 0001:0002c6b0       _trap_BotFreeGoalState     2002d6b0 f   g_syscalls.obj
 0001:0002c6d0       _trap_BotResetMoveState    2002d6d0 f   g_syscalls.obj
 0001:0002c6f0       _trap_BotAddAvoidSpot      2002d6f0 f   g_syscalls.obj
 0001:0002c720       _trap_BotMoveToGoal        2002d720 f   g_syscalls.obj
 0001:0002c750       _trap_BotMoveInDirection   2002d750 f   g_syscalls.obj
 0001:0002c780       _trap_BotResetAvoidReach   2002d780 f   g_syscalls.obj
 0001:0002c7a0       _trap_BotResetLastAvoidReach 2002d7a0 f   g_syscalls.obj
 0001:0002c7c0       _trap_BotMovementViewTarget 2002d7c0 f   g_syscalls.obj
 0001:0002c7f0       _trap_BotPredictVisiblePosition 2002d7f0 f   g_syscalls.obj
 0001:0002c820       _trap_BotAllocMoveState    2002d820 f   g_syscalls.obj
 0001:0002c830       _trap_BotFreeMoveState     2002d830 f   g_syscalls.obj
 0001:0002c850       _trap_BotInitMoveState     2002d850 f   g_syscalls.obj
 0001:0002c870       _trap_BotChooseBestFightWeapon 2002d870 f   g_syscalls.obj
 0001:0002c890       _trap_BotGetWeaponInfo     2002d890 f   g_syscalls.obj
 0001:0002c8b0       _trap_BotLoadWeaponWeights 2002d8b0 f   g_syscalls.obj
 0001:0002c8d0       _trap_BotAllocWeaponState  2002d8d0 f   g_syscalls.obj
 0001:0002c8e0       _trap_BotFreeWeaponState   2002d8e0 f   g_syscalls.obj
 0001:0002c900       _trap_BotResetWeaponState  2002d900 f   g_syscalls.obj
 0001:0002c920       _trap_GeneticParentsAndChildSelection 2002d920 f   g_syscalls.obj
 0001:0002c950       _Use_Target_Give           2002d950 f   g_target.obj
 0001:0002c9f0       _SP_target_give            2002d9f0 f   g_target.obj
 0001:0002ca00       _Use_target_remove_powerups 2002da00 f   g_target.obj
 0001:0002ca60       _SP_target_remove_powerups 2002da60 f   g_target.obj
 0001:0002ca70       _Think_Target_Delay        2002da70 f   g_target.obj
 0001:0002ca90       _Use_Target_Delay          2002da90 f   g_target.obj
 0001:0002caf0       _SP_target_delay           2002daf0 f   g_target.obj
 0001:0002cb50       _Use_Target_Score          2002db50 f   g_target.obj
 0001:0002cb70       _SP_target_score           2002db70 f   g_target.obj
 0001:0002cba0       _Use_Target_Print          2002dba0 f   g_target.obj
 0001:0002cc70       _SP_target_print           2002dc70 f   g_target.obj
 0001:0002cc80       _Use_Target_Speaker        2002dc80 f   g_target.obj
 0001:0002cd10       _SP_target_speaker         2002dd10 f   g_target.obj
 0001:0002ce60       _target_laser_think        2002de60 f   g_target.obj
 0001:0002cfd0       _target_laser_use          2002dfd0 f   g_target.obj
 0001:0002d020       _target_laser_start        2002e020 f   g_target.obj
 0001:0002d100       _SP_target_laser           2002e100 f   g_target.obj
 0001:0002d120       _target_teleporter_use     2002e120 f   g_target.obj
 0001:0002d170       _SP_target_teleporter      2002e170 f   g_target.obj
 0001:0002d1b0       _target_relay_use          2002e1b0 f   g_target.obj
 0001:0002d230       _SP_target_relay           2002e230 f   g_target.obj
 0001:0002d240       _target_kill_use           2002e240 f   g_target.obj
 0001:0002d260       _SP_target_kill            2002e260 f   g_target.obj
 0001:0002d320       _SP_target_location        2002e320 f   g_target.obj
 0001:0002d350       _TeamName                  2002e350 f   g_team.obj
 0001:0002d3b0       _PrintMsg                  2002e3b0 f   g_team.obj
 0001:0002d460       _AddTeamScore              2002e460 f   g_team.obj
 0001:0002d560       _OnSameTeam                2002e560 f   g_team.obj
 0001:0002d5a0       _Team_SetFlagStatus        2002e5a0 f   g_team.obj
 0001:0002d650       _Team_CheckDroppedItem     2002e650 f   g_team.obj
 0001:0002d760       _Team_ForceGesture         2002e760 f   g_team.obj
 0001:0002d800       _Team_FragBonuses          2002e800 f   g_team.obj
 0001:0002dd90       _Team_CheckHurtCarrier     2002ed90 f   g_team.obj
 0001:0002de20       _Team_ResetFlag            2002ee20 f   g_team.obj
 0001:0002deb0       _Team_TakeFlagSound        2002eeb0 f   g_team.obj
 0001:0002df50       _Team_CaptureFlagSound     2002ef50 f   g_team.obj
 0001:0002df90       _Team_ReturnFlag           2002ef90 f   g_team.obj
 0001:0002e050       _Team_FreeEntity           2002f050 f   g_team.obj
 0001:0002e180       _Team_DroppedFlagThink     2002f180 f   g_team.obj
 0001:0002e200       _Team_TouchOurFlag         2002f200 f   g_team.obj
 0001:0002e530       _Team_TouchEnemyFlag       2002f530 f   g_team.obj
 0001:0002e5e0       _Pickup_Team               2002f5e0 f   g_team.obj
 0001:0002e670       _Team_GetLocation          2002f670 f   g_team.obj
 0001:0002e730       _Team_GetLocationMsg       2002f730 f   g_team.obj
 0001:0002e7d0       _SelectRandomTeamSpawnPoint 2002f7d0 f   g_team.obj
 0001:0002e8a0       _SelectCTFSpawnPoint       2002f8a0 f   g_team.obj
 0001:0002e910       _TeamplayInfoMessage       2002f910 f   g_team.obj
 0001:0002eaf0       _CheckTeamStatus           2002faf0 f   g_team.obj
 0001:0002ebf0       _Team_InitGame             2002fbf0 f   g_team.obj
 0001:0002ecf0       _multi_wait                2002fcf0 f   g_trigger.obj
 0001:0002ed00       _multi_trigger             2002fd00 f   g_trigger.obj
 0001:0002edf0       _Use_Multi                 2002fdf0 f   g_trigger.obj
 0001:0002ee10       _Touch_Multi               2002fe10 f   g_trigger.obj
 0001:0002ee30       _trigger_always_think      2002fe30 f   g_trigger.obj
 0001:0002ee50       _SP_trigger_always         2002fe50 f   g_trigger.obj
 0001:0002ee70       _trigger_push_touch        2002fe70 f   g_trigger.obj
 0001:0002ee90       _AimAtTarget               2002fe90 f   g_trigger.obj
 0001:0002ef90       _Use_target_push           2002ff90 f   g_trigger.obj
 0001:0002f010       _SP_target_push            20030010 f   g_trigger.obj
 0001:0002f0f0       _trigger_teleporter_touch  200300f0 f   g_trigger.obj
 0001:0002f160       _hurt_use                  20030160 f   g_trigger.obj
 0001:0002f180       _hurt_touch                20030180 f   g_trigger.obj
 0001:0002f200       _func_timer_think          20030200 f   g_trigger.obj
 0001:0002f260       _func_timer_use            20030260 f   g_trigger.obj
 0001:0002f290       _SP_func_timer             20030290 f   g_trigger.obj
 0001:0002f340       _InitTrigger               20030340 f   g_trigger.obj
 0001:0002f3c0       _SP_trigger_multiple       200303c0 f   g_trigger.obj
 0001:0002f450       _SP_trigger_push           20030450 f   g_trigger.obj
 0001:0002f4b0       _SP_trigger_teleport       200304b0 f   g_trigger.obj
 0001:0002f510       _SP_trigger_hurt           20030510 f   g_trigger.obj
 0001:0002f580       _AddRemap                  20030580 f   g_utils.obj
 0001:0002f640       _BuildShaderStateConfig    20030640 f   g_utils.obj
 0001:0002f6d0       _G_FindConfigstringIndex   200306d0 f   g_utils.obj
 0001:0002f7c0       _G_ModelIndex              200307c0 f   g_utils.obj
 0001:0002f7e0       _G_SoundIndex              200307e0 f   g_utils.obj
 0001:0002f800       _G_TeamCommand             20030800 f   g_utils.obj
 0001:0002f870       _G_Find                    20030870 f   g_utils.obj
 0001:0002f900       _G_PickTarget              20030900 f   g_utils.obj
 0001:0002f990       _G_UseTargets              20030990 f   g_utils.obj
 0001:0002fa60       _vtos                      20030a60 f   g_utils.obj
 0001:0002fab0       _G_SetMovedir              20030ab0 f   g_utils.obj
 0001:0002fb90       _vectoyaw                  20030b90 f   g_utils.obj
 0001:0002fc10       _G_InitGentity             20030c10 f   g_utils.obj
 0001:0002fc50       _G_Spawn                   20030c50 f   g_utils.obj
 0001:0002fd80       _G_FreeEntity              20030d80 f   g_utils.obj
 0001:0002fdd0       _G_KillBox                 20030dd0 f   g_utils.obj
 0001:0002fea0       _G_AddPredictableEvent     20030ea0 f   g_utils.obj
 0001:0002fed0       _G_AddEvent                20030ed0 f   g_utils.obj
 0001:0002ff80       _G_SetOrigin               20030f80 f   g_utils.obj
 0001:0002ffd0       _G_TempEntity              20030fd0 f   g_utils.obj
 0001:000300a0       _G_Sound                   200310a0 f   g_utils.obj
 0001:000300c0       _SnapVectorTowards         200310c0 f   g_weapon.obj
 0001:00030110       _BFG_Fire                  20031110 f   g_weapon.obj
 0001:00030160       _weapon_grenadelauncher_fire 20031160 f   g_weapon.obj
 0001:000301d0       _Weapon_RocketLauncher_Fire 200311d0 f   g_weapon.obj
 0001:00030220       _Weapon_Plasmagun_Fire     20031220 f   g_weapon.obj
 0001:00030270       _Weapon_GrapplingHook_Fire 20031270 f   g_weapon.obj
 0001:000302e0       _Weapon_HookFree           200312e0 f   g_weapon.obj
 0001:00030320       _Weapon_HookThink          20031320 f   g_weapon.obj
 0001:00030410       _LogAccuracyHit            20031410 f   g_weapon.obj
 0001:00030460       _CalcMuzzlePoint           20031460 f   g_weapon.obj
 0001:00030500       _CalcMuzzlePointOrigin     20031500 f   g_weapon.obj
 0001:000305a0       _CheckGauntletAttack       200315a0 f   g_weapon.obj
 0001:00030730       _Bullet_Fire               20031730 f   g_weapon.obj
 0001:00030960       _ShotgunPellet             20031960 f   g_weapon.obj
 0001:00030a30       _ShotgunPattern            20031a30 f   g_weapon.obj
 0001:00030ba0       _weapon_supershotgun_fire  20031ba0 f   g_weapon.obj
 0001:00030c50       _weapon_railgun_fire       20031c50 f   g_weapon.obj
 0001:00030f00       _Weapon_LightningFire      20031f00 f   g_weapon.obj
 0001:00031060       _FireWeapon                20032060 f   g_weapon.obj
 0001:000311c0       _Q_crandom                 200321c0 f   q_math.obj
 0001:000311f0       _DirToByte                 200321f0 f   q_math.obj
 0001:000313b0       _vectoangles               200323b0 f   q_math.obj
 0001:000314c0       _ProjectPointOnPlane       200324c0 f   q_math.obj
 0001:00031540       _AngleMod                  20032540 f   q_math.obj
 0001:00031570       _AngleNormalize180         20032570 f   q_math.obj
 0001:000315b0       _RadiusFromBounds          200325b0 f   q_math.obj
 0001:00031630       _AddPointToBounds          20032630 f   q_math.obj
 0001:000316b0       _VectorNormalize           200326b0 f   q_math.obj
 0001:00031710       _VectorNormalize2          20032710 f   q_math.obj
 0001:00031780       _AngleVectors              20032780 f   q_math.obj
 0001:000318c0       _PerpendicularVector       200328c0 f   q_math.obj
 0001:000319b0       _COM_ParseExt              200329b0 f   q_shared.obj
 0001:00031b20       _Q_strrchr                 20032b20 f   q_shared.obj
 0001:00031b50       _Q_strncpyz                20032b50 f   q_shared.obj
 0001:00031bb0       _Q_stricmpn                20032bb0 f   q_shared.obj
 0001:00031c30       _Q_strncmp                 20032c30 f   q_shared.obj
 0001:00031c70       _Q_stricmp                 20032c70 f   q_shared.obj
 0001:00031ca0       _Q_strcat                  20032ca0 f   q_shared.obj
 0001:00031cf0       _Q_CleanStr                20032cf0 f   q_shared.obj
 0001:00031d40       _Com_sprintf               20032d40 f   q_shared.obj
 0001:00031dc0       _va                        20032dc0 f   q_shared.obj
 0001:00031e00       _Info_ValueForKey          20032e00 f   q_shared.obj
 0001:00031f00       _Info_RemoveKey            20032f00 f   q_shared.obj
 0001:00032000       _Info_Validate             20033000 f   q_shared.obj
 0001:00032030       _Info_SetValueForKey       20033030 f   q_shared.obj
 0001:00032200       _COM_Parse                 20033200 f   q_shared.obj
 0001:00032210       _atol                      20033210 f   LIBC:atox.obj
 0001:00032268       _atoi                      20033268 f   LIBC:atox.obj
 0001:0003226d       _srand                     2003326d f   LIBC:rand.obj
 0001:00032277       _rand                      20033277 f   LIBC:rand.obj
 0001:0003229a       __fpclear                  2003329a f   LIBC:fpinit.obj
 0001:0003229b       __cfltcvt_init             2003329b f   LIBC:fpinit.obj
 0001:000322d3       __fpmath                   200332d3 f   LIBC:fpinit.obj
 0001:000322f4       __ftol2                    200332f4 f   LIBC:ftol2.obj
 0001:00032370       _strncpy                   20033370 f   LIBC:strncpy.obj
 0001:00032494       _atof                      20033494 f   LIBC:atof.obj
 0001:000324df       _sscanf                    200334df f   LIBC:sscanf.obj
 0001:00032513       _toupper                   20033513 f   LIBC:toupper.obj
 0001:000325f0       _memmove                   200335f0 f   LIBC:memmove.obj
 0001:00032930       _strstr                    20033930 f   LIBC:strstr.obj
 0001:000329b6       _vsprintf                  200339b6 f   LIBC:vsprintf.obj
 0001:00032a20       _strchr                    20033a20 f   LIBC:strchr.obj
 0001:00032a26       ___from_strstr_to_strchr   20033a26     LIBC:strchr.obj
 0001:00032ae0       __alloca_probe             20033ae0     LIBC:chkstk.obj
 0001:00032ae0       __chkstk                   20033ae0 f   LIBC:chkstk.obj
 0001:00032b1d       _tolower                   20033b1d f   LIBC:tolower.obj
 0001:00032c00       _ceil                      20033c00 f   LIBC:ceil_pentium4.obj
 0001:00032c40       __ceil_pentium4            20033c40 f   LIBC:ceil_pentium4.obj
 0001:00032d90       _qsort                     20033d90 f   LIBC:qsort.obj
 0001:00033013       __CRT_INIT@12              20034013 f   LIBC:dllcrt0.obj
 0001:0003311e       __DllMainCRTStartup@12     2003411e f   LIBC:dllcrt0.obj
 0001:00033202       __amsg_exit                20034202 f   LIBC:dllcrt0.obj
 0001:00033235       __ismbcspace               20034235 f   LIBC:ismbspc.obj
 0001:000332d0       __allmul                   200342d0 f   LIBC:llmul.obj
 0001:00033304       __forcdecpt                20034304 f   LIBC:cvt.obj
 0001:0003335c       __cropzeros                2003435c f   LIBC:cvt.obj
 0001:000333a7       __positive                 200343a7 f   LIBC:cvt.obj
 0001:000333c1       __fassign                  200343c1 f   LIBC:cvt.obj
 0001:0003341c       __cftoe                    2003441c f   LIBC:cvt.obj
 0001:0003350d       __cftof                    2003450d f   LIBC:cvt.obj
 0001:000335ea       __cftog                    200345ea f   LIBC:cvt.obj
 0001:00033694       __cfltcvt                  20034694 f   LIBC:cvt.obj
 0001:000336e5       __setdefaultprecision      200346e5 f   LIBC:fp8.obj
 0001:000336f7       __ms_p5_test_fdiv          200346f7 f   LIBC:testfdiv.obj
 0001:00033737       __ms_p5_mp_test_fdiv       20034737 f   LIBC:testfdiv.obj
 0001:00033760       __fltin                    20034760 f   LIBC:cfin.obj
 0001:00033800       _strlen                    20034800 f   LIBC:strlen.obj
 0001:0003388b       __isctype                  2003488b f   LIBC:isctype.obj
 0001:00033951       __input                    20034951 f   LIBC:input.obj
 0001:000347b8       ___crtLCMapStringA         200357b8 f   LIBC:a_map.obj
 0001:00034b74       __flsbuf                   20035b74 f   LIBC:_flsbuf.obj
 0001:00034d18       __output                   20035d18 f   LIBC:output.obj
 0001:00035512       ___libm_error_support      20036512 f   LIBC:libm_error.obj
 0001:000357d3       ___sse2_available_init     200367d3 f   LIBC:cpu_disp.obj
 0001:000358a1       __ceil_default             200368a1 f   LIBC:ceil.obj
 0001:00035974       ___crtExitProcess          20036974 f   LIBC:crt0dat.obj
 0001:000359a4       __cinit                    200369a4 f   LIBC:crt0dat.obj
 0001:00035acf       __exit                     20036acf f   LIBC:crt0dat.obj
 0001:00035ae0       __cexit                    20036ae0 f   LIBC:crt0dat.obj
 0001:00035aef       __ioinit                   20036aef f   LIBC:ioinit.obj
 0001:00035c9a       __ioterm                   20036c9a f   LIBC:ioinit.obj
 0001:00035cbd       __setenvp                  20036cbd f   LIBC:stdenvp.obj
 0001:00035ef0       __setargv                  20036ef0 f   LIBC:stdargv.obj
 0001:00035f92       ___heap_select             20036f92 f   LIBC:heapinit.obj
 0001:00035fac       __heap_init                20036fac f   LIBC:heapinit.obj
 0001:00035ffd       __heap_term                20036ffd f   LIBC:heapinit.obj
 0001:0003607c       ___crtGetEnvironmentStringsA 2003707c f   LIBC:a_env.obj
 0001:0003619e       __RTC_Initialize           2003719e f   LIBC:initsect.obj
 0001:000361e2       __RTC_Terminate            200371e2 f   LIBC:initsect.obj
 0001:00036226       __XcptFilter               20037226 f   LIBC:winxfltr.obj
 0001:00036397       ___CppXcptFilter           20037397 f   LIBC:winxfltr.obj
 0001:000363b2       _DllMain@12                200373b2 f   LIBC:dllmain.obj
 0001:000363d4       __SEH_prolog               200373d4 f   LIBC:sehprolg.obj
 0001:0003640f       __SEH_epilog               2003740f f   LIBC:sehprolg.obj
 0001:00036428       __except_handler3          20037428 f   LIBC:exsup3.obj
 0001:0003650e       __seh_longjmp_unwind@4     2003750e f   LIBC:exsup3.obj
 0001:00036529       __NMSG_WRITE               20037529 f   LIBC:crt0msg.obj
 0001:000366a0       __FF_MSGBANNER             200376a0 f   LIBC:crt0msg.obj
 0001:000366d9       ___crtGetStringTypeA       200376d9 f   LIBC:a_str.obj
 0001:00036a77       __setmbcp                  20037a77 f   LIBC:mbctype.obj
 0001:00036c5d       ___initmbctable            20037c5d f   LIBC:mbctype.obj
 0001:00036c7b       __ZeroTail                 20037c7b f   LIBC:intrncvt.obj
 0001:00036cad       __IncMan                   20037cad f   LIBC:intrncvt.obj
 0001:00036cfa       __RoundMan                 20037cfa f   LIBC:intrncvt.obj
 0001:00036d6c       __CopyMan                  20037d6c f   LIBC:intrncvt.obj
 0001:00036d87       __IsZeroMan                20037d87 f   LIBC:intrncvt.obj
 0001:00036da0       __ShrMan                   20037da0 f   LIBC:intrncvt.obj
 0001:00036e1b       __ld12cvt                  20037e1b f   LIBC:intrncvt.obj
 0001:00036f73       __ld12tod                  20037f73 f   LIBC:intrncvt.obj
 0001:00036f89       __ld12tof                  20037f89 f   LIBC:intrncvt.obj
 0001:00036f9f       __atodbl                   20037f9f f   LIBC:intrncvt.obj
 0001:00036fdc       __atoflt                   20037fdc f   LIBC:intrncvt.obj
 0001:00037020       _strcpy                    20038020 f   LIBC:strcat.obj
 0001:00037030       _strcat                    20038030 f   LIBC:strcat.obj
 0001:00037118       __fptostr                  20038118 f   LIBC:_fptostr.obj
 0001:0003718f       ___dtold                   2003818f f   LIBC:cfout.obj
 0001:00037249       __fltout                   20038249 f   LIBC:cfout.obj
 0001:000372c0       _memset                    200382c0 f   LIBC:memset.obj
 0001:00037320       __fptrap                   20038320 f   LIBC:crt0fp.obj
 0001:00037449       __control87                20038449 f   LIBC:ieee87.obj
 0001:0003747b       __controlfp                2003847b f   LIBC:ieee87.obj
 0001:00037491       ___strgtold12              20038491 f   LIBC:strgtold.obj
 0001:00037949       @__security_check_cookie@4 20038949 f   LIBC:secchk.obj
 0001:00037957       __filbuf                   20038957 f   LIBC:_filbuf.obj
 0001:00037a35       _ungetc                    20038a35 f   LIBC:ungetc.obj
 0001:00037aa1       _isspace                   20038aa1 f   LIBC:_ctype.obj
 0001:00037aca       _free                      20038aca f   LIBC:free.obj
 0001:00037b02       _mbtowc                    20038b02 f   LIBC:mbtowc.obj
 0001:00037bca       __heap_alloc               20038bca f   LIBC:malloc.obj
 0001:00037c10       __nh_malloc                20038c10 f   LIBC:malloc.obj
 0001:00037c3c       _malloc                    20038c3c f   LIBC:malloc.obj
 0001:00037c4e       __resetstkoflw             20038c4e f   LIBC:resetstk.obj
 0001:00037d31       ___ansicp                  20038d31 f   LIBC:convrtcp.obj
 0001:00037d74       ___convertcp               20038d74 f   LIBC:convrtcp.obj
 0001:00037f3d       __lseek                    20038f3d f   LIBC:lseek.obj
 0001:00037fc9       __write                    20038fc9 f   LIBC:write.obj
 0001:000381b9       __getbuf                   200391b9 f   LIBC:_getbuf.obj
 0001:000381fd       __isatty                   200391fd f   LIBC:isatty.obj
 0001:00038224       ___initstdio               20039224 f   LIBC:_file.obj
 0001:000382ca       ___endstdio                200392ca f   LIBC:_file.obj
 0001:000382de       _wctomb                    200392de f   LIBC:wctomb.obj
 0001:00038350       __aulldvrm                 20039350 f   LIBC:ulldvrm.obj
 0001:000383e5       __matherr                  200393e5 f   LIBC:matherr.obj
 0001:000383f0       _strncmp                   200393f0 f   LIBC:strncmp.obj
 0001:00038429       __raise_exc                20039429 f   LIBC:fpexcept.obj
 0001:000386ce       __handle_exc               200396ce f   LIBC:fpexcept.obj
 0001:000388f2       __set_errno                200398f2 f   LIBC:fpexcept.obj
 0001:00038918       __errcode                  20039918 f   LIBC:fpexcept.obj
 0001:00038945       __umatherr                 20039945 f   LIBC:fpexcept.obj
 0001:000389e5       __handle_qnan1             200399e5 f   LIBC:fpexcept.obj
 0001:00038a37       __except1                  20039a37 f   LIBC:fpexcept.obj
 0001:00038aef       __frnd                     20039aef f   LIBC:frnd.obj
 0001:00038b00       __set_exp                  20039b00 f   LIBC:util.obj
 0001:00038b2a       __sptype                   20039b2a f   LIBC:util.obj
 0001:00038b85       __decomp                   20039b85 f   LIBC:util.obj
 0001:00038c41       __statfp                   20039c41 f   LIBC:fpctrl.obj
 0001:00038c4c       __clrfp                    20039c4c f   LIBC:fpctrl.obj
 0001:00038c58       __ctrlfp                   20039c58 f   LIBC:fpctrl.obj
 0001:00038c7c       __set_statfp               20039c7c f   LIBC:fpctrl.obj
 0001:00038cd2       __onexit                   20039cd2 f   LIBC:onexit.obj
 0001:00038d54       _atexit                    20039d54 f   LIBC:onexit.obj
 0001:00038d66       ___onexitinit              20039d66 f   LIBC:onexit.obj
 0001:00038d8e       ___sbh_heap_init           20039d8e f   LIBC:sbheap.obj
 0001:00038dd6       ___sbh_find_block          20039dd6 f   LIBC:sbheap.obj
 0001:00038e01       ___sbh_free_block          20039e01 f   LIBC:sbheap.obj
 0001:00039119       ___sbh_alloc_new_region    2003a119 f   LIBC:sbheap.obj
 0001:000391d0       ___sbh_alloc_new_group     2003a1d0 f   LIBC:sbheap.obj
 0001:000392d6       ___sbh_resize_block        2003a2d6 f   LIBC:sbheap.obj
 0001:000395b5       ___sbh_alloc_block         2003a5b5 f   LIBC:sbheap.obj
 0001:000398c0       _memcpy                    2003a8c0 f   LIBC:memcpy.obj
 0001:00039c00       __global_unwind2           2003ac00 f   LIBC:exsup.obj
 0001:00039c42       __local_unwind2            2003ac42 f   LIBC:exsup.obj
 0001:00039c9a       __NLG_Return2              2003ac9a     LIBC:exsup.obj
 0001:00039caa       __abnormal_termination     2003acaa f   LIBC:exsup.obj
 0001:00039ccd       __NLG_Notify1              2003accd f   LIBC:exsup.obj
 0001:00039cd6       __NLG_Notify               2003acd6 f   LIBC:exsup.obj
 0001:00039ce9       __NLG_Dispatch             2003ace9     LIBC:exsup.obj
 0001:00039cee       __ValidateEH3RN            2003acee f   LIBC:eh3valid.obj
 0001:00039f17       ___crtMessageBoxA          2003af17 f   LIBC:crtmbox.obj
 0001:0003a010       _calloc                    2003b010 f   LIBC:calloc.obj
 0001:0003a08b       ___addl                    2003b08b f   LIBC:mantold.obj
 0001:0003a0ac       ___add_12                  2003b0ac f   LIBC:mantold.obj
 0001:0003a10a       ___shl_12                  2003b10a f   LIBC:mantold.obj
 0001:0003a138       ___shr_12                  2003b138 f   LIBC:mantold.obj
 0001:0003a165       ___mtold12                 2003b165 f   LIBC:mantold.obj
 0001:0003a243       _$I10_OUTPUT               2003b243 f   LIBC:x10fout.obj
 0001:0003a4d1       ___ld12mul                 2003b4d1 f   LIBC:tenpow.obj
 0001:0003a703       ___multtenpow12            2003b703 f   LIBC:tenpow.obj
 0001:0003a789       ___security_init_cookie    2003b789 f   LIBC:seccinit.obj
 0001:0003a7ef       ___security_error_handler  2003b7ef f   LIBC:secfail.obj
 0001:0003a937       __read                     2003b937 f   LIBC:read.obj
 0001:0003ab25       __callnewh                 2003bb25 f   LIBC:handler.obj
 0001:0003ab40       __dosmaperr                2003bb40 f   LIBC:dosmap.obj
 0001:0003ab9f       __free_osfhnd              2003bb9f f   LIBC:osfinfo.obj
 0001:0003ac19       __get_osfhandle            2003bc19 f   LIBC:osfinfo.obj
 0001:0003ac55       __lseeki64                 2003bc55 f   LIBC:lseeki64.obj
 0001:0003acf4       __fcloseall                2003bcf4 f   LIBC:closeall.obj
 0001:0003ad4c       __flush                    2003bd4c f   LIBC:fflush.obj
 0001:0003ada9       _fflush                    2003bda9 f   LIBC:fflush.obj
 0001:0003ae51       __flushall                 2003be51 f   LIBC:fflush.obj
 0001:0003ae5a       _realloc                   2003be5a f   LIBC:realloc.obj
 0001:0003afbc       __msize                    2003bfbc f   LIBC:msize.obj
 0001:0003aff4       _fclose                    2003bff4 f   LIBC:fclose.obj
 0001:0003b04a       __commit                   2003c04a f   LIBC:commit.obj
 0001:0003b0a1       __close                    2003c0a1 f   LIBC:close.obj
 0001:0003b154       __freebuf                  2003c154 f   LIBC:_freebuf.obj
 0001:0003b180       _RtlUnwind@16              2003c180 f   kernel32:KERNEL32.dll
 0002:00000000       __imp__GetCommandLineA@0   2003d000     kernel32:KERNEL32.dll
 0002:00000004       __imp__GetVersionExA@4     2003d004     kernel32:KERNEL32.dll
 0002:00000008       __imp__GetProcAddress@8    2003d008     kernel32:KERNEL32.dll
 0002:0000000c       __imp__GetModuleHandleA@4  2003d00c     kernel32:KERNEL32.dll
 0002:00000010       __imp__LCMapStringA@24     2003d010     kernel32:KERNEL32.dll
 0002:00000014       __imp__WideCharToMultiByte@32 2003d014     kernel32:KERNEL32.dll
 0002:00000018       __imp__MultiByteToWideChar@24 2003d018     kernel32:KERNEL32.dll
 0002:0000001c       __imp__GetLastError@0      2003d01c     kernel32:KERNEL32.dll
 0002:00000020       __imp__LCMapStringW@24     2003d020     kernel32:KERNEL32.dll
 0002:00000024       __imp__ExitProcess@4       2003d024     kernel32:KERNEL32.dll
 0002:00000028       __imp__TerminateProcess@8  2003d028     kernel32:KERNEL32.dll
 0002:0000002c       __imp__GetCurrentProcess@0 2003d02c     kernel32:KERNEL32.dll
 0002:00000030       __imp__SetHandleCount@4    2003d030     kernel32:KERNEL32.dll
 0002:00000034       __imp__GetStdHandle@4      2003d034     kernel32:KERNEL32.dll
 0002:00000038       __imp__GetFileType@4       2003d038     kernel32:KERNEL32.dll
 0002:0000003c       __imp__GetStartupInfoA@4   2003d03c     kernel32:KERNEL32.dll
 0002:00000040       __imp__GetModuleFileNameA@12 2003d040     kernel32:KERNEL32.dll
 0002:00000044       __imp__HeapDestroy@4       2003d044     kernel32:KERNEL32.dll
 0002:00000048       __imp__HeapCreate@12       2003d048     kernel32:KERNEL32.dll
 0002:0000004c       __imp__VirtualFree@12      2003d04c     kernel32:KERNEL32.dll
 0002:00000050       __imp__HeapFree@12         2003d050     kernel32:KERNEL32.dll
 0002:00000054       __imp__FreeEnvironmentStringsA@4 2003d054     kernel32:KERNEL32.dll
 0002:00000058       __imp__GetEnvironmentStrings@0 2003d058     kernel32:KERNEL32.dll
 0002:0000005c       __imp__FreeEnvironmentStringsW@4 2003d05c     kernel32:KERNEL32.dll
 0002:00000060       __imp__GetEnvironmentStringsW@0 2003d060     kernel32:KERNEL32.dll
 0002:00000064       __imp__UnhandledExceptionFilter@4 2003d064     kernel32:KERNEL32.dll
 0002:00000068       __imp__DisableThreadLibraryCalls@4 2003d068     kernel32:KERNEL32.dll
 0002:0000006c       __imp__WriteFile@20        2003d06c     kernel32:KERNEL32.dll
 0002:00000070       __imp__GetStringTypeA@20   2003d070     kernel32:KERNEL32.dll
 0002:00000074       __imp__GetStringTypeW@16   2003d074     kernel32:KERNEL32.dll
 0002:00000078       __imp__GetACP@0            2003d078     kernel32:KERNEL32.dll
 0002:0000007c       __imp__GetOEMCP@0          2003d07c     kernel32:KERNEL32.dll
 0002:00000080       __imp__GetCPInfo@8         2003d080     kernel32:KERNEL32.dll
 0002:00000084       __imp__HeapAlloc@12        2003d084     kernel32:KERNEL32.dll
 0002:00000088       __imp__VirtualProtect@16   2003d088     kernel32:KERNEL32.dll
 0002:0000008c       __imp__VirtualAlloc@16     2003d08c     kernel32:KERNEL32.dll
 0002:00000090       __imp__GetSystemInfo@4     2003d090     kernel32:KERNEL32.dll
 0002:00000094       __imp__VirtualQuery@12     2003d094     kernel32:KERNEL32.dll
 0002:00000098       __imp__GetLocaleInfoA@16   2003d098     kernel32:KERNEL32.dll
 0002:0000009c       __imp__SetFilePointer@16   2003d09c     kernel32:KERNEL32.dll
 0002:000000a0       __imp__RaiseException@16   2003d0a0     kernel32:KERNEL32.dll
 0002:000000a4       __imp__HeapReAlloc@16      2003d0a4     kernel32:KERNEL32.dll
 0002:000000a8       __imp__RtlUnwind@16        2003d0a8     kernel32:KERNEL32.dll
 0002:000000ac       __imp__InterlockedExchange@8 2003d0ac     kernel32:KERNEL32.dll
 0002:000000b0       __imp__LoadLibraryA@4      2003d0b0     kernel32:KERNEL32.dll
 0002:000000b4       __imp__QueryPerformanceCounter@4 2003d0b4     kernel32:KERNEL32.dll
 0002:000000b8       __imp__GetTickCount@0      2003d0b8     kernel32:KERNEL32.dll
 0002:000000bc       __imp__GetCurrentThreadId@0 2003d0bc     kernel32:KERNEL32.dll
 0002:000000c0       __imp__GetCurrentProcessId@0 2003d0c0     kernel32:KERNEL32.dll
 0002:000000c4       __imp__GetSystemTimeAsFileTime@4 2003d0c4     kernel32:KERNEL32.dll
 0002:000000c8       __imp__ReadFile@20         2003d0c8     kernel32:KERNEL32.dll
 0002:000000cc       __imp__SetStdHandle@8      2003d0cc     kernel32:KERNEL32.dll
 0002:000000d0       __imp__HeapSize@12         2003d0d0     kernel32:KERNEL32.dll
 0002:000000d4       __imp__FlushFileBuffers@4  2003d0d4     kernel32:KERNEL32.dll
 0002:000000d8       __imp__CloseHandle@4       2003d0d8     kernel32:KERNEL32.dll
 0002:000000dc       \177KERNEL32_NULL_THUNK_DATA 2003d0dc     kernel32:KERNEL32.dll
 0002:000000e0       ??_C@_01PFHFFBPC@t?$AA@    2003d0e0     ai_chat.obj
 0002:000000e4       ??_C@_01EFFIKLCJ@n?$AA@    2003d0e4     ai_chat.obj
 0002:000000e8       ??_C@_0O@OCOCOONB@sv_maxclients?$AA@ 2003d0e8     ai_chat.obj
 0002:000000f8       __real@38000100            2003d0f8     ai_chat.obj
 0002:000000fc       ??_C@_07KMNEBLH@mapname?$AA@ 2003d0fc     ai_chat.obj
 0002:00000104       ??_C@_0BB@FPHHFAJG@?$FLunknown?5weapon?$FN?$AA@ 2003d104     ai_chat.obj
 0002:00000118       ??_C@_07MKHABLGK@Grapple?$AA@ 2003d118     ai_chat.obj
 0002:00000120       ??_C@_06PNKEMFGD@BFG10K?$AA@ 2003d120     ai_chat.obj
 0002:00000128       ??_C@_0O@HOCKKNKE@Lightning?5Gun?$AA@ 2003d128     ai_chat.obj
 0002:00000138       ??_C@_07NMJDHEIK@Railgun?$AA@ 2003d138     ai_chat.obj
 0002:00000140       ??_C@_09MBHKGILD@Plasmagun?$AA@ 2003d140     ai_chat.obj
 0002:0000014c       ??_C@_0BA@DJIGCIDL@Rocket?5Launcher?$AA@ 2003d14c     ai_chat.obj
 0002:0000015c       ??_C@_0BB@GIEOMMBO@Grenade?5Launcher?$AA@ 2003d15c     ai_chat.obj
 0002:00000170       ??_C@_0L@KDNGMPND@Machinegun?$AA@ 2003d170     ai_chat.obj
 0002:0000017c       ??_C@_08ELAHAPJB@Gauntlet?$AA@ 2003d17c     ai_chat.obj
 0002:00000188       ??_C@_07DGIAOJJ@Shotgun?$AA@ 2003d188     ai_chat.obj
 0002:00000190       __real@4021cccccccccccd    2003d190     ai_chat.obj
 0002:00000198       __real@00000000            2003d198     ai_chat.obj
 0002:0000019c       __real@41200000            2003d19c     ai_chat.obj
 0002:000001a0       __real@3f800000            2003d1a0     ai_chat.obj
 0002:000001a4       __real@42000000            2003d1a4     ai_chat.obj
 0002:000001a8       __real@41c00000            2003d1a8     ai_chat.obj
 0002:000001ac       ??_C@_0L@PKHLIBCF@game_enter?$AA@ 2003d1ac     ai_chat.obj
 0002:000001b8       ??_C@_0O@IGAOFANI@?$FLinvalid?5var?$FN?$AA@ 2003d1b8     ai_chat.obj
 0002:000001c8       __real@41c80000            2003d1c8     ai_chat.obj
 0002:000001cc       ??_C@_09PIOCENHO@game_exit?$AA@ 2003d1cc     ai_chat.obj
 0002:000001d8       ??_C@_0M@CJNDJGDH@level_start?$AA@ 2003d1d8     ai_chat.obj
 0002:000001e4       ??_C@_06IMDBNOMM@vtaunt?$AA@ 2003d1e4     ai_chat.obj
 0002:000001ec       ??_C@_09PILOJEEK@level_end?$AA@ 2003d1ec     ai_chat.obj
 0002:000001f8       ??_C@_0P@LPKGAAGE@level_end_lose?$AA@ 2003d1f8     ai_chat.obj
 0002:00000208       ??_C@_0BC@GKFLFIDK@level_end_victory?$AA@ 2003d208     ai_chat.obj
 0002:0000021c       ??_C@_0O@EGKCFKBF@death_suicide?$AA@ 2003d21c     ai_chat.obj
 0002:0000022c       ??_C@_0N@INLGGPBP@death_praise?$AA@ 2003d22c     ai_chat.obj
 0002:0000023c       ??_C@_0N@EPKIJPHK@death_insult?$AA@ 2003d23c     ai_chat.obj
 0002:0000024c       ??_C@_09HPMGADCC@death_bfg?$AA@ 2003d24c     ai_chat.obj
 0002:00000258       ??_C@_0L@OLPOCBHN@death_rail?$AA@ 2003d258     ai_chat.obj
 0002:00000264       ??_C@_0P@GODBEIFH@death_gauntlet?$AA@ 2003d264     ai_chat.obj
 0002:00000278       __real@3fe0000000000000    2003d278     ai_chat.obj
 0002:00000280       ??_C@_0P@CLLHBMMH@death_telefrag?$AA@ 2003d280     ai_chat.obj
 0002:00000290       ??_C@_0P@FHLBDKHM@death_cratered?$AA@ 2003d290     ai_chat.obj
 0002:000002a0       ??_C@_0L@JGPKJCJO@death_lava?$AA@ 2003d2a0     ai_chat.obj
 0002:000002ac       ??_C@_0M@ENLBBGB@death_slime?$AA@ 2003d2ac     ai_chat.obj
 0002:000002b8       ??_C@_0M@BCPGKKBA@death_drown?$AA@ 2003d2b8     ai_chat.obj
 0002:000002c4       ??_C@_0P@LLJEDFBD@death_teammate?$AA@ 2003d2c4     ai_chat.obj
 0002:000002d4       ??_C@_07PANFCHNN@?$FLworld?$FN?$AA@ 2003d2d4     ai_chat.obj
 0002:000002dc       ??_C@_0M@NDKPNHB@kill_praise?$AA@ 2003d2dc     ai_chat.obj
 0002:000002e8       ??_C@_0M@MPCEANBE@kill_insult?$AA@ 2003d2e8     ai_chat.obj
 0002:000002f4       ??_C@_0O@MOMICIAK@kill_telefrag?$AA@ 2003d2f4     ai_chat.obj
 0002:00000304       ??_C@_09HNPOIBHL@kill_rail?$AA@ 2003d304     ai_chat.obj
 0002:00000310       ??_C@_0O@ILEOHMJK@kill_gauntlet?$AA@ 2003d310     ai_chat.obj
 0002:00000320       ??_C@_0O@FOOLABNO@kill_teammate?$AA@ 2003d320     ai_chat.obj
 0002:00000330       ??_C@_0O@CCLFCPCH@enemy_suicide?$AA@ 2003d330     ai_chat.obj
 0002:00000340       ??_C@_0M@GJHANCBL@hit_talking?$AA@ 2003d340     ai_chat.obj
 0002:0000034c       ??_C@_0M@NEMKKKCP@hit_nodeath?$AA@ 2003d34c     ai_chat.obj
 0002:00000358       ??_C@_0L@HALGAHGK@hit_nokill?$AA@ 2003d358     ai_chat.obj
 0002:00000364       ??_C@_0O@BCFFFDNI@random_insult?$AA@ 2003d364     ai_chat.obj
 0002:00000374       ??_C@_0M@DCDJELGA@random_misc?$AA@ 2003d374     ai_chat.obj
 0002:00000380       __real@3fd0000000000000    2003d380     ai_chat.obj
 0002:00000388       __real@3fb999999999999a    2003d388     ai_chat.obj
 0002:00000390       __real@40000000            2003d390     ai_chat.obj
 0002:00000398       __real@404e000000000000    2003d398     ai_cmd.obj
 0002:000003a0       __real@44e10000            2003d3a0     ai_cmd.obj
 0002:000003a4       __real@44160000            2003d3a4     ai_cmd.obj
 0002:000003a8       __real@4cbebc20            2003d3a8     ai_cmd.obj
 0002:000003ac       ??_C@_0CC@BCALNIDF@I?5need?5more?5key?5points?5to?5patrol@ 2003d3ac     ai_cmd.obj
 0002:000003d0       ??_C@_0BB@PGBIDPPC@what?5do?5you?5say?$DP?$AA@ 2003d3d0     ai_cmd.obj
 0002:000003e4       __real@42700000            2003d3e4     ai_cmd.obj
 0002:000003e8       ??_C@_0M@HCHCFBDA@whereareyou?$AA@ 2003d3e8     ai_cmd.obj
 0002:000003f4       ??_C@_07BANGEKHA@whereis?$AA@ 2003d3f4     ai_cmd.obj
 0002:000003fc       ??_C@_05NBAJGCGG@whois?$AA@ 2003d3fc     ai_cmd.obj
 0002:00000404       __real@42f00000            2003d404     ai_cmd.obj
 0002:00000408       ??_C@_03ICICOMAL@yes?$AA@  2003d408     ai_cmd.obj
 0002:0000040c       ??_C@_0L@CCGDOBMA@keepinmind?$AA@ 2003d40c     ai_cmd.obj
 0002:00000418       __real@43340000            2003d418     ai_cmd.obj
 0002:0000041c       ??_C@_0L@OAEJIBOJ@joinedteam?$AA@ 2003d41c     ai_cmd.obj
 0002:00000428       ??_C@_08NKJDPEPF@leftteam?$AA@ 2003d428     ai_cmd.obj
 0002:00000434       ??_C@_06NJFEFPHF@noteam?$AA@ 2003d434     ai_cmd.obj
 0002:0000043c       ??_C@_06NHKPLCFO@inteam?$AA@ 2003d43c     ai_cmd.obj
 0002:00000444       ??_C@_0BD@PGFNLHLB@checkpoint_confirm?$AA@ 2003d444     ai_cmd.obj
 0002:00000458       ??_C@_0BC@PAJMIFOG@?$CF1?40f?5?$CF1?40f?5?$CF1?40f?$AA@ 2003d458     ai_cmd.obj
 0002:0000046c       ??_C@_0BD@GKCAPLMB@checkpoint_invalid?$AA@ 2003d46c     ai_cmd.obj
 0002:00000480       ??_C@_08OEKJENGB@?$CFf?5?$CFf?5?$CFf?$AA@ 2003d480     ai_cmd.obj
 0002:0000048c       __real@42c80000            2003d48c     ai_cmd.obj
 0002:00000490       __real@43fa0000            2003d490     ai_cmd.obj
 0002:00000494       __real@42400000            2003d494     ai_cmd.obj
 0002:00000498       __real@4040000000000000    2003d498     ai_cmd.obj
 0002:000004a0       __real@402381d7dbf487fd    2003d4a0     ai_cmd.obj
 0002:000004a8       ??_C@_09FLIJNDLN@dismissed?$AA@ 2003d4a8     ai_cmd.obj
 0002:000004b4       ??_C@_05CPCHEFAA@taunt?$AA@ 2003d4b4     ai_cmd.obj
 0002:000004bc       ??_C@_04BJJEOANI@kill?$AA@ 2003d4bc     ai_cmd.obj
 0002:000004c4       ??_C@_0BF@EGOEAANC@I?8m?5the?5team?5leader?6?$AA@ 2003d4c4     ai_cmd.obj
 0002:000004dc       ??_C@_07IFIHEGLH@roaming?$AA@ 2003d4dc     ai_cmd.obj
 0002:000004e4       ??_C@_0O@PNEKPGNP@returningflag?$AA@ 2003d4e4     ai_cmd.obj
 0002:000004f4       ??_C@_0M@BGGCILAH@rushingbase?$AA@ 2003d4f4     ai_cmd.obj
 0002:00000500       ??_C@_0O@KMOOAPPA@capturingflag?$AA@ 2003d500     ai_cmd.obj
 0002:00000510       ??_C@_0L@GHJELNDI@patrolling?$AA@ 2003d510     ai_cmd.obj
 0002:0000051c       ??_C@_07IKBLJPBH@camping?$AA@ 2003d51c     ai_cmd.obj
 0002:00000524       ??_C@_07EFNGDOD@killing?$AA@ 2003d524     ai_cmd.obj
 0002:0000052c       ??_C@_0M@EEGCLMEK@gettingitem?$AA@ 2003d52c     ai_cmd.obj
 0002:00000538       ??_C@_09GNBACBHC@defending?$AA@ 2003d538     ai_cmd.obj
 0002:00000544       ??_C@_0N@FBKCFEPP@accompanying?$AA@ 2003d544     ai_cmd.obj
 0002:00000554       ??_C@_07OIGCHEPH@helping?$AA@ 2003d554     ai_cmd.obj
 0002:00000560       __real@3ff0000000000000    2003d560     ai_cmd.obj
 0002:00000568       ??_C@_08CBBFJFMD@location?$AA@ 2003d568     ai_cmd.obj
 0002:00000574       ??_C@_04OBGPFBCN@blue?$AA@ 2003d574     ai_cmd.obj
 0002:0000057c       ??_C@_0N@LHJHAMNN@teamlocation?$AA@ 2003d57c     ai_cmd.obj
 0002:0000058c       ??_C@_03FAAAOPJM@red?$AA@  2003d58c     ai_cmd.obj
 0002:00000590       __real@3fd999999999999a    2003d590     ai_cmd.obj
 0002:00000598       ??_C@_09MDBFHCAB@Blue?5Flag?$AA@ 2003d598     ai_cmd.obj
 0002:000005a4       ??_C@_08GAOGPIJL@Red?5Flag?$AA@ 2003d5a4     ai_cmd.obj
 0002:000005b0       ??_C@_0M@ICCAHGAD@Heavy?5Armor?$AA@ 2003d5b0     ai_cmd.obj
 0002:000005bc       ??_C@_05JOOFIMIN@Armor?$AA@ 2003d5bc     ai_cmd.obj
 0002:000005c4       ??_C@_06FDKFDAP@Flight?$AA@ 2003d5c4     ai_cmd.obj
 0002:000005cc       ??_C@_0N@LCCEENAK@Invisibility?$AA@ 2003d5cc     ai_cmd.obj
 0002:000005dc       ??_C@_05HOIAGEJD@Speed?$AA@ 2003d5dc     ai_cmd.obj
 0002:000005e4       ??_C@_0M@ONKEJEFE@Battle?5Suit?$AA@ 2003d5e4     ai_cmd.obj
 0002:000005f0       ??_C@_0N@CBPBLBHG@Regeneration?$AA@ 2003d5f0     ai_cmd.obj
 0002:00000600       ??_C@_0M@KOJLOALK@Quad?5Damage?$AA@ 2003d600     ai_cmd.obj
 0002:0000060c       ??_C@_0BE@NHGFGLLF@unknown?5match?5type?6?$AA@ 2003d60c     ai_cmd.obj
 0002:00000620       ??_C@_0DL@ENJHCNMJ@the?5part?5of?5my?5brain?5to?5create?5f@ 2003d620     ai_cmd.obj
 0002:0000065b       ??_C@_00CNPNBAHC@?$AA@     2003d65b     ai_dmnet.obj
 0002:0000065c       ??_C@_0CM@FBOPNIPA@?$CFs?5at?5?$CF1?41f?5switched?5more?5than?5?$CF@ 2003d65c     ai_dmnet.obj
 0002:00000688       ??_C@_0CE@EJLGIIOB@?$CFs?5at?5?$CF2?41f?5entered?5?$CFs?3?5?$CFs?5from?5@ 2003d688     ai_dmnet.obj
 0002:000006ac       __real@447a0000            2003d6ac     ai_dmnet.obj
 0002:000006b0       __real@40c00000            2003d6b0     ai_dmnet.obj
 0002:000006b4       __real@41a00000            2003d6b4     ai_dmnet.obj
 0002:000006b8       ??_C@_0N@INDGBJCC@onreturnflag?$AA@ 2003d6b8     ai_dmnet.obj
 0002:000006c8       ??_C@_0BB@BFOOKAAN@returnflag_start?$AA@ 2003d6c8     ai_dmnet.obj
 0002:000006dc       ??_C@_09DPAAIBFE@ongetflag?$AA@ 2003d6dc     ai_dmnet.obj
 0002:000006e8       ??_C@_0BC@BPHAAOLA@captureflag_start?$AA@ 2003d6e8     ai_dmnet.obj
 0002:000006fc       ??_C@_0M@JOFDEJLG@patrol_stop?$AA@ 2003d6fc     ai_dmnet.obj
 0002:00000708       ??_C@_0N@IKJEFKFP@patrol_start?$AA@ 2003d708     ai_dmnet.obj
 0002:00000718       ??_C@_04MKEOLIJC@?5to?5?$AA@ 2003d718     ai_dmnet.obj
 0002:00000720       ??_C@_0L@IJFFADDJ@inposition?$AA@ 2003d720     ai_dmnet.obj
 0002:0000072c       ??_C@_0M@PEOBAIFC@camp_arrive?$AA@ 2003d72c     ai_dmnet.obj
 0002:00000738       __real@45610000            2003d738     ai_dmnet.obj
 0002:0000073c       ??_C@_09BHIDKEB@camp_stop?$AA@ 2003d73c     ai_dmnet.obj
 0002:00000748       ??_C@_0L@KJNCBGJD@camp_start?$AA@ 2003d748     ai_dmnet.obj
 0002:00000754       ??_C@_0O@EJODLBHP@getitem_gotit?$AA@ 2003d754     ai_dmnet.obj
 0002:00000764       ??_C@_0BB@GOIMPKGP@getitem_notthere?$AA@ 2003d764     ai_dmnet.obj
 0002:00000778       ??_C@_0O@LBCALMFN@getitem_start?$AA@ 2003d778     ai_dmnet.obj
 0002:00000788       ??_C@_09KGAMDJKG@kill_done?$AA@ 2003d788     ai_dmnet.obj
 0002:00000794       ??_C@_0L@DMKJIHAF@kill_start?$AA@ 2003d794     ai_dmnet.obj
 0002:000007a0       __real@40400000            2003d7a0     ai_dmnet.obj
 0002:000007a4       __real@45992000            2003d7a4     ai_dmnet.obj
 0002:000007a8       ??_C@_0M@DFCLNMCD@defend_stop?$AA@ 2003d7a8     ai_dmnet.obj
 0002:000007b4       ??_C@_09DPKMICOA@ondefense?$AA@ 2003d7b4     ai_dmnet.obj
 0002:000007c0       ??_C@_0N@KFKEFAB@defend_start?$AA@ 2003d7c0     ai_dmnet.obj
 0002:000007d0       ??_C@_0BF@DCOBNKPB@accompany_cannotfind?$AA@ 2003d7d0     ai_dmnet.obj
 0002:000007e8       ??_C@_0BM@KDEEGPGK@BotLongTermGoal?3?5go?5for?5air?$AA@ 2003d7e8     ai_dmnet.obj
 0002:00000804       __real@41000000            2003d804     ai_dmnet.obj
 0002:00000808       __real@3fe999999999999a    2003d808     ai_dmnet.obj
 0002:00000810       __real@3fa999999999999a    2003d810     ai_dmnet.obj
 0002:00000818       ??_C@_0BB@FONGAGIJ@accompany_arrive?$AA@ 2003d818     ai_dmnet.obj
 0002:0000082c       __real@41700000            2003d82c     ai_dmnet.obj
 0002:00000830       __real@40a00000            2003d830     ai_dmnet.obj
 0002:00000838       __real@3fe6666666666666    2003d838     ai_dmnet.obj
 0002:00000840       __real@40800000            2003d840     ai_dmnet.obj
 0002:00000844       ??_C@_0P@JLGJIDCE@accompany_stop?$AA@ 2003d844     ai_dmnet.obj
 0002:00000854       ??_C@_0BA@JEJAJCPN@accompany_start?$AA@ 2003d854     ai_dmnet.obj
 0002:00000864       __real@461c4000            2003d864     ai_dmnet.obj
 0002:00000868       ??_C@_0L@JEGDCFOO@help_start?$AA@ 2003d868     ai_dmnet.obj
 0002:00000874       __real@48742400            2003d874     ai_dmnet.obj
 0002:00000878       ??_C@_08LJGLPHPA@followme?$AA@ 2003d878     ai_dmnet.obj
 0002:00000884       ??_C@_09GJKBJNFC@lead_stop?$AA@ 2003d884     ai_dmnet.obj
 0002:00000890       ??_C@_05PJLLPND@stand?$AA@ 2003d890     ai_dmnet.obj
 0002:00000898       ??_C@_0BI@BGMGILOO@observer?3?5left?5observer?$AA@ 2003d898     ai_dmnet.obj
 0002:000008b0       ??_C@_0BD@MNFAOLC@respawn?3?5respawned?$AA@ 2003d8b0     ai_dmnet.obj
 0002:000008c4       ??_C@_0N@JAICAHME@battle?5fight?$AA@ 2003d8c4     ai_dmnet.obj
 0002:000008d4       ??_C@_0L@EFLDDLAJ@battle?5NBG?$AA@ 2003d8d4     ai_dmnet.obj
 0002:000008e0       ??_C@_08BDAIAION@observer?$AA@ 2003d8e0     ai_dmnet.obj
 0002:000008ec       ??_C@_07PABIOCAD@respawn?$AA@ 2003d8ec     ai_dmnet.obj
 0002:000008f8       __real@3fd3333333333333    2003d8f8     ai_dmnet.obj
 0002:00000900       ??_C@_0BE@EEPGNAKO@battle?5retreat?3?5nbg?$AA@ 2003d900     ai_dmnet.obj
 0002:00000914       __real@3c23d70a            2003d914     ai_dmnet.obj
 0002:00000918       ??_C@_0BL@IFDBGGDM@battle?5retreat?3?5no?5way?5out?$AA@ 2003d918     ai_dmnet.obj
 0002:00000934       ??_C@_0BO@JHDCIIFI@battle?5retreat?3?5another?5enemy?$AA@ 2003d934     ai_dmnet.obj
 0002:00000954       ??_C@_0BL@KBIAJDEJ@battle?5retreat?3?5lost?5enemy?$AA@ 2003d954     ai_dmnet.obj
 0002:00000970       ??_C@_0N@JLOOIPJK@battle?5chase?$AA@ 2003d970     ai_dmnet.obj
 0002:00000980       ??_C@_0BP@PDKIMDBN@battle?5retreat?3?5wants?5to?5chase?$AA@ 2003d980     ai_dmnet.obj
 0002:000009a0       ??_C@_0BL@NMDPGNGL@battle?5retreat?3?5enemy?5dead?$AA@ 2003d9a0     ai_dmnet.obj
 0002:000009bc       ??_C@_0BJ@BKIHIJBD@battle?5retreat?3?5no?5enemy?$AA@ 2003d9bc     ai_dmnet.obj
 0002:000009d8       ??_C@_0BJ@MIHKKBKF@battle?5retreat?3?5bot?5dead?$AA@ 2003d9d8     ai_dmnet.obj
 0002:000009f4       ??_C@_0BN@IHDFIOBO@battle?5retreat?3?5intermission?$AA@ 2003d9f4     ai_dmnet.obj
 0002:00000a14       ??_C@_0BJ@IOJPHBCK@battle?5retreat?3?5observer?$AA@ 2003da14     ai_dmnet.obj
 0002:00000a30       ??_C@_0P@ELFCJAMH@battle?5retreat?$AA@ 2003da30     ai_dmnet.obj
 0002:00000a40       ??_C@_0BH@PKDGJGPO@battle?5chase?3?5time?5out?$AA@ 2003da40     ai_dmnet.obj
 0002:00000a58       ??_C@_0BP@DMHFNNNL@battle?5chase?3?5wants?5to?5retreat?$AA@ 2003da58     ai_dmnet.obj
 0002:00000a78       ??_C@_0BC@MBHDFOHG@battle?5chase?3?5nbg?$AA@ 2003da78     ai_dmnet.obj
 0002:00000a90       __real@4030000000000000    2003da90     ai_dmnet.obj
 0002:00000a98       ??_C@_0BM@JANANJEH@battle?5chase?3?5no?5enemy?5area?$AA@ 2003da98     ai_dmnet.obj
 0002:00000ab4       ??_C@_0BL@BJLICKPC@battle?5chase?3?5better?5enemy?$AA@ 2003dab4     ai_dmnet.obj
 0002:00000ad0       ??_C@_0BH@PIOMJOG@battle?5chase?3?5no?5enemy?$AA@ 2003dad0     ai_dmnet.obj
 0002:00000ae8       ??_C@_0BH@NNHDOBFA@battle?5chase?3?5bot?5dead?$AA@ 2003dae8     ai_dmnet.obj
 0002:00000b00       ??_C@_0BL@PKAILKOJ@battle?5chase?3?5intermission?$AA@ 2003db00     ai_dmnet.obj
 0002:00000b1c       ??_C@_0BH@JLJGDBNP@battle?5chase?3?5observer?$AA@ 2003db1c     ai_dmnet.obj
 0002:00000b34       ??_C@_0BP@KNHNJPON@battle?5fight?3?5wants?5to?5retreat?$AA@ 2003db34     ai_dmnet.obj
 0002:00000b54       ??_C@_0CB@IGGJLKOL@battle?5fight?3?5enemy?5out?5of?5sight@ 2003db54     ai_dmnet.obj
 0002:00000b78       ??_C@_0BP@NBCPEGCG@battle?5fight?3?5chat?5hit?5someone?$AA@ 2003db78     ai_dmnet.obj
 0002:00000b98       ??_C@_0CE@HNIMDJBG@battle?5fight?3?5chat?5health?5decrea@ 2003db98     ai_dmnet.obj
 0002:00000bbc       ??_C@_0BI@PALDJFNB@battle?5fight?3?5invisible?$AA@ 2003dbbc     ai_dmnet.obj
 0002:00000bd8       __real@3fc999999999999a    2003dbd8     ai_dmnet.obj
 0002:00000be0       ??_C@_0BJ@JCMOALOB@battle?5fight?3?5enemy?5dead?$AA@ 2003dbe0     ai_dmnet.obj
 0002:00000bfc       ??_C@_0BH@PAJNDMEE@battle?5fight?3?5no?5enemy?$AA@ 2003dbfc     ai_dmnet.obj
 0002:00000c14       ??_C@_0BH@CCGABEPC@battle?5fight?3?5bot?5dead?$AA@ 2003dc14     ai_dmnet.obj
 0002:00000c2c       ??_C@_0BL@OCIIHEED@battle?5fight?3?5intermission?$AA@ 2003dc2c     ai_dmnet.obj
 0002:00000c48       ??_C@_0BH@GEIFMEHN@battle?5fight?3?5observer?$AA@ 2003dc48     ai_dmnet.obj
 0002:00000c60       ??_C@_0BG@LLBOBEHC@seek?5nbg?3?5found?5enemy?$AA@ 2003dc60     ai_dmnet.obj
 0002:00000c78       ??_C@_0BD@KKPPPHA@seek?5nbg?3?5time?5out?$AA@ 2003dc78     ai_dmnet.obj
 0002:00000c8c       ??_C@_0BD@CNOKIINO@seek?5nbg?3?5bot?5dead?$AA@ 2003dc8c     ai_dmnet.obj
 0002:00000ca0       ??_C@_0BG@FJPIPBDN@seek?5nbg?3?5intermision?$AA@ 2003dca0     ai_dmnet.obj
 0002:00000cb8       ??_C@_0BD@GLAPFIFB@seek?5nbg?3?5observer?$AA@ 2003dcb8     ai_dmnet.obj
 0002:00000ccc       ??_C@_07ONOEGCJB@no?5goal?$AA@ 2003dccc     ai_dmnet.obj
 0002:00000cd4       ??_C@_08IFECKGCD@seek?5NBG?$AA@ 2003dcd4     ai_dmnet.obj
 0002:00000ce0       __real@3f847ae147ae147b    2003dce0     ai_dmnet.obj
 0002:00000ce8       ??_C@_0O@OMHBKBBP@ltg?5seek?3?5nbg?$AA@ 2003dce8     ai_dmnet.obj
 0002:00000cf8       ??_C@_0BG@NKJENDMP@seek?5ltg?3?5found?5enemy?$AA@ 2003dcf8     ai_dmnet.obj
 0002:00000d10       ??_C@_0BG@FMPBNGLO@seek?5ltg?3?5random?5chat?$AA@ 2003dd10     ai_dmnet.obj
 0002:00000d28       ??_C@_0BD@NIGGDFHE@seek?5ltg?3?5bot?5dead?$AA@ 2003dd28     ai_dmnet.obj
 0002:00000d3c       ??_C@_0BH@BIAHANPH@seek?5ltg?3?5intermission?$AA@ 2003dd3c     ai_dmnet.obj
 0002:00000d54       ??_C@_0BD@JOIDOFPL@seek?5ltg?3?5observer?$AA@ 2003dd54     ai_dmnet.obj
 0002:00000d68       ??_C@_08DHOALBGK@seek?5LTG?$AA@ 2003dd68     ai_dmnet.obj
 0002:00000d74       ??_C@_0BA@EJJPLHJN@stand?3?5time?5out?$AA@ 2003dd74     ai_dmnet.obj
 0002:00000d84       ??_C@_0BD@EFNKCGD@stand?3?5found?5enemy?$AA@ 2003dd84     ai_dmnet.obj
 0002:00000d98       ??_C@_0BD@FAEFJCHC@intermission?3?5chat?$AA@ 2003dd98     ai_dmnet.obj
 0002:00000dac       ??_C@_0N@IHDBPIFK@intermission?$AA@ 2003ddac     ai_dmnet.obj
 0002:00000dbc       ??_C@_0BN@CHDNEHF@activate?5entity?3?5found?5enemy?$AA@ 2003ddbc     ai_dmnet.obj
 0002:00000ddc       ??_C@_0BL@KOANFMEA@activate?5entity?3?5activated?$AA@ 2003dddc     ai_dmnet.obj
 0002:00000df8       ??_C@_0BK@GBGNKJEG@activate?5entity?3?5time?5out?$AA@ 2003ddf8     ai_dmnet.obj
 0002:00000e14       ??_C@_0BJ@EEHKLOIJ@activate?5entity?3?5no?5goal?$AA@ 2003de14     ai_dmnet.obj
 0002:00000e30       ??_C@_0BK@EGCINOOI@activate?5entity?3?5bot?5dead?$AA@ 2003de30     ai_dmnet.obj
 0002:00000e4c       ??_C@_0BO@DDGLLAGC@activate?5entity?3?5intermission?$AA@ 2003de4c     ai_dmnet.obj
 0002:00000e6c       ??_C@_0BI@CFBHMKPG@active?5entity?3?5observer?$AA@ 2003de6c     ai_dmnet.obj
 0002:00000e84       ??_C@_0BF@JGNGECFP@battle?5nbg?3?5time?5out?$AA@ 2003de84     ai_dmnet.obj
 0002:00000e9c       ??_C@_0BH@PFIKNLIP@battle?5nbg?3?5enemy?5dead?$AA@ 2003de9c     ai_dmnet.obj
 0002:00000eb4       ??_C@_0BF@GDGOBNEH@battle?5nbg?3?5no?5enemy?$AA@ 2003deb4     ai_dmnet.obj
 0002:00000ecc       ??_C@_0BF@LBJDDFPB@battle?5nbg?3?5bot?5dead?$AA@ 2003decc     ai_dmnet.obj
 0002:00000ee4       ??_C@_0BJ@JPCFIHPK@battle?5nbg?3?5intermission?$AA@ 2003dee4     ai_dmnet.obj
 0002:00000f00       ??_C@_0BF@PHHGOFHO@battle?5nbg?3?5observer?$AA@ 2003df00     ai_dmnet.obj
 0002:00000f18       ??_C@_0BA@OLIPHEKA@activate?5entity?$AA@ 2003df18     ai_dmnet.obj
 0002:00000f28       ??_C@_02KAJCLHKP@no?$AA@   2003df28     ai_dmq3.obj
 0002:00000f2c       ??_C@_0BG@EPIHOAD@?$FLclient?5out?5of?5range?$FN?$AA@ 2003df2c     ai_dmq3.obj
 0002:00000f44       ??_C@_0CB@FEANAAEF@ClientName?3?5client?5out?5of?5range?6@ 2003df44     ai_dmq3.obj
 0002:00000f68       ??_C@_05NCCFOPHA@model?$AA@ 2003df68     ai_dmq3.obj
 0002:00000f70       ??_C@_01LBDDMOBJ@?$FN?$AA@ 2003df70     ai_dmq3.obj
 0002:00000f74       ??_C@_01OHGJGJJP@?$FL?$AA@ 2003df74     ai_dmq3.obj
 0002:00000f78       ??_C@_01CLKCMJKC@?5?$AA@   2003df78     ai_dmq3.obj
 0002:00000f7c       __real@41b80000            2003df7c     ai_dmq3.obj
 0002:00000f80       ??_C@_0CF@BEIOCA@BotCreateWayPoint?3?5Out?5of?5waypoi@ 2003df80     ai_dmq3.obj
 0002:00000fa8       __real@42480000            2003dfa8     ai_dmq3.obj
 0002:00000fac       __real@42a00000            2003dfac     ai_dmq3.obj
 0002:00000fb0       __real@42aa0000            2003dfb0     ai_dmq3.obj
 0002:00000fb4       __real@42b40000            2003dfb4     ai_dmq3.obj
 0002:00000fb8       __real@42be0000            2003dfb8     ai_dmq3.obj
 0002:00000fbc       __real@428c0000            2003dfbc     ai_dmq3.obj
 0002:00000fc0       __real@47c34f80            2003dfc0     ai_dmq3.obj
 0002:00000fc8       __real@3fefae147ae147ae    2003dfc8     ai_dmq3.obj
 0002:00000fd0       __real@43960000            2003dfd0     ai_dmq3.obj
 0002:00000fd4       __real@42200000            2003dfd4     ai_dmq3.obj
 0002:00000fd8       __real@43480000            2003dfd8     ai_dmq3.obj
 0002:00000fe0       __real@4058000000000000    2003dfe0     ai_dmq3.obj
 0002:00000fe8       __real@3fe8000000000000    2003dfe8     ai_dmq3.obj
 0002:00000ff0       __real@44480000            2003dff0     ai_dmq3.obj
 0002:00000ff8       __real@3feccccccccccccd    2003dff8     ai_dmq3.obj
 0002:00001000       __real@3fedeb851eb851ec    2003e000     ai_dmq3.obj
 0002:00001008       __real@c066800000000000    2003e008     ai_dmq3.obj
 0002:00001010       __real@4076800000000000    2003e010     ai_dmq3.obj
 0002:00001018       __real@4066800000000000    2003e018     ai_dmq3.obj
 0002:00001020       __real@3fee666666666666    2003e020     ai_dmq3.obj
 0002:00001028       __real@3f50624dd2f1a9fc    2003e028     ai_dmq3.obj
 0002:00001030       __real@390fd66c            2003e030     ai_dmq3.obj
 0002:00001034       __real@49202e40            2003e034     ai_dmq3.obj
 0002:00001038       __real@408c200000000000    2003e038     ai_dmq3.obj
 0002:00001040       __real@40af400000000000    2003e040     ai_dmq3.obj
 0002:00001048       __real@43b40000            2003e048     ai_dmq3.obj
 0002:0000104c       __real@3bda740e            2003e04c     ai_dmq3.obj
 0002:00001050       __real@43160000            2003e050     ai_dmq3.obj
 0002:00001054       __real@45c80000            2003e054     ai_dmq3.obj
 0002:00001058       __real@4024000000000000    2003e058     ai_dmq3.obj
 0002:00001060       __real@4034000000000000    2003e060     ai_dmq3.obj
 0002:00001068       __real@4049000000000000    2003e068     ai_dmq3.obj
 0002:00001070       __real@42800000            2003e070     ai_dmq3.obj
 0002:00001078       __real@3fe3333333333333    2003e078     ai_dmq3.obj
 0002:00001080       __real@44800000            2003e080     ai_dmq3.obj
 0002:00001084       __real@41800000            2003e084     ai_dmq3.obj
 0002:00001088       __real@3f333333            2003e088     ai_dmq3.obj
 0002:0000108c       __real@45100000            2003e08c     ai_dmq3.obj
 0002:00001090       __real@3ecccccd            2003e090     ai_dmq3.obj
 0002:00001098       __real@407f400000000000    2003e098     ai_dmq3.obj
 0002:000010a0       __real@41400000            2003e0a0     ai_dmq3.obj
 0002:000010a4       ??_C@_0N@IFIOEJJO@mpq3tourney6?$AA@ 2003e0a4     ai_dmq3.obj
 0002:000010b8       __real@4020000000000000    2003e0b8     ai_dmq3.obj
 0002:000010c0       __real@44660000            2003e0c0     ai_dmq3.obj
 0002:000010c4       __real@43b00000            2003e0c4     ai_dmq3.obj
 0002:000010c8       __real@43980000            2003e0c8     ai_dmq3.obj
 0002:000010cc       __real@44280000            2003e0cc     ai_dmq3.obj
 0002:000010d0       __real@43ea0000            2003e0d0     ai_dmq3.obj
 0002:000010d4       __real@434c0000            2003e0d4     ai_dmq3.obj
 0002:000010d8       __real@44710000            2003e0d8     ai_dmq3.obj
 0002:000010dc       __real@442f0000            2003e0dc     ai_dmq3.obj
 0002:000010e0       ??_C@_0L@IMOIIFCE@q3tourney6?$AA@ 2003e0e0     ai_dmq3.obj
 0002:000010f0       __real@bff0000000000000    2003e0f0     ai_dmq3.obj
 0002:000010f8       __real@44000000            2003e0f8     ai_dmq3.obj
 0002:000010fc       ??_C@_06KJINILIP@health?$AA@ 2003e0fc     ai_dmq3.obj
 0002:00001104       ??_C@_05FECBCJJD@angle?$AA@ 2003e104     ai_dmq3.obj
 0002:0000110c       ??_C@_03MHHCOBAB@lip?$AA@  2003e10c     ai_dmq3.obj
 0002:00001110       __real@461c3c00            2003e110     ai_dmq3.obj
 0002:00001114       ??_C@_0N@EDJICHIO@target_delay?$AA@ 2003e114     ai_dmq3.obj
 0002:00001124       ??_C@_0N@JGBHMGAI@target_relay?$AA@ 2003e124     ai_dmq3.obj
 0002:00001134       ??_C@_0L@LNOJFPAO@func_timer?$AA@ 2003e134     ai_dmq3.obj
 0002:00001140       ??_C@_0BB@LKHFHPEP@trigger_multiple?$AA@ 2003e140     ai_dmq3.obj
 0002:00001158       __real@4014000000000000    2003e158     ai_dmq3.obj
 0002:00001160       ??_C@_0DO@JNGNHOKO@BotGetActivateGoal?3?5entity?5with?5@ 2003e160     ai_dmq3.obj
 0002:000011a0       ??_C@_0DA@LAOMJDKC@BotGetActivateGoal?3?5no?5entity?5wi@ 2003e1a0     ai_dmq3.obj
 0002:000011d0       ??_C@_06JJLAMBGK@target?$AA@ 2003e1d0     ai_dmq3.obj
 0002:000011d8       ??_C@_0DO@HIKLPKA@BotGetActivateGoal?3?5entity?5with?5@ 2003e1d8     ai_dmq3.obj
 0002:00001218       ??_C@_0L@FEPNPAJD@targetname?$AA@ 2003e218     ai_dmq3.obj
 0002:00001224       ??_C@_0M@PNMKBMEP@func_button?$AA@ 2003e224     ai_dmq3.obj
 0002:00001230       ??_C@_06NHCMNMEH@origin?$AA@ 2003e230     ai_dmq3.obj
 0002:00001238       ??_C@_0L@HLIKNEFC@spawnflags?$AA@ 2003e238     ai_dmq3.obj
 0002:00001244       ??_C@_09KJCKJKEG@func_door?$AA@ 2003e244     ai_dmq3.obj
 0002:00001250       ??_C@_09CNJINBGN@classname?$AA@ 2003e250     ai_dmq3.obj
 0002:0000125c       ??_C@_0DD@KCKJBPAH@BotGetActivateGoal?3?5no?5entity?5fo@ 2003e25c     ai_dmq3.obj
 0002:00001290       ??_C@_03COCDEFBB@?$CK?$CFd?$AA@ 2003e290     ai_dmq3.obj
 0002:00001294       ??_C@_0BF@GIIMEEEB@BotGoForActivateGoal?$AA@ 2003e294     ai_dmq3.obj
 0002:000012ac       ??_C@_0CE@HJEADBFH@BotCheckConsoleMessages?3?5reply?5c@ 2003e2ac     ai_dmq3.obj
 0002:000012d0       __real@3ff8000000000000    2003e2d0     ai_dmq3.obj
 0002:000012d8       ??_C@_0BK@IPGPBJPO@?$CK?$CK?$CK?$CK?5no?5valid?5reply?5?$CK?$CK?$CK?$CK?6?$AA@ 2003e2d8     ai_dmq3.obj
 0002:000012f4       ??_C@_0BK@ICOBFDNE@?9?9?9?9?9?9?9?9?9?9?9?9?9?9?9?9?9?9?9?9?9?9?9?9?6?$AA@ 2003e2f4     ai_dmq3.obj
 0002:00001310       ??_C@_0O@BBHMLBKC@bot_testrchat?$AA@ 2003e310     ai_dmq3.obj
 0002:00001320       ??_C@_01HIHLOKLC@1?$AA@    2003e320     ai_dmq3.obj
 0002:00001324       ??_C@_0CP@JEHKHMIG@EV_GENERAL_SOUND?3?5eventParm?5?$CI?$CFd?$CJ@ 2003e324     ai_dmq3.obj
 0002:00001354       ??_C@_0O@LBBMLEKM@?$CKfalling1?4wav?$AA@ 2003e354     ai_dmq3.obj
 0002:00001364       ??_C@_0CO@MPBFDNLO@EV_GLOBAL_SOUND?3?5eventParm?5?$CI?$CFd?$CJ?5@ 2003e364     ai_dmq3.obj
 0002:00001394       ??_C@_0BP@NBLBCCPC@sound?1items?1poweruprespawn?4wav?$AA@ 2003e394     ai_dmq3.obj
 0002:000013b4       ??_C@_0CB@MGIHMDHM@BotDeathmatchAI?3?5chat?5enter?5game@ 2003e3b4     ai_dmq3.obj
 0002:000013d8       ??_C@_0BM@EKLHMNBH@BotDeathmatchAI?3?5no?5ai?5node?$AA@ 2003e3d8     ai_dmq3.obj
 0002:000013f4       ??_C@_07FDOFLCLN@team?5?$CFs?$AA@ 2003e3f4     ai_dmq3.obj
 0002:000013fc       ??_C@_03OMLNFKE@sex?$AA@   2003e3fc     ai_dmq3.obj
 0002:00001400       ??_C@_0BH@KKMLANHJ@CTF?5without?5Blue?5Flag?6?$AA@ 2003e400     ai_dmq3.obj
 0002:00001418       ??_C@_0BG@HPNDPJMP@CTF?5without?5Red?5Flag?6?$AA@ 2003e418     ai_dmq3.obj
 0002:00001430       ??_C@_09OGEBNCBM@g_spSkill?$AA@ 2003e430     ai_dmq3.obj
 0002:0000143c       ??_C@_01FDFGLJHB@2?$AA@    2003e43c     ai_dmq3.obj
 0002:00001440       ??_C@_0BF@JHNEDFAH@bot_predictobstacles?$AA@ 2003e440     ai_dmq3.obj
 0002:00001458       ??_C@_0O@ILENLOKO@bot_challenge?$AA@ 2003e458     ai_dmq3.obj
 0002:00001468       ??_C@_0L@JNAIAIAH@bot_nochat?$AA@ 2003e468     ai_dmq3.obj
 0002:00001474       ??_C@_0N@JOELMLFL@bot_fastchat?$AA@ 2003e474     ai_dmq3.obj
 0002:00001484       ??_C@_0M@HIPNFLBG@bot_grapple?$AA@ 2003e484     ai_dmq3.obj
 0002:00001490       ??_C@_01GBGANLPD@0?$AA@    2003e490     ai_dmq3.obj
 0002:00001494       ??_C@_0P@OLNMGHML@bot_rocketjump?$AA@ 2003e494     ai_dmq3.obj
 0002:000014a4       ??_C@_0L@GFINLBEC@g_gametype?$AA@ 2003e4a4     ai_dmq3.obj
 0002:000014b0       ??_C@_08EAEOGCCG@onfollow?$AA@ 2003e4b0     ai_dmq3.obj
 0002:000014bc       ??_C@_09BJNHNGHD@ihaveflag?$AA@ 2003e4bc     ai_dmq3.obj
 0002:000014c8       ??_C@_08OKGPDOIO@teamtask?$AA@ 2003e4c8     ai_dmq3.obj
 0002:000014d4       ??_C@_02DPKJAMEF@?$CFd?$AA@ 2003e4d4     ai_dmq3.obj
 0002:000014d8       __real@43000000            2003e4d8     ai_dmq3.obj
 0002:000014dc       __real@4479c000            2003e4dc     ai_dmq3.obj
 0002:000014e0       ??_C@_0BE@HKMNOMAG@unknown?5print?5type?6?$AA@ 2003e4e0     ai_main.obj
 0002:000014f4       ??_C@_0L@CNJLHKJM@?$FO1Exit?3?5?$CFs?$AA@ 2003e4f4     ai_main.obj
 0002:00001500       ??_C@_0M@GLOCHAGD@?$FO1Fatal?3?5?$CFs?$AA@ 2003e500     ai_main.obj
 0002:0000150c       ??_C@_0M@LKBEKEOF@?$FO1Error?3?5?$CFs?$AA@ 2003e50c     ai_main.obj
 0002:00001518       ??_C@_0O@LHCIHOMB@?$FO3Warning?3?5?$CFs?$AA@ 2003e518     ai_main.obj
 0002:00001528       ??_C@_02DKCKIIND@?$CFs?$AA@ 2003e528     ai_main.obj
 0002:0000152c       ??_C@_0BM@BOKNIJ@?$ANarea?5?$CFd?0?5cluster?5?$CFd?5?5?5?5?5?5?5?$AA@ 2003e52c     ai_main.obj
 0002:00001548       ??_C@_0CI@JOJDDOJC@?$AN?$FO1Solid?$CB?5?5?5?5?5?5?5?5?5?5?5?5?5?5?5?5?5?5?5?5?5?5?5@ 2003e548     ai_main.obj
 0002:00001570       ??_C@_0O@IFLBEIIP@?$AN?$FO1SOLID?5area?$AA@ 2003e570     ai_main.obj
 0002:00001580       ??_C@_0M@DHMCHLIE@?$ANemtpy?5area?$AA@ 2003e580     ai_main.obj
 0002:0000158c       ??_C@_02KNHHEEKP@?5?5?$AA@ 2003e58c     ai_main.obj
 0002:00001590       ??_C@_01OCOKONAJ@L?$AA@    2003e590     ai_main.obj
 0002:00001594       ??_C@_0P@LMJINGO@l?2?$CFs?2c?2?$CFs?2a?2?$CFs?$AA@ 2003e594     ai_main.obj
 0002:000015a4       ??_C@_0L@IPEIBHBA@roaming?5?$CFs?$AA@ 2003e5a4     ai_main.obj
 0002:000015b0       ??_C@_0L@ICJBNMIF@harvesting?$AA@ 2003e5b0     ai_main.obj
 0002:000015bc       ??_C@_0BJ@PEPADENJ@attacking?5the?5enemy?5base?$AA@ 2003e5bc     ai_main.obj
 0002:000015d8       ??_C@_0P@FJHLCNGM@returning?5flag?$AA@ 2003e5d8     ai_main.obj
 0002:000015e8       ??_C@_0N@GBHDPJKL@rushing?5base?$AA@ 2003e5e8     ai_main.obj
 0002:000015f8       ??_C@_0P@PCPLLEMM@capturing?5flag?$AA@ 2003e5f8     ai_main.obj
 0002:00001608       ??_C@_0L@GKAIHKNA@killing?5?$CFs?$AA@ 2003e608     ai_main.obj
 0002:00001614       ??_C@_0BA@FNOGAFMM@getting?5item?5?$CFs?$AA@ 2003e614     ai_main.obj
 0002:00001624       ??_C@_0N@FMPLLINE@defending?5?$CFs?$AA@ 2003e624     ai_main.obj
 0002:00001634       ??_C@_0BA@MCDBGPCI@accompanying?5?$CFs?$AA@ 2003e634     ai_main.obj
 0002:00001644       ??_C@_0L@MCMCNIDL@helping?5?$CFs?$AA@ 2003e644     ai_main.obj
 0002:00001650       ??_C@_02OBCNPDDN@F?5?$AA@  2003e650     ai_main.obj
 0002:00001654       __real@bf800000            2003e654     ai_main.obj
 0002:00001658       ??_C@_0BE@IDNEOHBL@bot_interbreedwrite?$AA@ 2003e658     ai_main.obj
 0002:00001670       __real@3fdccccccccccccd    2003e670     ai_main.obj
 0002:00001678       __real@c3340000            2003e678     ai_main.obj
 0002:0000167c       __real@43700000            2003e67c     ai_main.obj
 0002:00001680       __real@3ea28f5c            2003e680     ai_main.obj
 0002:00001684       __real@43360b61            2003e684     ai_main.obj
 0002:00001688       __real@3a83126f            2003e688     ai_main.obj
 0002:00001690       __real@3f76800000000000    2003e690     ai_main.obj
 0002:00001698       ??_C@_0BP@MGBLPCKB@BotAI?3?5client?5?$CFd?5is?5not?5setup?6?$AA@ 2003e698     ai_main.obj
 0002:000016b8       ??_C@_0BA@GNMFKLDC@clientLevelShot?$AA@ 2003e6b8     ai_main.obj
 0002:000016c8       ??_C@_06KBCJDMLG@scores?$AA@ 2003e6c8     ai_main.obj
 0002:000016d0       ??_C@_05PMMINOBP@tchat?$AA@ 2003e6d0     ai_main.obj
 0002:000016d8       ??_C@_04BLJLMHHG@chat?$AA@ 2003e6d8     ai_main.obj
 0002:000016e0       ??_C@_05IJDJACGD@print?$AA@ 2003e6e0     ai_main.obj
 0002:000016e8       ??_C@_02EODNHJKB@cs?$AA@   2003e6e8     ai_main.obj
 0002:000016ec       ??_C@_03DGFNDEPM@cp?5?$AA@ 2003e6ec     ai_main.obj
 0002:000016f0       ??_C@_0N@BLBFMIAO@botsession?$CFi?$AA@ 2003e6f0     ai_main.obj
 0002:00001700       ??_C@_0DD@CAOHNHKP@?$CFi?5?$CFi?5?$CFi?5?$CFi?5?$CFi?5?$CFi?5?$CFi?5?$CFi?5?$CFf?5?$CFf?5?$CFf@ 2003e700     ai_main.obj
 0002:00001734       ??_C@_0O@HIGNEDPK@bot_testichat?$AA@ 2003e734     ai_main.obj
 0002:00001744       ??_C@_0CA@KCEBJEJI@couldn?8t?5load?5skill?5?$CFf?5from?5?$CFs?6?$AA@ 2003e744     ai_main.obj
 0002:00001764       ??_C@_0BF@PINCHNMN@AAS?5not?5initialized?6?$AA@ 2003e764     ai_main.obj
 0002:0000177c       ??_C@_0CL@MOACODCL@BotAISetupClient?3?5client?5?$CFd?5alre@ 2003e77c     ai_main.obj
 0002:000017a8       ??_C@_05ECKEHJKK@cddir?$AA@ 2003e7a8     ai_main.obj
 0002:000017b0       ??_C@_09CIALLHHK@fs_cdpath?$AA@ 2003e7b0     ai_main.obj
 0002:000017bc       ??_C@_07GGMBKBFD@gamedir?$AA@ 2003e7bc     ai_main.obj
 0002:000017c4       ??_C@_07FMAMAFJE@fs_game?$AA@ 2003e7c4     ai_main.obj
 0002:000017cc       ??_C@_07BHPNMMNM@basedir?$AA@ 2003e7cc     ai_main.obj
 0002:000017d4       ??_C@_0M@DGDBFJN@fs_basepath?$AA@ 2003e7d4     ai_main.obj
 0002:000017e0       ??_C@_0BF@BBFOCAKO@bot_reloadcharacters?$AA@ 2003e7e0     ai_main.obj
 0002:000017f8       ??_C@_0BB@GMCJAANP@saveroutingcache?$AA@ 2003e7f8     ai_main.obj
 0002:0000180c       ??_C@_0BF@MDEDPJEF@bot_saveroutingcache?$AA@ 2003e80c     ai_main.obj
 0002:00001824       ??_C@_0M@MFMPGCMK@aasoptimize?$AA@ 2003e824     ai_main.obj
 0002:00001830       ??_C@_0BA@CHMPBPHA@bot_aasoptimize?$AA@ 2003e830     ai_main.obj
 0002:00001840       ??_C@_0L@MNCDALON@forcewrite?$AA@ 2003e840     ai_main.obj
 0002:0000184c       ??_C@_0P@HFCEKFCE@bot_forcewrite?$AA@ 2003e84c     ai_main.obj
 0002:0000185c       ??_C@_0BC@HJNNPMHF@forcereachability?$AA@ 2003e85c     ai_main.obj
 0002:00001870       ??_C@_0BG@GJKIOMNG@bot_forcereachability?$AA@ 2003e870     ai_main.obj
 0002:00001888       ??_C@_0BA@BADKHCEE@forceclustering?$AA@ 2003e888     ai_main.obj
 0002:00001898       ??_C@_0BE@HANIKEON@bot_forceclustering?$AA@ 2003e898     ai_main.obj
 0002:000018ac       ??_C@_0BG@HILKKLKJ@bot_visualizejumppads?$AA@ 2003e8ac     ai_main.obj
 0002:000018c4       ??_C@_06GCPOGFCC@nochat?$AA@ 2003e8c4     ai_main.obj
 0002:000018cc       ??_C@_03MGHMBJCF@log?$AA@  2003e8cc     ai_main.obj
 0002:000018d0       ??_C@_0O@IHEJFHJE@bot_developer?$AA@ 2003e8d0     ai_main.obj
 0002:000018e0       ??_C@_0P@HIDOFLAM@max_levelitems?$AA@ 2003e8e0     ai_main.obj
 0002:000018f0       ??_C@_0N@PMPJOGOE@max_aaslinks?$AA@ 2003e8f0     ai_main.obj
 0002:00001900       ??_C@_0P@HEEKJLPJ@sv_mapChecksum?$AA@ 2003e900     ai_main.obj
 0002:00001910       ??_C@_0M@KCCINJFC@maxentities?$AA@ 2003e910     ai_main.obj
 0002:0000191c       ??_C@_0L@JKCONGEA@maxclients?$AA@ 2003e91c     ai_main.obj
 0002:00001928       ??_C@_0BE@BBMLIECL@bot_interbreedcycle?$AA@ 2003e928     ai_main.obj
 0002:0000193c       ??_C@_02PIBHCBOA@20?$AA@   2003e93c     ai_main.obj
 0002:00001940       ??_C@_0BD@GLHGHIJE@bot_interbreedbots?$AA@ 2003e940     ai_main.obj
 0002:00001954       ??_C@_02PKFBJPLJ@10?$AA@   2003e954     ai_main.obj
 0002:00001958       ??_C@_0BD@MIDHDJEH@bot_interbreedchar?$AA@ 2003e958     ai_main.obj
 0002:0000196c       ??_C@_0BB@LICKAML@bot_testclusters?$AA@ 2003e96c     ai_main.obj
 0002:00001980       ??_C@_0O@NEGDFLLI@bot_testsolid?$AA@ 2003e980     ai_main.obj
 0002:00001990       ??_C@_0L@DIBKBFBJ@bot_report?$AA@ 2003e990     ai_main.obj
 0002:0000199c       ??_C@_09KJGEBPM@bot_pause?$AA@ 2003e99c     ai_main.obj
 0002:000019a8       ??_C@_0P@CMKPBNJI@bot_memorydump?$AA@ 2003e9a8     ai_main.obj
 0002:000019b8       ??_C@_0O@NKIABNEG@bot_thinktime?$AA@ 2003e9b8     ai_main.obj
 0002:000019c8       ??_C@_03GNABGMEE@100?$AA@  2003e9c8     ai_main.obj
 0002:000019cc       ??_C@_0BK@CCAPHDJA@addbot?5?$CFs?54?5free?5?$CFi?5?$CFs?$CFd?6?$AA@ 2003e9cc     ai_main.obj
 0002:000019e8       ??_C@_03HPLEMDKK@200?$AA@  2003e9e8     ai_main.obj
 0002:000019ec       ??_C@_0L@JEKILDFB@memorydump?$AA@ 2003e9ec     ai_main.obj
 0002:000019f8       ??_C@_0M@CFKBBDNA@?$BJ?$CI?$CFs?$BJ?$CJ?$BJ?3?5?$CFs?$AA@ 2003e9f8     ai_team.obj
 0002:00001a04       ??_C@_0M@KCHJGFOM@cmd_getflag?$AA@ 2003ea04     ai_team.obj
 0002:00001a10       ??_C@_0O@FNPCOJLM@cmd_accompany?$AA@ 2003ea10     ai_team.obj
 0002:00001a20       ??_C@_0BA@MJCDCBAL@cmd_accompanyme?$AA@ 2003ea20     ai_team.obj
 0002:00001a30       ??_C@_0P@MGOFKCGO@cmd_defendbase?$AA@ 2003ea30     ai_team.obj
 0002:00001a40       ??_C@_0O@EHLIMCMK@iamteamleader?$AA@ 2003ea40     ai_team.obj
 0002:00001a50       ??_C@_0BA@JCHIJEGJ@whoisteamleader?$AA@ 2003ea50     ai_team.obj
 0002:00001a60       ??_C@_0O@LCEABBKD@wantonoffense?$AA@ 2003ea60     ai_vcmd.obj
 0002:00001a70       ??_C@_0O@NOMCBHGI@wantondefense?$AA@ 2003ea70     ai_vcmd.obj
 0002:00001a80       ??_C@_0M@JLDAEMIJ@whoisleader?$AA@ 2003ea80     ai_vcmd.obj
 0002:00001a8c       ??_C@_0L@HELMBEII@stopleader?$AA@ 2003ea8c     ai_vcmd.obj
 0002:00001a98       ??_C@_0M@GEDMEPM@startleader?$AA@ 2003ea98     ai_vcmd.obj
 0002:00001aa4       ??_C@_0L@BCFFODB@returnflag?$AA@ 2003eaa4     ai_vcmd.obj
 0002:00001ab0       ??_C@_0BC@HILCMIJJ@followflagcarrier?$AA@ 2003eab0     ai_vcmd.obj
 0002:00001ac4       ??_C@_04LOFLEJM@camp?$AA@  2003eac4     ai_vcmd.obj
 0002:00001acc       ??_C@_06KPEKKPL@patrol?$AA@ 2003eacc     ai_vcmd.obj
 0002:00001ad4       ??_C@_0L@LIAONOLJ@defendflag?$AA@ 2003ead4     ai_vcmd.obj
 0002:00001ae0       ??_C@_06BMABBLML@defend?$AA@ 2003eae0     ai_vcmd.obj
 0002:00001ae8       ??_C@_07GBMLDGPP@offense?$AA@ 2003eae8     ai_vcmd.obj
 0002:00001af0       ??_C@_07NOFDDIA@getflag?$AA@ 2003eaf0     ai_vcmd.obj
 0002:00001af8       ??_C@_08DHCKJNNH@onpatrol?$AA@ 2003eaf8     ai_vcmd.obj
 0002:00001b04       ??_C@_08GBKLDCBE@EV_TAUNT?$AA@ 2003eb04     bg_misc.obj
 0002:00001b10       ??_C@_0BE@OHJHDFJH@EV_STOPLOOPINGSOUND?$AA@ 2003eb10     bg_misc.obj
 0002:00001b24       ??_C@_0O@PBPAKHP@EV_DEBUG_LINE?$AA@ 2003eb24     bg_misc.obj
 0002:00001b34       ??_C@_0BB@HHACOGHI@EV_LIGHTNINGBOLT?$AA@ 2003eb34     bg_misc.obj
 0002:00001b48       ??_C@_09GLJGDJEJ@EV_JUICED?$AA@ 2003eb48     bg_misc.obj
 0002:00001b54       ??_C@_0BA@NHKGBGBA@EV_INVUL_IMPACT?$AA@ 2003eb54     bg_misc.obj
 0002:00001b64       ??_C@_0BC@LMKNBBLF@EV_OBELISKEXPLODE?$AA@ 2003eb64     bg_misc.obj
 0002:00001b78       ??_C@_0M@KACLGFEA@EV_KAMIKAZE?$AA@ 2003eb78     bg_misc.obj
 0002:00001b84       ??_C@_0BK@PIFCIJEJ@EV_PROXIMITY_MINE_TRIGGER?$AA@ 2003eb84     bg_misc.obj
 0002:00001ba0       ??_C@_0BI@KNJAKDGK@EV_PROXIMITY_MINE_STICK?$AA@ 2003eba0     bg_misc.obj
 0002:00001bb8       ??_C@_0N@GAJBP@EV_SCOREPLUM?$AA@ 2003ebb8     bg_misc.obj
 0002:00001bc8       ??_C@_0O@JLGFLKBE@EV_GIB_PLAYER?$AA@ 2003ebc8     bg_misc.obj
 0002:00001bd8       ??_C@_0BB@EGIJIDAN@EV_POWERUP_REGEN?$AA@ 2003ebd8     bg_misc.obj
 0002:00001bec       ??_C@_0BG@CHAMNADK@EV_POWERUP_BATTLESUIT?$AA@ 2003ebec     bg_misc.obj
 0002:00001c04       ??_C@_0BA@HLHGHIIE@EV_POWERUP_QUAD?$AA@ 2003ec04     bg_misc.obj
 0002:00001c14       ??_C@_0M@PPLCDPP@EV_OBITUARY?$AA@ 2003ec14     bg_misc.obj
 0002:00001c20       ??_C@_09KNGHBIAK@EV_DEATH3?$AA@ 2003ec20     bg_misc.obj
 0002:00001c2c       ??_C@_09LEHMCJEL@EV_DEATH2?$AA@ 2003ec2c     bg_misc.obj
 0002:00001c38       ??_C@_09JPFBHKII@EV_DEATH1?$AA@ 2003ec38     bg_misc.obj
 0002:00001c44       ??_C@_07EMHHKOOH@EV_PAIN?$AA@ 2003ec44     bg_misc.obj
 0002:00001c4c       ??_C@_09ICDIPKFJ@EV_BULLET?$AA@ 2003ec4c     bg_misc.obj
 0002:00001c58       ??_C@_0L@LHBIHDML@EV_SHOTGUN?$AA@ 2003ec58     bg_misc.obj
 0002:00001c64       ??_C@_0N@HMLLJFGF@EV_RAILTRAIL?$AA@ 2003ec64     bg_misc.obj
 0002:00001c74       ??_C@_0BG@LPAHEABB@EV_MISSILE_MISS_METAL?$AA@ 2003ec74     bg_misc.obj
 0002:00001c8c       ??_C@_0BA@CAHALNAE@EV_MISSILE_MISS?$AA@ 2003ec8c     bg_misc.obj
 0002:00001c9c       ??_C@_0P@JFMFNBMO@EV_MISSILE_HIT?$AA@ 2003ec9c     bg_misc.obj
 0002:00001cac       ??_C@_0BD@MFLMCLPN@EV_BULLET_HIT_WALL?$AA@ 2003ecac     bg_misc.obj
 0002:00001cc0       ??_C@_0BE@KBABEJMP@EV_BULLET_HIT_FLESH?$AA@ 2003ecc0     bg_misc.obj
 0002:00001cd4       ??_C@_0BF@DDOIKLHD@EV_GLOBAL_TEAM_SOUND?$AA@ 2003ecd4     bg_misc.obj
 0002:00001cec       ??_C@_0BA@JAMKLOPJ@EV_GLOBAL_SOUND?$AA@ 2003ecec     bg_misc.obj
 0002:00001cfc       ??_C@_0BB@LJGGMAII@EV_GENERAL_SOUND?$AA@ 2003ecfc     bg_misc.obj
 0002:00001d10       ??_C@_0BC@ECIIAFLJ@EV_GRENADE_BOUNCE?$AA@ 2003ed10     bg_misc.obj
 0002:00001d24       ??_C@_0BH@FNNILPIN@EV_PLAYER_TELEPORT_OUT?$AA@ 2003ed24     bg_misc.obj
 0002:00001d3c       ??_C@_0BG@HBBJKNDP@EV_PLAYER_TELEPORT_IN?$AA@ 2003ed3c     bg_misc.obj
 0002:00001d54       ??_C@_0M@ECGFPIMP@EV_ITEM_POP?$AA@ 2003ed54     bg_misc.obj
 0002:00001d60       ??_C@_0BA@GJNCODNG@EV_ITEM_RESPAWN?$AA@ 2003ed60     bg_misc.obj
 0002:00001d70       ??_C@_0O@HHGOLJPJ@EV_USE_ITEM15?$AA@ 2003ed70     bg_misc.obj
 0002:00001d80       ??_C@_0O@GOHFIILI@EV_USE_ITEM14?$AA@ 2003ed80     bg_misc.obj
 0002:00001d90       ??_C@_0O@CBDEBOHP@EV_USE_ITEM13?$AA@ 2003ed90     bg_misc.obj
 0002:00001da0       ??_C@_0O@DICPCPDO@EV_USE_ITEM12?$AA@ 2003eda0     bg_misc.obj
 0002:00001db0       ??_C@_0O@BDACHMPN@EV_USE_ITEM11?$AA@ 2003edb0     bg_misc.obj
 0002:00001dc0       ??_C@_0O@KBJENLM@EV_USE_ITEM10?$AA@ 2003edc0     bg_misc.obj
 0002:00001dd0       ??_C@_0N@PHODCBCK@EV_USE_ITEM9?$AA@ 2003edd0     bg_misc.obj
 0002:00001de0       ??_C@_0N@OOPIBAGL@EV_USE_ITEM8?$AA@ 2003ede0     bg_misc.obj
 0002:00001df0       ??_C@_0N@GJGAAMKE@EV_USE_ITEM7?$AA@ 2003edf0     bg_misc.obj
 0002:00001e00       ??_C@_0N@HAHLDNOF@EV_USE_ITEM6?$AA@ 2003ee00     bg_misc.obj
 0002:00001e10       ??_C@_0N@FLFGGOCG@EV_USE_ITEM5?$AA@ 2003ee10     bg_misc.obj
 0002:00001e20       ??_C@_0N@ECENFPGH@EV_USE_ITEM4?$AA@ 2003ee20     bg_misc.obj
 0002:00001e30       ??_C@_0N@NAMMJKA@EV_USE_ITEM3?$AA@ 2003ee30     bg_misc.obj
 0002:00001e40       ??_C@_0N@BEBHPIOB@EV_USE_ITEM2?$AA@ 2003ee40     bg_misc.obj
 0002:00001e50       ??_C@_0N@DPDKKLCC@EV_USE_ITEM1?$AA@ 2003ee50     bg_misc.obj
 0002:00001e60       ??_C@_0N@CGCBJKGD@EV_USE_ITEM0?$AA@ 2003ee60     bg_misc.obj
 0002:00001e70       ??_C@_0P@PFJPAFGH@EV_FIRE_WEAPON?$AA@ 2003ee70     bg_misc.obj
 0002:00001e80       ??_C@_0BB@ENKPHJLP@EV_CHANGE_WEAPON?$AA@ 2003ee80     bg_misc.obj
 0002:00001e94       ??_C@_09NMIICG@EV_NOAMMO?$AA@ 2003ee94     bg_misc.obj
 0002:00001ea0       ??_C@_0BG@KFILGAMN@EV_GLOBAL_ITEM_PICKUP?$AA@ 2003eea0     bg_misc.obj
 0002:00001eb8       ??_C@_0P@BGIOEPCB@EV_ITEM_PICKUP?$AA@ 2003eeb8     bg_misc.obj
 0002:00001ec8       ??_C@_0P@NIPCJOBG@EV_WATER_CLEAR?$AA@ 2003eec8     bg_misc.obj
 0002:00001ed8       ??_C@_0P@MIAIODEJ@EV_WATER_UNDER?$AA@ 2003eed8     bg_misc.obj
 0002:00001ee8       ??_C@_0P@LHDMOIIG@EV_WATER_LEAVE?$AA@ 2003eee8     bg_misc.obj
 0002:00001ef8       ??_C@_0P@GCDBKPMP@EV_WATER_TOUCH?$AA@ 2003eef8     bg_misc.obj
 0002:00001f08       ??_C@_07GKBEHGAP@EV_JUMP?$AA@ 2003ef08     bg_misc.obj
 0002:00001f10       ??_C@_0M@BPNFGBOJ@EV_JUMP_PAD?$AA@ 2003ef10     bg_misc.obj
 0002:00001f1c       ??_C@_0M@LKJJNJOM@EV_FALL_FAR?$AA@ 2003ef1c     bg_misc.obj
 0002:00001f28       ??_C@_0P@MGFLMCKC@EV_FALL_MEDIUM?$AA@ 2003ef28     bg_misc.obj
 0002:00001f38       ??_C@_0O@EAFDHAJM@EV_FALL_SHORT?$AA@ 2003ef38     bg_misc.obj
 0002:00001f48       ??_C@_0L@HOOIOPKF@EV_STEP_16?$AA@ 2003ef48     bg_misc.obj
 0002:00001f54       ??_C@_0L@BKIECKKB@EV_STEP_12?$AA@ 2003ef54     bg_misc.obj
 0002:00001f60       ??_C@_09EHOLDGNN@EV_STEP_8?$AA@ 2003ef60     bg_misc.obj
 0002:00001f6c       ??_C@_09OLFOHJNB@EV_STEP_4?$AA@ 2003ef6c     bg_misc.obj
 0002:00001f78       ??_C@_07FFIIIPLH@EV_SWIM?$AA@ 2003ef78     bg_misc.obj
 0002:00001f80       ??_C@_0M@NPJBGELA@EV_FOOTWADE?$AA@ 2003ef80     bg_misc.obj
 0002:00001f8c       ??_C@_0O@HLJHKIDH@EV_FOOTSPLASH?$AA@ 2003ef8c     bg_misc.obj
 0002:00001f9c       ??_C@_0BC@DIJMAMMI@EV_FOOTSTEP_METAL?$AA@ 2003ef9c     bg_misc.obj
 0002:00001fb0       ??_C@_0M@HLKBOJPO@EV_FOOTSTEP?$AA@ 2003efb0     bg_misc.obj
 0002:00001fbc       ??_C@_07JFMDDPHJ@EV_NONE?$AA@ 2003efbc     bg_misc.obj
 0002:00001fc4       ??_C@_0BB@EMIIAFKA@icons?1iconf_blu1?$AA@ 2003efc4     bg_misc.obj
 0002:00001fd8       ??_C@_0BI@FKICCNIF@models?1flags?1b_flag?4md3?$AA@ 2003efd8     bg_misc.obj
 0002:00001ff0       ??_C@_0BC@NLKCOFAB@team_CTF_blueflag?$AA@ 2003eff0     bg_misc.obj
 0002:00002004       ??_C@_0BB@EMIEBEOP@icons?1iconf_red1?$AA@ 2003f004     bg_misc.obj
 0002:00002018       ??_C@_0BI@PEHEOJEO@models?1flags?1r_flag?4md3?$AA@ 2003f018     bg_misc.obj
 0002:00002030       ??_C@_0BB@JNMMCIHG@team_CTF_redflag?$AA@ 2003f030     bg_misc.obj
 0002:00002044       ??_C@_0N@GLEPEEPG@icons?1flight?$AA@ 2003f044     bg_misc.obj
 0002:00002054       ??_C@_0CI@IADFFEDP@models?1powerups?1instant?1flight_r@ 2003f054     bg_misc.obj
 0002:0000207c       ??_C@_0CD@MKDGJOMG@models?1powerups?1instant?1flight?4m@ 2003f07c     bg_misc.obj
 0002:000020a0       ??_C@_0BH@COLFHEAE@sound?1items?1flight?4wav?$AA@ 2003f0a0     bg_misc.obj
 0002:000020b8       ??_C@_0M@MBNKEMMH@item_flight?$AA@ 2003f0b8     bg_misc.obj
 0002:000020c4       ??_C@_0BG@LHDLOKKN@sound?1items?1regen?4wav?$AA@ 2003f0c4     bg_misc.obj
 0002:000020dc       ??_C@_0M@FDCLJBFC@icons?1regen?$AA@ 2003f0dc     bg_misc.obj
 0002:000020e8       ??_C@_0CH@FANACKJM@models?1powerups?1instant?1regen_ri@ 2003f0e8     bg_misc.obj
 0002:00002110       ??_C@_0CC@OEAPIKIN@models?1powerups?1instant?1regen?4md@ 2003f110     bg_misc.obj
 0002:00002134       ??_C@_0BN@OBGKHNFF@sound?1items?1regeneration?4wav?$AA@ 2003f134     bg_misc.obj
 0002:00002154       ??_C@_0L@MMGPPPDM@item_regen?$AA@ 2003f154     bg_misc.obj
 0002:00002160       ??_C@_0M@FDDJPHJJ@icons?1invis?$AA@ 2003f160     bg_misc.obj
 0002:0000216c       ??_C@_0CH@IMIHJDNC@models?1powerups?1instant?1invis_ri@ 2003f16c     bg_misc.obj
 0002:00002194       ??_C@_0CC@HBONCEML@models?1powerups?1instant?1invis?4md@ 2003f194     bg_misc.obj
 0002:000021b8       ??_C@_0BN@OJBEBLGB@sound?1items?1invisibility?4wav?$AA@ 2003f1b8     bg_misc.obj
 0002:000021d8       ??_C@_0L@MMHNJJPH@item_invis?$AA@ 2003f1d8     bg_misc.obj
 0002:000021e4       ??_C@_0M@CFINMGCL@icons?1haste?$AA@ 2003f1e4     bg_misc.obj
 0002:000021f0       ??_C@_0CH@KKDDKNEF@models?1powerups?1instant?1haste_ri@ 2003f1f0     bg_misc.obj
 0002:00002218       ??_C@_0CC@NKPAJCMI@models?1powerups?1instant?1haste?4md@ 2003f218     bg_misc.obj
 0002:0000223c       ??_C@_0BG@IJMEPCOI@sound?1items?1haste?4wav?$AA@ 2003f23c     bg_misc.obj
 0002:00002254       ??_C@_0L@LKMJKIEF@item_haste?$AA@ 2003f254     bg_misc.obj
 0002:00002260       ??_C@_0DA@OCPACKGN@sound?1items?1airout?4wav?5sound?1ite@ 2003f260     bg_misc.obj
 0002:00002290       ??_C@_0BB@MGICBJOH@icons?1envirosuit?$AA@ 2003f290     bg_misc.obj
 0002:000022a4       ??_C@_0CI@KAEDJDGE@models?1powerups?1instant?1enviro_r@ 2003f2a4     bg_misc.obj
 0002:000022cc       ??_C@_0CD@JLGNIGLA@models?1powerups?1instant?1enviro?4m@ 2003f2cc     bg_misc.obj
 0002:000022f0       ??_C@_0BI@DEKBIKDD@sound?1items?1protect?4wav?$AA@ 2003f2f0     bg_misc.obj
 0002:00002308       ??_C@_0M@HBCGNAN@item_enviro?$AA@ 2003f308     bg_misc.obj
 0002:00002314       ??_C@_0DA@PPPPKFJI@sound?1items?1damage2?4wav?5sound?1it@ 2003f314     bg_misc.obj
 0002:00002344       ??_C@_0L@DICHEOBB@icons?1quad?$AA@ 2003f344     bg_misc.obj
 0002:00002350       ??_C@_0CG@JNMBMLHJ@models?1powerups?1instant?1quad_rin@ 2003f350     bg_misc.obj
 0002:00002378       ??_C@_0CB@HIFGFDGN@models?1powerups?1instant?1quad?4md3@ 2003f378     bg_misc.obj
 0002:0000239c       ??_C@_0BL@GLEJLOCA@sound?1items?1quaddamage?4wav?$AA@ 2003f39c     bg_misc.obj
 0002:000023b8       ??_C@_09MDKNIFFH@item_quad?$AA@ 2003f3b8     bg_misc.obj
 0002:000023c4       ??_C@_0BL@GLIFPGGG@sound?1items?1use_medkit?4wav?$AA@ 2003f3c4     bg_misc.obj
 0002:000023e0       ??_C@_06JDLGEHAD@Medkit?$AA@ 2003f3e0     bg_misc.obj
 0002:000023e8       ??_C@_0N@PNMDFAPK@icons?1medkit?$AA@ 2003f3e8     bg_misc.obj
 0002:000023f8       ??_C@_0CL@LOBKLABC@models?1powerups?1holdable?1medkit_@ 2003f3f8     bg_misc.obj
 0002:00002424       ??_C@_0CE@NKMJILL@models?1powerups?1holdable?1medkit?4@ 2003f424     bg_misc.obj
 0002:00002448       ??_C@_0BA@PDDMBOCP@holdable_medkit?$AA@ 2003f448     bg_misc.obj
 0002:00002458       ??_C@_0BE@PCKJDFFA@Personal?5Teleporter?$AA@ 2003f458     bg_misc.obj
 0002:0000246c       ??_C@_0BB@HCFICFKF@icons?1teleporter?$AA@ 2003f46c     bg_misc.obj
 0002:00002480       ??_C@_0CI@FHEOFFOB@models?1powerups?1holdable?1telepor@ 2003f480     bg_misc.obj
 0002:000024a8       ??_C@_0BJ@PNIOAJDI@sound?1items?1holdable?4wav?$AA@ 2003f4a8     bg_misc.obj
 0002:000024c4       ??_C@_0BE@GNEKBMLB@holdable_teleporter?$AA@ 2003f4c4     bg_misc.obj
 0002:000024d8       ??_C@_08LIBOGPIN@Bfg?5Ammo?$AA@ 2003f4d8     bg_misc.obj
 0002:000024e4       ??_C@_0BA@NIKNDLKG@icons?1icona_bfg?$AA@ 2003f4e4     bg_misc.obj
 0002:000024f4       ??_C@_0BP@BOBKFIKJ@models?1powerups?1ammo?1bfgam?4md3?$AA@ 2003f4f4     bg_misc.obj
 0002:00002514       ??_C@_08EHEJHGBG@ammo_bfg?$AA@ 2003f514     bg_misc.obj
 0002:00002520       ??_C@_05INIOBJHH@Slugs?$AA@ 2003f520     bg_misc.obj
 0002:00002528       ??_C@_0BE@DPOADFL@icons?1icona_railgun?$AA@ 2003f528     bg_misc.obj
 0002:0000253c       ??_C@_0CD@CAJEPMME@models?1powerups?1ammo?1railgunam?4m@ 2003f53c     bg_misc.obj
 0002:00002560       ??_C@_0L@JEFOIHIM@ammo_slugs?$AA@ 2003f560     bg_misc.obj
 0002:0000256c       ??_C@_07MLLADOAB@Rockets?$AA@ 2003f56c     bg_misc.obj
 0002:00002574       ??_C@_0BD@BFBJLPJK@icons?1icona_rocket?$AA@ 2003f574     bg_misc.obj
 0002:00002588       ??_C@_0CC@KCOEDLFM@models?1powerups?1ammo?1rocketam?4md@ 2003f588     bg_misc.obj
 0002:000025ac       ??_C@_0N@CLEPKBOE@ammo_rockets?$AA@ 2003f5ac     bg_misc.obj
 0002:000025bc       ??_C@_09JCCOMJEA@Lightning?$AA@ 2003f5bc     bg_misc.obj
 0002:000025c8       ??_C@_0BG@MEGMAGOM@icons?1icona_lightning?$AA@ 2003f5c8     bg_misc.obj
 0002:000025e0       ??_C@_0CF@HDAADIIL@models?1powerups?1ammo?1lightningam@ 2003f5e0     bg_misc.obj
 0002:00002608       ??_C@_0P@NBJHKAMD@ammo_lightning?$AA@ 2003f608     bg_misc.obj
 0002:00002618       ??_C@_05KCAMIOGJ@Cells?$AA@ 2003f618     bg_misc.obj
 0002:00002620       ??_C@_0BD@NCNJEHKB@icons?1icona_plasma?$AA@ 2003f620     bg_misc.obj
 0002:00002634       ??_C@_0CC@FGLALJGN@models?1powerups?1ammo?1plasmaam?4md@ 2003f634     bg_misc.obj
 0002:00002658       ??_C@_0L@LLNMBAJC@ammo_cells?$AA@ 2003f658     bg_misc.obj
 0002:00002664       ??_C@_08PMBIADEN@Grenades?$AA@ 2003f664     bg_misc.obj
 0002:00002670       ??_C@_0BE@LHOKGGAM@icons?1icona_grenade?$AA@ 2003f670     bg_misc.obj
 0002:00002684       ??_C@_0CD@HNOBKKLC@models?1powerups?1ammo?1grenadeam?4m@ 2003f684     bg_misc.obj
 0002:000026a8       ??_C@_0O@CMJIOKCF@ammo_grenades?$AA@ 2003f6a8     bg_misc.obj
 0002:000026b8       ??_C@_07DHNDKCGP@Bullets?$AA@ 2003f6b8     bg_misc.obj
 0002:000026c0       ??_C@_0BH@HMOAGCNP@icons?1icona_machinegun?$AA@ 2003f6c0     bg_misc.obj
 0002:000026d8       ??_C@_0CG@OLENEOKN@models?1powerups?1ammo?1machineguna@ 2003f6d8     bg_misc.obj
 0002:00002700       ??_C@_0N@NHCMDNIK@ammo_bullets?$AA@ 2003f700     bg_misc.obj
 0002:00002710       ??_C@_06PBPEPGGL@Shells?$AA@ 2003f710     bg_misc.obj
 0002:00002718       ??_C@_0BE@NMAFHJEI@icons?1icona_shotgun?$AA@ 2003f718     bg_misc.obj
 0002:0000272c       ??_C@_0CD@MBAGJHDE@models?1powerups?1ammo?1shotgunam?4m@ 2003f72c     bg_misc.obj
 0002:00002750       ??_C@_0BH@DPAADLFH@sound?1misc?1am_pkup?4wav?$AA@ 2003f750     bg_misc.obj
 0002:00002768       ??_C@_0M@NLICANGB@ammo_shells?$AA@ 2003f768     bg_misc.obj
 0002:00002774       ??_C@_0P@CFJPDDC@Grappling?5Hook?$AA@ 2003f774     bg_misc.obj
 0002:00002784       ??_C@_0BE@DPKNJNBE@icons?1iconw_grapple?$AA@ 2003f784     bg_misc.obj
 0002:00002798       ??_C@_0CE@LFAGANA@models?1weapons2?1grapple?1grapple?4@ 2003f798     bg_misc.obj
 0002:000027bc       ??_C@_0BF@MEMGGPGH@weapon_grapplinghook?$AA@ 2003f7bc     bg_misc.obj
 0002:000027d4       ??_C@_0BA@NCCNKCA@icons?1iconw_bfg?$AA@ 2003f7d4     bg_misc.obj
 0002:000027e4       ??_C@_0BM@HHDGGOHP@models?1weapons2?1bfg?1bfg?4md3?$AA@ 2003f7e4     bg_misc.obj
 0002:00002800       ??_C@_0L@JBGNLNGG@weapon_bfg?$AA@ 2003f800     bg_misc.obj
 0002:0000280c       ??_C@_0L@JFFCGJF@Plasma?5Gun?$AA@ 2003f80c     bg_misc.obj
 0002:00002818       ??_C@_0BD@NADHMFK@icons?1iconw_plasma?$AA@ 2003f818     bg_misc.obj
 0002:0000282c       ??_C@_0CC@EHGHEDND@models?1weapons2?1plasma?1plasma?4md@ 2003f82c     bg_misc.obj
 0002:00002850       ??_C@_0BB@LBHAKENA@weapon_plasmagun?$AA@ 2003f850     bg_misc.obj
 0002:00002864       ??_C@_0BE@CJEOPCPE@icons?1iconw_railgun?$AA@ 2003f864     bg_misc.obj
 0002:00002878       ??_C@_0CE@JHJFFEBE@models?1weapons2?1railgun?1railgun?4@ 2003f878     bg_misc.obj
 0002:0000289c       ??_C@_0P@FEPBKEBF@weapon_railgun?$AA@ 2003f89c     bg_misc.obj
 0002:000028ac       ??_C@_0BG@CHEJEOPA@icons?1iconw_lightning?$AA@ 2003f8ac     bg_misc.obj
 0002:000028c4       ??_C@_0CI@MNAFJDPO@models?1weapons2?1lightning?1lightn@ 2003f8c4     bg_misc.obj
 0002:000028ec       ??_C@_0BB@OCCEAFCD@weapon_lightning?$AA@ 2003f8ec     bg_misc.obj
 0002:00002900       ??_C@_0BD@MKMDIEGB@icons?1iconw_rocket?$AA@ 2003f900     bg_misc.obj
 0002:00002914       ??_C@_0CE@GGGFLKKE@models?1weapons2?1rocketl?1rocketl?4@ 2003f914     bg_misc.obj
 0002:00002938       ??_C@_0BG@HJKONAJE@weapon_rocketlauncher?$AA@ 2003f938     bg_misc.obj
 0002:00002950       ??_C@_0EG@LFEMOCGK@sound?1weapons?1grenade?1hgrenb1a?4w@ 2003f950     bg_misc.obj
 0002:00002998       ??_C@_0BE@JNFKJHKD@icons?1iconw_grenade?$AA@ 2003f998     bg_misc.obj
 0002:000029ac       ??_C@_0CG@INCGOMDL@models?1weapons2?1grenadel?1grenade@ 2003f9ac     bg_misc.obj
 0002:000029d4       ??_C@_0BH@DGCCJPLM@weapon_grenadelauncher?$AA@ 2003f9d4     bg_misc.obj
 0002:000029ec       ??_C@_0BH@GIACBLNI@icons?1iconw_machinegun?$AA@ 2003f9ec     bg_misc.obj
 0002:00002a04       ??_C@_0CK@BBPFNIFO@models?1weapons2?1machinegun?1machi@ 2003fa04     bg_misc.obj
 0002:00002a30       ??_C@_0BC@HHBNPFPN@weapon_machinegun?$AA@ 2003fa30     bg_misc.obj
 0002:00002a44       ??_C@_0BE@PGLFIIOH@icons?1iconw_shotgun?$AA@ 2003fa44     bg_misc.obj
 0002:00002a58       ??_C@_0CE@CJGCHKCN@models?1weapons2?1shotgun?1shotgun?4@ 2003fa58     bg_misc.obj
 0002:00002a7c       ??_C@_0P@ILAKNOAG@weapon_shotgun?$AA@ 2003fa7c     bg_misc.obj
 0002:00002a8c       ??_C@_0BF@PMEPIOCM@icons?1iconw_gauntlet?$AA@ 2003fa8c     bg_misc.obj
 0002:00002aa4       ??_C@_0CG@PFPPJBAC@models?1weapons2?1gauntlet?1gauntle@ 2003faa4     bg_misc.obj
 0002:00002acc       ??_C@_0BG@BBKFHONL@sound?1misc?1w_pkup?4wav?$AA@ 2003facc     bg_misc.obj
 0002:00002ae4       ??_C@_0BA@CLDPODJE@weapon_gauntlet?$AA@ 2003fae4     bg_misc.obj
 0002:00002af4       ??_C@_0M@IOJDMPNO@Mega?5Health?$AA@ 2003faf4     bg_misc.obj
 0002:00002b00       ??_C@_0BB@EGPGIMOM@icons?1iconh_mega?$AA@ 2003fb00     bg_misc.obj
 0002:00002b14       ??_C@_0CH@NEGHBKPB@models?1powerups?1health?1mega_sphe@ 2003fb14     bg_misc.obj
 0002:00002b3c       ??_C@_0CG@PDJMMGME@models?1powerups?1health?1mega_cros@ 2003fb3c     bg_misc.obj
 0002:00002b64       ??_C@_0BJ@FGLGEHNG@sound?1items?1m_health?4wav?$AA@ 2003fb64     bg_misc.obj
 0002:00002b80       ??_C@_0BB@PBGAONGH@item_health_mega?$AA@ 2003fb80     bg_misc.obj
 0002:00002b94       ??_C@_09EBELOOOD@50?5Health?$AA@ 2003fb94     bg_misc.obj
 0002:00002ba0       ??_C@_0BA@IGNANAGL@icons?1iconh_red?$AA@ 2003fba0     bg_misc.obj
 0002:00002bb0       ??_C@_0CI@CEEMEFNH@models?1powerups?1health?1large_sph@ 2003fbb0     bg_misc.obj
 0002:00002bd8       ??_C@_0CH@NHFAKEFE@models?1powerups?1health?1large_cro@ 2003fbd8     bg_misc.obj
 0002:00002c00       ??_C@_0BJ@ILCAJOFD@sound?1items?1l_health?4wav?$AA@ 2003fc00     bg_misc.obj
 0002:00002c1c       ??_C@_0BC@JGDLKFIO@item_health_large?$AA@ 2003fc1c     bg_misc.obj
 0002:00002c30       ??_C@_09OJAALANF@25?5Health?$AA@ 2003fc30     bg_misc.obj
 0002:00002c3c       ??_C@_0BD@CDBLAHCA@icons?1iconh_yellow?$AA@ 2003fc3c     bg_misc.obj
 0002:00002c50       ??_C@_0CJ@NCCPDHOD@models?1powerups?1health?1medium_sp@ 2003fc50     bg_misc.obj
 0002:00002c7c       ??_C@_0CI@NAEMLIB@models?1powerups?1health?1medium_cr@ 2003fc7c     bg_misc.obj
 0002:00002ca4       ??_C@_0BJ@OLHMCLBI@sound?1items?1n_health?4wav?$AA@ 2003fca4     bg_misc.obj
 0002:00002cc0       ??_C@_0M@KCNAKNNL@item_health?$AA@ 2003fcc0     bg_misc.obj
 0002:00002ccc       ??_C@_08IAIFJOAI@5?5Health?$AA@ 2003fccc     bg_misc.obj
 0002:00002cd8       ??_C@_0BC@IMNPBGFF@icons?1iconh_green?$AA@ 2003fcd8     bg_misc.obj
 0002:00002cec       ??_C@_0CI@MPAPPIIE@models?1powerups?1health?1small_sph@ 2003fcec     bg_misc.obj
 0002:00002d14       ??_C@_0CH@JKNLMIJB@models?1powerups?1health?1small_cro@ 2003fd14     bg_misc.obj
 0002:00002d3c       ??_C@_0BJ@BIFHONLM@sound?1items?1s_health?4wav?$AA@ 2003fd3c     bg_misc.obj
 0002:00002d58       ??_C@_0BC@DOHAFEBI@item_health_small?$AA@ 2003fd58     bg_misc.obj
 0002:00002d6c       ??_C@_0BA@CEJNPBJG@icons?1iconr_red?$AA@ 2003fd6c     bg_misc.obj
 0002:00002d7c       ??_C@_0CE@EGJFDJJK@models?1powerups?1armor?1armor_red?4@ 2003fd7c     bg_misc.obj
 0002:00002da0       ??_C@_0BA@EKKMHIH@item_armor_body?$AA@ 2003fda0     bg_misc.obj
 0002:00002db0       ??_C@_0BD@BKPFMPMP@icons?1iconr_yellow?$AA@ 2003fdb0     bg_misc.obj
 0002:00002dc4       ??_C@_0CE@PHKMKHKB@models?1powerups?1armor?1armor_yel?4@ 2003fdc4     bg_misc.obj
 0002:00002de8       ??_C@_0BI@KNMPECGK@sound?1misc?1ar2_pkup?4wav?$AA@ 2003fde8     bg_misc.obj
 0002:00002e00       ??_C@_0BC@FPPLPJIL@item_armor_combat?$AA@ 2003fe00     bg_misc.obj
 0002:00002e14       ??_C@_0M@PJIPIDNH@Armor?5Shard?$AA@ 2003fe14     bg_misc.obj
 0002:00002e20       ??_C@_0BC@LPFHDODA@icons?1iconr_shard?$AA@ 2003fe20     bg_misc.obj
 0002:00002e34       ??_C@_0CH@NEKDLKN@models?1powerups?1armor?1shard_sphe@ 2003fe34     bg_misc.obj
 0002:00002e5c       ??_C@_0CA@NOFOCCIK@models?1powerups?1armor?1shard?4md3?$AA@ 2003fe5c     bg_misc.obj
 0002:00002e7c       ??_C@_0BI@DECNCEGL@sound?1misc?1ar1_pkup?4wav?$AA@ 2003fe7c     bg_misc.obj
 0002:00002e94       ??_C@_0BB@DDGIAABK@item_armor_shard?$AA@ 2003fe94     bg_misc.obj
 0002:00002ea8       ??_C@_0CB@DEACFJO@Couldn?8t?5find?5item?5for?5weapon?5?$CFi@ 2003fea8     bg_misc.obj
 0002:00002ecc       ??_C@_0BM@NECGLAIF@BG_CanItemBeGrabbed?3?5IT_BAD?$AA@ 2003fecc     bg_misc.obj
 0002:00002ee8       ??_C@_0CI@MFONMA@BG_CanItemBeGrabbed?3?5index?5out?5o@ 2003fee8     bg_misc.obj
 0002:00002f10       ??_C@_0CK@DNBGNAED@BG_EvaluateTrajectory?3?5unknown?5t@ 2003ff10     bg_misc.obj
 0002:00002f40       __real@4079000000000000    2003ff40     bg_misc.obj
 0002:00002f48       __real@40c90fdb            2003ff48     bg_misc.obj
 0002:00002f4c       ??_C@_0CP@MCFPOIMF@BG_EvaluateTrajectoryDelta?3?5unkn@ 2003ff4c     bg_misc.obj
 0002:00002f7c       __real@42340000            2003ff7c     bg_misc.obj
 0002:00002f80       __real@c2100000            2003ff80     bg_misc.obj
 0002:00002f84       __real@42100000            2003ff84     bg_misc.obj
 0002:00002f88       __real@c2480000            2003ff88     bg_misc.obj
 0002:00002f8c       __real@42300000            2003ff8c     bg_misc.obj
 0002:00002f90       __real@405fc00000000000    2003ff90     bg_pmove.obj
 0002:00002f98       __real@41f00000            2003ff98     bg_pmove.obj
 0002:00002f9c       __real@3f7fbe87            2003ff9c     bg_pmove.obj
 0002:00002fa0       __real@3f8020c5            2003ffa0     bg_pmove.obj
 0002:00002fa4       __real@c1800000            2003ffa4     bg_pmove.obj
 0002:00002fa8       __real@3fd5555555555555    2003ffa8     bg_pmove.obj
 0002:00002fb0       __real@40e00000            2003ffb0     bg_pmove.obj
 0002:00002fb8       __real@3f1a36e2eb1c432d    2003ffb8     bg_pmove.obj
 0002:00002fc0       __real@3f000000            2003ffc0     bg_pmove.obj
 0002:00002fc4       ??_C@_0N@KJCNHCBK@?$CFi?3allsolid?6?$AA@ 2003ffc4     bg_pmove.obj
 0002:00002fd4       ??_C@_08EOGJDHPF@?$CFi?3lift?6?$AA@ 2003ffd4     bg_pmove.obj
 0002:00002fe0       __real@c3480000            2003ffe0     bg_pmove.obj
 0002:00002fe4       ??_C@_08KACHPCJN@?$CFi?3Land?6?$AA@ 2003ffe4     bg_pmove.obj
 0002:00002ff0       ??_C@_09OPMLNNOA@?$CFi?3steep?6?$AA@ 2003fff0     bg_pmove.obj
 0002:00002ffc       ??_C@_0M@CKJFDFGH@?$CFi?3kickoff?6?$AA@ 2003fffc     bg_pmove.obj
 0002:00003008       __real@3e99999a            20040008     bg_pmove.obj
 0002:00003010       __real@3fe89d89d89d89d8    20040010     bg_pmove.obj
 0002:00003018       ??_C@_0M@CDHDENEF@?$CFi?3stepped?6?$AA@ 20040018     bg_slidemove.obj
 0002:00003024       __real@41300000            20040024     bg_slidemove.obj
 0002:00003028       ??_C@_0BE@FLPNHHPN@?$CFi?3bend?5can?8t?5step?6?$AA@ 20040028     bg_slidemove.obj
 0002:0000303c       __real@41900000            2004003c     bg_slidemove.obj
 0002:00003040       __real@3fe6c16c16c16c17    20040040     g_active.obj
 0002:00003048       __real@437f0000            20040048     g_active.obj
 0002:0000304c       ??_C@_0BH@CIEIFFOL@sound?1player?1gurp2?4wav?$AA@ 2004004c     g_active.obj
 0002:00003064       ??_C@_0BH@KONMCHEF@sound?1player?1gurp1?4wav?$AA@ 20040064     g_active.obj
 0002:0000307c       ??_C@_0L@FMIBJCKG@?$CKdrown?4wav?$AA@ 2004007c     g_active.obj
 0002:00003088       ??_C@_0CJ@OOBJBOCC@cp?5?$CCTen?5seconds?5until?5inactivity@ 20040088     g_active.obj
 0002:000030b4       ??_C@_0BK@CMFHJBAI@Dropped?5due?5to?5inactivity?$AA@ 200400b4     g_active.obj
 0002:000030d0       __real@3ff199999999999a    200400d0     g_active.obj
 0002:000030d8       __real@3ff4cccccccccccd    200400d8     g_active.obj
 0002:000030e0       ??_C@_0L@JLBEBBAD@pmove_msec?$AA@ 200400e0     g_active.obj
 0002:000030ec       ??_C@_02NCPIBIBE@33?$AA@   200400ec     g_active.obj
 0002:000030f0       ??_C@_01KJLJFBPL@8?$AA@    200400f0     g_active.obj
 0002:000030f4       ??_C@_09HCJPKLNL@?5?$CFi?5?$CFi?5?$CFi?$AA@ 200400f4     g_arenas.obj
 0002:00003100       ??_C@_0CB@CLLCPLDB@postgame?5?$CFi?5?$CFi?5?$CFi?5?$CFi?5?$CFi?5?$CFi?5?$CFi?5?$CFi@ 20040100     g_arenas.obj
 0002:00003124       ??_C@_0BL@HAGGIKPH@postgame?5?$CFi?5?$CFi?50?50?50?50?50?50?$AA@ 20040124     g_arenas.obj
 0002:00003140       ??_C@_0BL@MJMDOODN@?$FO1ERROR?3?5out?5of?5gentities?6?$AA@ 20040140     g_arenas.obj
 0002:0000315c       ??_C@_0N@NHMKEGEN@g_podiumDrop?$AA@ 2004015c     g_arenas.obj
 0002:0000316c       ??_C@_0N@CBICAJMD@g_podiumDist?$AA@ 2004016c     g_arenas.obj
 0002:0000317c       ??_C@_06NPKMJLHA@podium?$AA@ 2004017c     g_arenas.obj
 0002:00003184       ??_C@_0CF@MDONDONI@models?1mapobjects?1podium?1podium4@ 20040184     g_arenas.obj
 0002:000031ac       ??_C@_0BE@IKMJLADL@Max?5infos?5exceeded?6?$AA@ 200401ac     g_bot.obj
 0002:000031c0       ??_C@_0BI@BMEIBPEH@Missing?5?$HL?5in?5info?5file?6?$AA@ 200401c0     g_bot.obj
 0002:000031d8       ??_C@_0BN@HAJDHEGK@Unexpected?5end?5of?5info?5file?6?$AA@ 200401d8     g_bot.obj
 0002:000031f8       ??_C@_06CBHGEMFM@?$DMNULL?$DO?$AA@ 200401f8     g_bot.obj
 0002:00003200       ??_C@_01CELHOKLL@?$HN?$AA@ 20040200     g_bot.obj
 0002:00003204       ??_C@_01HCONENDN@?$HL?$AA@ 20040204     g_bot.obj
 0002:00003208       ??_C@_0CO@OKDDPLPD@?$FO1file?5too?5large?3?5?$CFs?5is?5?$CFi?0?5max?5@ 20040208     g_bot.obj
 0002:00003238       ??_C@_0BG@BJEIGKLP@?$FO1file?5not?5found?3?5?$CFs?6?$AA@ 20040238     g_bot.obj
 0002:00003250       ??_C@_03IHCLBPIC@num?$AA@  20040250     g_bot.obj
 0002:00003254       ??_C@_02IKAHHCAI@?$CFi?$AA@ 20040254     g_bot.obj
 0002:00003258       ??_C@_0BC@MIFKOHOA@?$CFi?5arenas?5parsed?6?$AA@ 20040258     g_bot.obj
 0002:0000326c       ??_C@_08IDJEBFOJ@scripts?1?$AA@ 2004026c     g_bot.obj
 0002:00003278       ??_C@_07OMEBBDEO@scripts?$AA@ 20040278     g_bot.obj
 0002:00003280       ??_C@_06IPPMLGON@?4arena?$AA@ 20040280     g_bot.obj
 0002:00003288       ??_C@_0BD@KEINBKFE@scripts?1arenas?4txt?$AA@ 20040288     g_bot.obj
 0002:0000329c       ??_C@_0N@BFDKEKMB@g_arenasFile?$AA@ 2004029c     g_bot.obj
 0002:000032ac       ??_C@_03HBNNNHNM@map?$AA@  200402ac     g_bot.obj
 0002:000032b0       ??_C@_0CD@DFNICLKJ@play?5sound?1player?1announce?1?$CFs?4wa@ 200402b0     g_bot.obj
 0002:000032d4       ??_C@_07DLHCIBDH@default?$AA@ 200402d4     g_bot.obj
 0002:000032dc       ??_C@_0BE@HKGNLKGC@addbot?5?$CFs?5?$CFf?5?$CFs?5?$CFi?6?$AA@ 200402dc     g_bot.obj
 0002:000032f0       ??_C@_04MEMAJGDJ@name?$AA@ 200402f0     g_bot.obj
 0002:000032f8       ??_C@_08CKHMKINC@kick?5?$CFs?6?$AA@ 200402f8     g_bot.obj
 0002:00003304       ??_C@_0BJ@JBHOCGJI@?$FO3Unable?5to?5delay?5spawn?6?$AA@ 20040304     g_bot.obj
 0002:00003320       ??_C@_0BI@KOJDMFEB@BotAISetupClient?5failed?$AA@ 20040320     g_bot.obj
 0002:00003338       ??_C@_04KADBPNCB@team?$AA@ 20040338     g_bot.obj
 0002:00003340       ??_C@_05ODMCMJAJ@skill?$AA@ 20040340     g_bot.obj
 0002:00003348       ??_C@_0O@HKBPPLKD@characterfile?$AA@ 20040348     g_bot.obj
 0002:00003358       ??_C@_0BJ@GPLOPMDF@?$CF?916s?5?$CF?916s?5?$CF?920s?5?$CF?920s?6?$AA@ 20040358     g_bot.obj
 0002:00003374       ??_C@_0BB@OCLCLNLB@bots?1default_c?4c?$AA@ 20040374     g_bot.obj
 0002:00003388       ??_C@_06GJLCKOIA@aifile?$AA@ 20040388     g_bot.obj
 0002:00003390       ??_C@_0O@CLCMCGPB@visor?1default?$AA@ 20040390     g_bot.obj
 0002:000033a0       ??_C@_07PNOKIGNH@funname?$AA@ 200403a0     g_bot.obj
 0002:000033a8       ??_C@_0O@PCBPGDGA@UnnamedPlayer?$AA@ 200403a8     g_bot.obj
 0002:000033b8       ??_C@_0EB@OHFELCCO@?$FO1name?5?5?5?5?5?5?5?5?5?5?5?5?5model?5?5?5?5?5?5?5?5@ 200403b8     g_bot.obj
 0002:000033fc       ??_C@_0BG@FOPKNLEB@addbot?5?$CFs?5?$CFf?5free?5?$CFi?6?$AA@ 200403fc     g_bot.obj
 0002:00003414       ??_C@_01BMBHCPLG@5?$AA@    20040414     g_bot.obj
 0002:00003418       ??_C@_0BA@KCNHFFOD@?$CFi?5bots?5parsed?6?$AA@ 20040418     g_bot.obj
 0002:00003428       ??_C@_04NONLJGOA@?4bot?$AA@ 20040428     g_bot.obj
 0002:00003430       ??_C@_0BB@LMBKKAOC@scripts?1bots?4txt?$AA@ 20040430     g_bot.obj
 0002:00003444       ??_C@_0L@IDJNDIMJ@g_botsFile?$AA@ 20040444     g_bot.obj
 0002:00003450       ??_C@_0L@BKCPIMBP@bot_enable?$AA@ 20040450     g_bot.obj
 0002:0000345c       ??_C@_04OOIACBCD@bots?$AA@ 2004045c     g_bot.obj
 0002:00003464       ??_C@_08FACPJMEJ@training?$AA@ 20040464     g_bot.obj
 0002:00003470       ??_C@_07BELCMIIP@special?$AA@ 20040470     g_bot.obj
 0002:00003478       ??_C@_09KPHKOKCC@timelimit?$AA@ 20040478     g_bot.obj
 0002:00003484       ??_C@_09GCIEGDDN@fraglimit?$AA@ 20040484     g_bot.obj
 0002:00003490       ??_C@_0P@IGNPDGBD@bot_minplayers?$AA@ 20040490     g_bot.obj
 0002:000034a0       ??_C@_05CEDINIPN@?$CF5?42f?$AA@ 200404a0     g_bot.obj
 0002:000034a8       ??_C@_0FB@BKCBGING@?$FO1Start?5server?5with?5more?5?8open?8?5@ 200404a8     g_bot.obj
 0002:000034fc       ??_C@_0DE@MKFCEMGM@?$FO1Unable?5to?5add?5bot?4?5?5All?5player@ 200404fc     g_bot.obj
 0002:00003530       ??_C@_0CG@GFPKDAFH@?$FO1Error?3?5bot?5has?5no?5aifile?5speci@ 20040530     g_bot.obj
 0002:00003558       ??_C@_06KEONFOCA@color2?$AA@ 20040558     g_bot.obj
 0002:00003560       ??_C@_01FAMBOPH@4?$AA@     20040560     g_bot.obj
 0002:00003564       ??_C@_06IPMAANOD@color1?$AA@ 20040564     g_bot.obj
 0002:0000356c       ??_C@_04ICKCIGNO@male?$AA@ 2004056c     g_bot.obj
 0002:00003574       ??_C@_06LFOIHHME@gender?$AA@ 20040574     g_bot.obj
 0002:0000357c       ??_C@_0P@JMIBMNM@team_headmodel?$AA@ 2004057c     g_bot.obj
 0002:0000358c       ??_C@_09DHBBGOBJ@headmodel?$AA@ 2004058c     g_bot.obj
 0002:00003598       ??_C@_0L@KEDOKIKJ@team_model?$AA@ 20040598     g_bot.obj
 0002:000035a4       ??_C@_02PEECMOAB@90?$AA@   200405a4     g_bot.obj
 0002:000035a8       ??_C@_02PONMODAL@70?$AA@   200405a8     g_bot.obj
 0002:000035ac       ??_C@_08HBHLIHAM@handicap?$AA@ 200405ac     g_bot.obj
 0002:000035b8       ??_C@_02PNFIDHGF@50?$AA@   200405b8     g_bot.obj
 0002:000035bc       ??_C@_05NBLIHODN@?$CF1?42f?$AA@ 200405bc     g_bot.obj
 0002:000035c4       ??_C@_05DGPADKBM@snaps?$AA@ 200405c4     g_bot.obj
 0002:000035cc       ??_C@_04HCCHHEEF@rate?$AA@ 200405cc     g_bot.obj
 0002:000035d4       ??_C@_05GFEIOEMO@25000?$AA@ 200405d4     g_bot.obj
 0002:000035dc       ??_C@_0BP@NGBNIFAK@?$FO1Error?3?5Bot?5?8?$CFs?8?5not?5defined?6?$AA@ 200405dc     g_bot.obj
 0002:000035fc       ??_C@_0N@GEFCGCPK@loaddefered?6?$AA@ 200405fc     g_bot.obj
 0002:0000360c       ??_C@_0L@FBHMLJNH@cl_running?$AA@ 2004060c     g_bot.obj
 0002:00003618       ??_C@_0ED@LBGLLNI@Usage?3?5Addbot?5?$DMbotname?$DO?5?$FLskill?51@ 20040618     g_bot.obj
 0002:0000365c       ??_C@_08MDEJHCAF@nohumans?$AA@ 2004065c     g_client.obj
 0002:00003668       ??_C@_06JHOFIDHH@nobots?$AA@ 20040668     g_client.obj
 0002:00003670       ??_C@_0BH@IGAFCIL@info_player_deathmatch?$AA@ 20040670     g_client.obj
 0002:00003688       __real@41100000            20040688     g_client.obj
 0002:0000368c       ??_C@_0BM@DGHFFJBI@Couldn?8t?5find?5a?5spawn?5point?$AA@ 2004068c     g_client.obj
 0002:000036a8       ??_C@_07ILHJIGAO@bodyque?$AA@ 200406a8     g_client.obj
 0002:000036b0       ??_C@_0BO@IFHBFKHP@ClientUserinfoChanged?3?5?$CFi?5?$CFs?6?$AA@ 200406b0     g_client.obj
 0002:000036d0       ??_C@_0GA@GJMCBBDN@n?2?$CFs?2t?2?$CFi?2model?2?$CFs?2hmodel?2?$CFs?2g_r@ 200406d0     g_client.obj
 0002:00003730       ??_C@_0EO@IELCCCFM@n?2?$CFs?2t?2?$CFi?2model?2?$CFs?2hmodel?2?$CFs?2c1?2@ 20040730     g_client.obj
 0002:00003780       ??_C@_0L@CPNMJIBN@g_blueteam?$AA@ 20040780     g_client.obj
 0002:0000378c       ??_C@_09LPNHELAH@g_redteam?$AA@ 2004078c     g_client.obj
 0002:00003798       ??_C@_0M@IKKMOBIP@teamoverlay?$AA@ 20040798     g_client.obj
 0002:000037a4       ??_C@_01OJONOECF@b?$AA@    200407a4     g_client.obj
 0002:000037a8       ??_C@_01KDCPPGHE@r?$AA@    200407a8     g_client.obj
 0002:000037ac       ??_C@_0BM@IJFFLPEN@print?5?$CC?$CFs?$FO7?5renamed?5to?5?$CFs?6?$CC?$AA@ 200407ac     g_client.obj
 0002:000037c8       ??_C@_0L@PGGJLCHO@scoreboard?$AA@ 200407c8     g_client.obj
 0002:000037d4       ??_C@_0BA@PKAEEJJB@cg_predictItems?$AA@ 200407d4     g_client.obj
 0002:000037e4       ??_C@_09IPAEKDAI@localhost?$AA@ 200407e4     g_client.obj
 0002:000037f0       ??_C@_02GIIHKPLE@ip?$AA@   200407f0     g_client.obj
 0002:000037f4       ??_C@_0O@JBDOHEEF@?2name?2badinfo?$AA@ 200407f4     g_client.obj
 0002:00003804       ??_C@_0BI@LLOHFCPM@print?5?$CC?$CFs?$FO7?5connected?6?$CC?$AA@ 20040804     g_client.obj
 0002:0000381c       ??_C@_0BD@LEMBFDEN@ClientConnect?3?5?$CFi?6?$AA@ 2004081c     g_client.obj
 0002:00003830       ??_C@_0BB@KINAMDJK@BotConnectfailed?$AA@ 20040830     g_client.obj
 0002:00003844       ??_C@_0BB@GKDCDICO@Invalid?5password?$AA@ 20040844     g_client.obj
 0002:00003858       ??_C@_04CGFJFPFD@none?$AA@ 20040858     g_client.obj
 0002:00003860       ??_C@_08NLHBPEGP@password?$AA@ 20040860     g_client.obj
 0002:0000386c       ??_C@_0CB@BAJJGAM@You?5are?5banned?5from?5this?5server?4@ 2004086c     g_client.obj
 0002:00003890       ??_C@_06BALNJMNP@player?$AA@ 20040890     g_client.obj
 0002:00003898       ??_C@_0N@GGGDBMDO@disconnected?$AA@ 20040898     g_client.obj
 0002:000038a8       ??_C@_0BG@PJMKPFGA@ClientDisconnect?3?5?$CFi?6?$AA@ 200408a8     g_client.obj
 0002:000038c0       ??_C@_0BB@JCCEPCGJ@ClientBegin?3?5?$CFi?6?$AA@ 200408c0     g_client.obj
 0002:000038d4       ??_C@_0BP@PGPGIDAG@print?5?$CC?$CFs?$FO7?5entered?5the?5game?6?$CC?$AA@ 200408d4     g_client.obj
 0002:000038f4       ??_C@_09OKMOBHEE@Harvester?$AA@ 200408f4     g_cmds.obj
 0002:00003900       ??_C@_08JKIFACLF@Overload?$AA@ 20040900     g_cmds.obj
 0002:0000390c       ??_C@_0N@FCMBHKKN@One?5Flag?5CTF?$AA@ 2004090c     g_cmds.obj
 0002:0000391c       ??_C@_0BB@OOIHNFAG@Capture?5the?5Flag?$AA@ 2004091c     g_cmds.obj
 0002:00003930       ??_C@_0BA@KHHNIIJE@Team?5Deathmatch?$AA@ 20040930     g_cmds.obj
 0002:00003940       ??_C@_0O@NNAOEDOE@Single?5Player?$AA@ 20040940     g_cmds.obj
 0002:00003950       ??_C@_0L@FENDKKGN@Tournament?$AA@ 20040950     g_cmds.obj
 0002:0000395c       ??_C@_0N@PCEMCJC@Free?5For?5All?$AA@ 2004095c     g_cmds.obj
 0002:0000396c       ??_C@_06MHOMHIDM@report?$AA@ 2004096c     g_cmds.obj
 0002:00003974       ??_C@_0BD@JFEBCONJ@search?5and?5destroy?$AA@ 20040974     g_cmds.obj
 0002:00003988       ??_C@_0P@BDHIOPIB@guard?5location?$AA@ 20040988     g_cmds.obj
 0002:00003998       ??_C@_08NJPHEENP@cover?5me?$AA@ 20040998     g_cmds.obj
 0002:000039a4       ??_C@_09NKPGKNPA@come?5here?$AA@ 200409a4     g_cmds.obj
 0002:000039b0       ??_C@_0BD@BGOJJIFC@hold?5this?5position?$AA@ 200409b0     g_cmds.obj
 0002:000039c4       ??_C@_0BD@BEPMJBOM@hold?5your?5position?$AA@ 200409c4     g_cmds.obj
 0002:000039d8       ??_C@_0BC@BADCIGBJ@scores?5?$CFi?5?$CFi?5?$CFi?$CFs?$AA@ 200409d8     g_cmds.obj
 0002:000039ec       ??_C@_0CL@EAFNPFGA@?5?$CFi?5?$CFi?5?$CFi?5?$CFi?5?$CFi?5?$CFi?5?$CFi?5?$CFi?5?$CFi?5?$CFi?5?$CF@ 200409ec     g_cmds.obj
 0002:00003a18       ??_C@_0DA@KHFNLLBI@print?5?$CCYou?5must?5be?5alive?5to?5use?5@ 20040a18     g_cmds.obj
 0002:00003a48       ??_C@_0DA@DLJNDFCJ@print?5?$CCCheats?5are?5not?5enabled?5on@ 20040a48     g_cmds.obj
 0002:00003a78       ??_C@_0CG@OFMIDLCG@print?5?$CCUser?5?$CFs?5is?5not?5on?5the?5ser@ 20040a78     g_cmds.obj
 0002:00003aa0       ??_C@_0BN@FGLBNIJH@print?5?$CCBad?5client?5slot?3?5?$CFi?6?$CC?$AA@ 20040aa0     g_cmds.obj
 0002:00003ac0       ??_C@_0CB@IOMDOEKP@print?5?$CCClient?5?$CFi?5is?5not?5active?6?$CC@ 20040ac0     g_cmds.obj
 0002:00003ae4       ??_C@_06CHFMFANC@assist?$AA@ 20040ae4     g_cmds.obj
 0002:00003aec       ??_C@_0O@DCIHIELO@gauntletaward?$AA@ 20040aec     g_cmds.obj
 0002:00003afc       ??_C@_0L@GBLMIJON@impressive?$AA@ 20040afc     g_cmds.obj
 0002:00003b08       ??_C@_09MBDMPFOO@excellent?$AA@ 20040b08     g_cmds.obj
 0002:00003b14       ??_C@_05JJEJIJLL@armor?$AA@ 20040b14     g_cmds.obj
 0002:00003b1c       ??_C@_04PGKJFGNK@ammo?$AA@ 20040b1c     g_cmds.obj
 0002:00003b24       ??_C@_07PKKCMMCH@weapons?$AA@ 20040b24     g_cmds.obj
 0002:00003b2c       ??_C@_03NFKEKGGK@all?$AA@  20040b2c     g_cmds.obj
 0002:00003b30       ??_C@_0L@GPCEIOHM@print?5?$CC?$CFs?$CC?$AA@ 20040b30     g_cmds.obj
 0002:00003b3c       ??_C@_0M@MCLKHHDH@godmode?5ON?6?$AA@ 20040b3c     g_cmds.obj
 0002:00003b48       ??_C@_0N@POKEKLLJ@godmode?5OFF?6?$AA@ 20040b48     g_cmds.obj
 0002:00003b58       ??_C@_0N@OBJNJDJO@notarget?5ON?6?$AA@ 20040b58     g_cmds.obj
 0002:00003b68       ??_C@_0O@FBINJHBB@notarget?5OFF?6?$AA@ 20040b68     g_cmds.obj
 0002:00003b78       ??_C@_0L@MDMNIPJN@noclip?5ON?6?$AA@ 20040b78     g_cmds.obj
 0002:00003b84       ??_C@_0M@MIKGJGLH@noclip?5OFF?6?$AA@ 20040b84     g_cmds.obj
 0002:00003b90       ??_C@_0CP@EMMMGMNN@print?5?$CCMust?5be?5in?5g_gametype?50?5f@ 20040b90     g_cmds.obj
 0002:00003bc0       ??_C@_0BO@HCBBHHLG@cp?5?$CC?$CFs?$FO7?5joined?5the?5battle?4?6?$CC?$AA@ 20040bc0     g_cmds.obj
 0002:00003be0       ??_C@_0CC@CKOABLEC@cp?5?$CC?$CFs?$FO7?5joined?5the?5spectators?4?6@ 20040be0     g_cmds.obj
 0002:00003c04       ??_C@_0CB@MALDLCDE@cp?5?$CC?$CFs?$FO7?5joined?5the?5blue?5team?4?6?$CC@ 20040c04     g_cmds.obj
 0002:00003c28       ??_C@_0CA@FCJONFGI@cp?5?$CC?$CFs?$FO7?5joined?5the?5red?5team?4?6?$CC?$AA@ 20040c28     g_cmds.obj
 0002:00003c48       ??_C@_0CG@BNBAGBGM@cp?5?$CCBlue?5team?5has?5too?5many?5playe@ 20040c48     g_cmds.obj
 0002:00003c70       ??_C@_0CF@OMMGDNAE@cp?5?$CCRed?5team?5has?5too?5many?5player@ 20040c70     g_cmds.obj
 0002:00003c98       ??_C@_01LKDEMHDF@s?$AA@    20040c98     g_cmds.obj
 0002:00003c9c       ??_C@_09FNMDCDOI@spectator?$AA@ 20040c9c     g_cmds.obj
 0002:00003ca8       ??_C@_07NNICNDK@follow2?$AA@ 20040ca8     g_cmds.obj
 0002:00003cb0       ??_C@_07CGPFHOPJ@follow1?$AA@ 20040cb0     g_cmds.obj
 0002:00003cb8       ??_C@_05DBKDOICH@score?$AA@ 20040cb8     g_cmds.obj
 0002:00003cc0       ??_C@_0DM@NEIAOCHE@print?5?$CCMay?5not?5switch?5teams?5more@ 20040cc0     g_cmds.obj
 0002:00003cfc       ??_C@_0BI@PDLENAMN@print?5?$CCSpectator?5team?6?$CC?$AA@ 20040cfc     g_cmds.obj
 0002:00003d14       ??_C@_0BD@COAKLBJE@print?5?$CCFree?5team?6?$CC?$AA@ 20040d14     g_cmds.obj
 0002:00003d28       ??_C@_0BC@HGAENHGG@print?5?$CCRed?5team?6?$CC?$AA@ 20040d28     g_cmds.obj
 0002:00003d3c       ??_C@_0BD@PGCCOEMO@print?5?$CCBlue?5team?6?$CC?$AA@ 20040d3c     g_cmds.obj
 0002:00003d50       ??_C@_0BO@KJIMFOBJ@Cmd_FollowCycle_f?3?5bad?5dir?5?$CFi?$AA@ 20040d50     g_cmds.obj
 0002:00003d70       ??_C@_0O@CCPEDGNK@?$CFs?5?$CC?$CFs?$CFc?$CFc?$CFs?$CC?$AA@ 20040d70     g_cmds.obj
 0002:00003d80       ??_C@_05JMJKDBEJ@?$CFs?$CFs?6?$AA@ 20040d80     g_cmds.obj
 0002:00003d88       ??_C@_0O@FGLMEIPO@?$BJ?$CI?$CFs?$CFc?$CFc?$BJ?$CJ?$BJ?3?5?$AA@ 20040d88     g_cmds.obj
 0002:00003d98       ??_C@_0BD@LHDLGCNL@?$BJ?$CI?$CFs?$CFc?$CFc?$BJ?$CJ?5?$CI?$CFs?$CJ?$BJ?3?5?$AA@ 20040d98     g_cmds.obj
 0002:00003dac       ??_C@_0BB@OADDLILN@sayteam?3?5?$CFs?3?5?$CFs?6?$AA@ 20040dac     g_cmds.obj
 0002:00003dc0       ??_C@_0O@FNNABOLL@?$BJ?$FL?$CFs?$CFc?$CFc?$BJ?$FN?$BJ?3?5?$AA@ 20040dc0     g_cmds.obj
 0002:00003dd0       ??_C@_0BD@GLHHAOBD@?$BJ?$FL?$CFs?$CFc?$CFc?$BJ?$FN?5?$CI?$CFs?$CJ?$BJ?3?5?$AA@ 20040dd0     g_cmds.obj
 0002:00003de4       ??_C@_09GPHNFPKO@?$CFs?$CFc?$CFc?$BJ?3?5?$AA@ 20040de4     g_cmds.obj
 0002:00003df0       ??_C@_0N@PIPLJLA@say?3?5?$CFs?3?5?$CFs?6?$AA@ 20040df0     g_cmds.obj
 0002:00003e00       ??_C@_0BE@DNAOGBCN@tell?3?5?$CFs?5to?5?$CFs?3?5?$CFs?6?$AA@ 20040e00     g_cmds.obj
 0002:00003e14       ??_C@_0P@GLNDPPNN@?$CFs?5?$CFd?5?$CFd?5?$CFd?5?$CFs?$AA@ 20040e14     g_cmds.obj
 0002:00003e24       ??_C@_05LBAAHPBE@vchat?$AA@ 20040e24     g_cmds.obj
 0002:00003e2c       ??_C@_05BLGJOHFB@vtell?$AA@ 20040e2c     g_cmds.obj
 0002:00003e34       ??_C@_06FPNOEFND@vtchat?$AA@ 20040e34     g_cmds.obj
 0002:00003e3c       ??_C@_0O@PGEGBHPB@voice?3?5?$CFs?5?$CFs?6?$AA@ 20040e3c     g_cmds.obj
 0002:00003e4c       ??_C@_0BF@KNCPEACI@vtell?3?5?$CFs?5to?5?$CFs?3?5?$CFs?6?$AA@ 20040e4c     g_cmds.obj
 0002:00003e64       ??_C@_06GEFAPDPP@praise?$AA@ 20040e64     g_cmds.obj
 0002:00003e6c       ??_C@_0M@MIDAEIOB@print?5?$CC?$CFs?6?$CC?$AA@ 20040e6c     g_cmds.obj
 0002:00003e78       ??_C@_0KJ@BAKDCPAJ@print?5?$CCVote?5commands?5are?3?5map_re@ 20040e78     g_cmds.obj
 0002:00003f24       ??_C@_0BO@PMPHENKD@print?5?$CCInvalid?5vote?5string?4?6?$CC?$AA@ 20040f24     g_cmds.obj
 0002:00003f44       ??_C@_0BL@LDCKNKB@print?5?$CC?$CFs?5called?5a?5vote?4?6?$CC?$AA@ 20040f44     g_cmds.obj
 0002:00003f60       ??_C@_07CMIPDAGF@?$CFs?5?$CC?$CFs?$CC?$AA@ 20040f60     g_cmds.obj
 0002:00003f68       ??_C@_0N@NPFCFAAA@vstr?5nextmap?$AA@ 20040f68     g_cmds.obj
 0002:00003f78       ??_C@_0BK@IOHPLFMM@print?5?$CCnextmap?5not?5set?4?6?$CC?$AA@ 20040f78     g_cmds.obj
 0002:00003f94       ??_C@_0BI@EHIPCLJD@?$CFs?5?$CFs?$DL?5set?5nextmap?5?$CC?$CFs?$CC?$AA@ 20040f94     g_cmds.obj
 0002:00003fac       ??_C@_0BL@HOKFFIC@print?5?$CCInvalid?5gametype?4?6?$CC?$AA@ 20040fac     g_cmds.obj
 0002:00003fc8       ??_C@_05DNIIFBMG@?$CFs?5?$CFs?$AA@ 20040fc8     g_cmds.obj
 0002:00003fd0       ??_C@_05DIALNFFA@?$CFs?5?$CFd?$AA@ 20040fd0     g_cmds.obj
 0002:00003fd8       ??_C@_03OFAPEBGM@?$CFs?6?$AA@ 20040fd8     g_cmds.obj
 0002:00003fdc       ??_C@_0L@LPENDGCI@g_doWarmup?$AA@ 20040fdc     g_cmds.obj
 0002:00003fe8       ??_C@_0L@NBDAICFL@clientkick?$AA@ 20040fe8     g_cmds.obj
 0002:00003ff4       ??_C@_04FNIJDBCC@kick?$AA@ 20040ff4     g_cmds.obj
 0002:00003ffc       ??_C@_07MCHHMPMB@nextmap?$AA@ 20040ffc     g_cmds.obj
 0002:00004004       ??_C@_0M@NBIMEKNE@map_restart?$AA@ 20041004     g_cmds.obj
 0002:00004010       ??_C@_0DC@KBNBHNDJ@print?5?$CCNot?5allowed?5to?5call?5a?5vot@ 20041010     g_cmds.obj
 0002:00004044       ??_C@_0DG@PHEGLJKA@print?5?$CCYou?5have?5called?5the?5maxim@ 20041044     g_cmds.obj
 0002:0000407c       ??_C@_0CI@IOOGHLKJ@print?5?$CCA?5vote?5is?5already?5in?5prog@ 2004107c     g_cmds.obj
 0002:000040a4       ??_C@_0CC@MKEOLBNH@print?5?$CCVoting?5not?5allowed?5here?4?6@ 200410a4     g_cmds.obj
 0002:000040c8       ??_C@_0BE@KBOHCPHM@print?5?$CCVote?5cast?4?6?$CC?$AA@ 200410c8     g_cmds.obj
 0002:000040dc       ??_C@_0CL@KIACKMGK@print?5?$CCNot?5allowed?5to?5vote?5as?5sp@ 200410dc     g_cmds.obj
 0002:00004108       ??_C@_0BM@JAOFDBMB@print?5?$CCVote?5already?5cast?4?6?$CC?$AA@ 20041108     g_cmds.obj
 0002:00004124       ??_C@_0BO@JJMMHDFC@print?5?$CCNo?5vote?5in?5progress?4?6?$CC?$AA@ 20041124     g_cmds.obj
 0002:00004144       ??_C@_0DC@JMKMFJGE@print?5?$CCTeam?5vote?5commands?5are?3?5l@ 20041144     g_cmds.obj
 0002:00004178       ??_C@_0DA@BDICJJF@print?5?$CC?$CFs?5is?5not?5a?5valid?5player?5@ 20041178     g_cmds.obj
 0002:000041a8       ??_C@_0CA@ENAIANHJ@print?5?$CC?$CFs?5called?5a?5team?5vote?4?6?$CC?$AA@ 200411a8     g_cmds.obj
 0002:000041c8       ??_C@_06DFLPLEOP@leader?$AA@ 200411c8     g_cmds.obj
 0002:000041d0       ??_C@_0DL@IFNKHCNG@print?5?$CCYou?5have?5called?5the?5maxim@ 200411d0     g_cmds.obj
 0002:0000420c       ??_C@_0CN@INNKCADJ@print?5?$CCA?5team?5vote?5is?5already?5in@ 2004120c     g_cmds.obj
 0002:0000423c       ??_C@_0BJ@DCKHGAB@print?5?$CCTeam?5vote?5cast?4?6?$CC?$AA@ 2004123c     g_cmds.obj
 0002:00004258       ??_C@_0CB@LGGMNIHI@print?5?$CCTeam?5vote?5already?5cast?4?6?$CC@ 20041258     g_cmds.obj
 0002:0000427c       ??_C@_0CD@BLODMPFK@print?5?$CCNo?5team?5vote?5in?5progress?4@ 2004127c     g_cmds.obj
 0002:000042a0       ??_C@_0CF@GJFHLKOA@print?5?$CCusage?3?5setviewpos?5x?5y?5z?5y@ 200412a0     g_cmds.obj
 0002:000042c8       ??_C@_0BI@FJNBDMBJ@print?5?$CCunknown?5cmd?5?$CFs?6?$CC?$AA@ 200412c8     g_cmds.obj
 0002:000042e0       ??_C@_05BLKJBNOD@stats?$AA@ 200412e0     g_cmds.obj
 0002:000042e8       ??_C@_0L@CCEFBCKP@setviewpos?$AA@ 200412e8     g_cmds.obj
 0002:000042f4       ??_C@_02DPGMDCM@gc?$AA@    200412f4     g_cmds.obj
 0002:000042f8       ??_C@_08OLLMCBNG@teamvote?$AA@ 200412f8     g_cmds.obj
 0002:00004304       ??_C@_0N@JDBKAFAM@callteamvote?$AA@ 20041304     g_cmds.obj
 0002:00004314       ??_C@_04GHHIKFLG@vote?$AA@ 20041314     g_cmds.obj
 0002:0000431c       ??_C@_08NNMLCPB@callvote?$AA@ 2004131c     g_cmds.obj
 0002:00004328       ??_C@_05LCFPHLEE@where?$AA@ 20041328     g_cmds.obj
 0002:00004330       ??_C@_0L@FFKCNEMH@followprev?$AA@ 20041330     g_cmds.obj
 0002:0000433c       ??_C@_0L@GBHEMAKD@follownext?$AA@ 2004133c     g_cmds.obj
 0002:00004348       ??_C@_06HNJAFFAK@follow?$AA@ 20041348     g_cmds.obj
 0002:00004350       ??_C@_09EFOFPGPE@levelshot?$AA@ 20041350     g_cmds.obj
 0002:0000435c       ??_C@_06IHODGGMJ@noclip?$AA@ 2004135c     g_cmds.obj
 0002:00004364       ??_C@_08HPLPOCJL@notarget?$AA@ 20041364     g_cmds.obj
 0002:00004370       ??_C@_03DKFAMNOH@god?$AA@  20041370     g_cmds.obj
 0002:00004374       ??_C@_04BMBHJADG@give?$AA@ 20041374     g_cmds.obj
 0002:0000437c       ??_C@_06JMKGCPMO@votell?$AA@ 2004137c     g_cmds.obj
 0002:00004384       ??_C@_0L@GKKIAMHC@vosay_team?$AA@ 20041384     g_cmds.obj
 0002:00004390       ??_C@_05EGEGDMMG@vosay?$AA@ 20041390     g_cmds.obj
 0002:00004398       ??_C@_09CPIJOHHK@vsay_team?$AA@ 20041398     g_cmds.obj
 0002:000043a4       ??_C@_04IBCNHBFH@vsay?$AA@ 200413a4     g_cmds.obj
 0002:000043ac       ??_C@_04LBPCFPDD@tell?$AA@ 200413ac     g_cmds.obj
 0002:000043b4       ??_C@_08NBFNGOHN@say_team?$AA@ 200413b4     g_cmds.obj
 0002:000043c0       ??_C@_03BANJEMDJ@say?$AA@  200413c0     g_cmds.obj
 0002:000043c4       ??_C@_0M@BGKKOPE@MOD_GRAPPLE?$AA@ 200413c4     g_combat.obj
 0002:000043d0       ??_C@_0BB@JHNHPELL@MOD_TRIGGER_HURT?$AA@ 200413d0     g_combat.obj
 0002:000043e4       ??_C@_0BB@HMLMKPCA@MOD_TARGET_LASER?$AA@ 200413e4     g_combat.obj
 0002:000043f8       ??_C@_0M@NECNIJDJ@MOD_SUICIDE?$AA@ 200413f8     g_combat.obj
 0002:00004404       ??_C@_0M@JONLOPJN@MOD_FALLING?$AA@ 20041404     g_combat.obj
 0002:00004410       ??_C@_0N@IMHJNLFF@MOD_TELEFRAG?$AA@ 20041410     g_combat.obj
 0002:00004420       ??_C@_09GPMGMMBL@MOD_CRUSH?$AA@ 20041420     g_combat.obj
 0002:0000442c       ??_C@_08LEPCJCFO@MOD_LAVA?$AA@ 2004142c     g_combat.obj
 0002:00004438       ??_C@_09KBJPPHD@MOD_SLIME?$AA@ 20041438     g_combat.obj
 0002:00004444       ??_C@_09MAPLCDLI@MOD_WATER?$AA@ 20041444     g_combat.obj
 0002:00004450       ??_C@_0P@OHBIPEGK@MOD_BFG_SPLASH?$AA@ 20041450     g_combat.obj
 0002:00004460       ??_C@_07EOLOFKFM@MOD_BFG?$AA@ 20041460     g_combat.obj
 0002:00004468       ??_C@_0O@GLCOIAIP@MOD_LIGHTNING?$AA@ 20041468     g_combat.obj
 0002:00004478       ??_C@_0M@BHIJMBBE@MOD_RAILGUN?$AA@ 20041478     g_combat.obj
 0002:00004484       ??_C@_0BC@PIBHLJKK@MOD_PLASMA_SPLASH?$AA@ 20041484     g_combat.obj
 0002:00004498       ??_C@_0L@JPCJGHHF@MOD_PLASMA?$AA@ 20041498     g_combat.obj
 0002:000044a4       ??_C@_0BC@KJDNONBC@MOD_ROCKET_SPLASH?$AA@ 200414a4     g_combat.obj
 0002:000044b8       ??_C@_0L@FIOJJPEO@MOD_ROCKET?$AA@ 200414b8     g_combat.obj
 0002:000044c4       ??_C@_0BD@PLGCKMBF@MOD_GRENADE_SPLASH?$AA@ 200414c4     g_combat.obj
 0002:000044d8       ??_C@_0M@KDJNKEED@MOD_GRENADE?$AA@ 200414d8     g_combat.obj
 0002:000044e4       ??_C@_0P@DNHADEBJ@MOD_MACHINEGUN?$AA@ 200414e4     g_combat.obj
 0002:000044f4       ??_C@_0N@MJPPIPMF@MOD_GAUNTLET?$AA@ 200414f4     g_combat.obj
 0002:00004504       ??_C@_0M@MIHCLLAH@MOD_SHOTGUN?$AA@ 20041504     g_combat.obj
 0002:00004510       ??_C@_0M@BKDMLGAO@MOD_UNKNOWN?$AA@ 20041510     g_combat.obj
 0002:0000451c       ??_C@_0P@LIDDFKFD@kamikaze?5timer?$AA@ 2004151c     g_combat.obj
 0002:0000452c       ??_C@_0BB@JDBGHPJP@team_blueobelisk?$AA@ 2004152c     g_combat.obj
 0002:00004540       ??_C@_0BA@GIMOGCGC@team_redobelisk?$AA@ 20041540     g_combat.obj
 0002:00004550       ??_C@_0CE@HGPMHBOH@Kill?3?5?$CFi?5?$CFi?5?$CFi?3?5?$CFs?5killed?5?$CFs?5by?5@ 20041550     g_combat.obj
 0002:00004574       ??_C@_0P@BDPEDPJP@?$DMbad?5obituary?$DO?$AA@ 20041574     g_combat.obj
 0002:00004584       ??_C@_07GECLLGBL@?$DMworld?$DO?$AA@ 20041584     g_combat.obj
 0002:0000458c       ??_C@_0N@HGAIBNNB@?$DMnon?9client?$DO?$AA@ 2004158c     g_combat.obj
 0002:000045a0       __real@3fe51eb851eb851f    200415a0     g_combat.obj
 0002:000045a8       ??_C@_0CM@LEIIGBFN@?$CFi?3?5client?3?$CFi?5health?3?$CFi?5damage?3?$CF@ 200415a8     g_combat.obj
 0002:000045d4       __real@3ba3d70a            200415d4     g_combat.obj
 0002:000045d8       __real@402e000000000000    200415d8     g_combat.obj
 0002:000045e0       __real@43400000            200415e0     g_items.obj
 0002:000045e4       ??_C@_0CA@FLGMIHAB@sound?1items?1kamikazerespawn?4wav?$AA@ 200415e4     g_items.obj
 0002:00004604       ??_C@_0BM@BNLFEEPK@RespawnItem?3?5bad?5teammaster?$AA@ 20041604     g_items.obj
 0002:00004620       ??_C@_0N@OCCHADDH@Item?3?5?$CFi?5?$CFs?6?$AA@ 20041620     g_items.obj
 0002:00004630       __real@4069000000000000    20041630     g_items.obj
 0002:00004638       __real@4046800000000000    20041638     g_items.obj
 0002:00004640       ??_C@_0CJ@EMOANFCC@FinishSpawningItem?3?5?$CFs?5startsoli@ 20041640     g_items.obj
 0002:0000466c       __real@45800000            2004166c     g_items.obj
 0002:00004670       ??_C@_0CH@HHMBIMLK@?$FO3WARNING?3?5No?5team_CTF_blueflag?5@ 20041670     g_items.obj
 0002:00004698       ??_C@_0CG@DNHJENHJ@?$FO3WARNING?3?5No?5team_CTF_redflag?5i@ 20041698     g_items.obj
 0002:000046c0       ??_C@_0BD@LOGEPNHD@RegisterItem?3?5NULL?$AA@ 200416c0     g_items.obj
 0002:000046d4       ??_C@_0BF@PHBDLOMN@?$CFi?5items?5registered?6?$AA@ 200416d4     g_items.obj
 0002:000046ec       ??_C@_0L@BHNPAADM@disable_?$CFs?$AA@ 200416ec     g_items.obj
 0002:000046f8       ??_C@_0O@MNEGCFDN@noglobalsound?$AA@ 200416f8     g_items.obj
 0002:00004708       ??_C@_04PNOAOIAG@wait?$AA@ 20041708     g_items.obj
 0002:00004710       ??_C@_06NLFCANPD@random?$AA@ 20041710     g_items.obj
 0002:00004718       __real@c0000000            20041718     g_items.obj
 0002:0000471c       ??_C@_0L@NIHHPBKG@g_rankings?$AA@ 2004171c     g_main.obj
 0002:00004728       ??_C@_0M@HOGKGHBI@pmove_fixed?$AA@ 20041728     g_main.obj
 0002:00004734       ??_C@_0BA@EKPBHCCJ@g_smoothClients?$AA@ 20041734     g_main.obj
 0002:00004744       ??_C@_0N@JIFICDHI@g_listEntity?$AA@ 20041744     g_main.obj
 0002:00004754       ??_C@_0M@MECNLONK@g_allowVote?$AA@ 20041754     g_main.obj
 0002:00004760       ??_C@_02PFIAKEDG@80?$AA@   20041760     g_main.obj
 0002:00004764       ??_C@_09DKNLLEN@com_blood?$AA@ 20041764     g_main.obj
 0002:00004770       ??_C@_06IBNENCEO@g_motd?$AA@ 20041770     g_main.obj
 0002:00004778       ??_C@_0N@CGHOHBHC@g_debugAlloc?$AA@ 20041778     g_main.obj
 0002:00004788       ??_C@_0O@JCLHDLKF@g_debugDamage?$AA@ 20041788     g_main.obj
 0002:00004798       ??_C@_0M@EPOBGCBB@g_debugMove?$AA@ 20041798     g_main.obj
 0002:000047a4       ??_C@_0N@JGEKALLI@g_inactivity?$AA@ 200417a4     g_main.obj
 0002:000047b4       ??_C@_0P@JEPDGNEP@g_forcerespawn?$AA@ 200417b4     g_main.obj
 0002:000047c4       ??_C@_02PJNFELNH@30?$AA@   200417c4     g_main.obj
 0002:000047c8       ??_C@_0BE@CNNPIPEC@g_weaponTeamRespawn?$AA@ 200417c8     g_main.obj
 0002:000047dc       ??_C@_0BA@CMOCDPF@g_weaponrespawn?$AA@ 200417dc     g_main.obj
 0002:000047ec       ??_C@_01EKENIIDA@3?$AA@    200417ec     g_main.obj
 0002:000047f0       ??_C@_0N@LCBCFAFA@g_quadfactor?$AA@ 200417f0     g_main.obj
 0002:00004800       ??_C@_04KOJKLCBG@1000?$AA@ 20041800     g_main.obj
 0002:00004808       ??_C@_0M@PDFGFIOM@g_knockback?$AA@ 20041808     g_main.obj
 0002:00004814       ??_C@_03BAAJCDMO@800?$AA@  20041814     g_main.obj
 0002:00004818       ??_C@_09HNGNBNKN@g_gravity?$AA@ 20041818     g_main.obj
 0002:00004824       ??_C@_03MEIMHAKB@320?$AA@  20041824     g_main.obj
 0002:00004828       ??_C@_07KCHPCPJD@g_speed?$AA@ 20041828     g_main.obj
 0002:00004830       ??_C@_09BJOAODLF@dedicated?$AA@ 20041830     g_main.obj
 0002:0000483c       ??_C@_0L@MLCEEGBP@g_needpass?$AA@ 2004183c     g_main.obj
 0002:00004848       ??_C@_0M@NIKBMNDP@g_filterBan?$AA@ 20041848     g_main.obj
 0002:00004854       ??_C@_08NKMDLNHL@g_banIPs?$AA@ 20041854     g_main.obj
 0002:00004860       ??_C@_0L@GHAPAPFD@g_password?$AA@ 20041860     g_main.obj
 0002:0000486c       ??_C@_09IPDDEHO@g_logSync?$AA@ 2004186c     g_main.obj
 0002:00004878       ??_C@_09BNLGBMID@games?4log?$AA@ 20041878     g_main.obj
 0002:00004884       ??_C@_05PJEIAAGC@g_log?$AA@ 20041884     g_main.obj
 0002:0000488c       ??_C@_08HAMOJLDA@g_warmup?$AA@ 2004188c     g_main.obj
 0002:00004898       ??_C@_0BD@CLGJCDLA@g_teamForceBalance?$AA@ 20041898     g_main.obj
 0002:000048ac       ??_C@_0P@PONBNCIE@g_teamAutoJoin?$AA@ 200418ac     g_main.obj
 0002:000048bc       ??_C@_0P@IEOFAMLI@g_friendlyFire?$AA@ 200418bc     g_main.obj
 0002:000048cc       ??_C@_0BF@LICFCALK@g_synchronousClients?$AA@ 200418cc     g_main.obj
 0002:000048e4       ??_C@_0N@FCAHJCDA@capturelimit?$AA@ 200418e4     g_main.obj
 0002:000048f4       ??_C@_07GMGCLCAP@dmflags?$AA@ 200418f4     g_main.obj
 0002:000048fc       ??_C@_0BB@JCLDAPBF@g_maxGameClients?$AA@ 200418fc     g_main.obj
 0002:00004910       ??_C@_0L@DFBEGALI@sv_mapname?$AA@ 20041910     g_main.obj
 0002:0000491c       ??_C@_0M@GHMJJAD@g_restarted?$AA@ 2004191c     g_main.obj
 0002:00004928       ??_C@_0M@BBDAHLGI@May?525?52008?$AA@ 20041928     g_main.obj
 0002:00004934       ??_C@_08CLLHAKFA@gamedate?$AA@ 20041934     g_main.obj
 0002:00004940       ??_C@_06KOMAFLML@baseq3?$AA@ 20041940     g_main.obj
 0002:00004948       ??_C@_08HCPAIKAO@gamename?$AA@ 20041948     g_main.obj
 0002:00004954       ??_C@_09NFOPKLIK@sv_cheats?$AA@ 20041954     g_main.obj
 0002:00004960       ??_C@_0BL@EIPAHDOP@?$CFi?5teams?5with?5?$CFi?5entities?6?$AA@ 20041960     g_main.obj
 0002:0000497c       ??_C@_0DA@HFHMPEPI@g_gametype?5?$CFi?5is?5out?5of?5range?0?5d@ 2004197c     g_main.obj
 0002:000049ac       ??_C@_0CC@FFJICNKE@print?5?$CCServer?3?5?$CFs?5changed?5to?5?$CFs?6@ 200419ac     g_main.obj
 0002:000049d0       ??_C@_01INIBCBCB@f?$AA@    200419d0     g_main.obj
 0002:000049d4       ??_C@_0BJ@LMMLDPE@info_player_intermission?$AA@ 200419d4     g_main.obj
 0002:000049f0       ??_C@_0O@PKDALKNK@vstr?5nextmap?6?$AA@ 200419f0     g_main.obj
 0002:00004a00       ??_C@_0P@BKKOFHJN@map_restart?50?6?$AA@ 20041a00     g_main.obj
 0002:00004a10       ??_C@_09OHCHOIDO@?$CF3i?3?$CFi?$CFi?5?$AA@ 20041a10     g_main.obj
 0002:00004a1c       ??_C@_0CE@CGGOAMCD@score?3?5?$CFi?5?5ping?3?5?$CFi?5?5client?3?5?$CFi?5@ 20041a1c     g_main.obj
 0002:00004a40       ??_C@_0BB@HEGEAGAN@red?3?$CFi?5?5blue?3?$CFi?6?$AA@ 20041a40     g_main.obj
 0002:00004a54       ??_C@_09KHIKBPEI@Exit?3?5?$CFs?6?$AA@ 20041a54     g_main.obj
 0002:00004a60       ??_C@_0CE@BHHEOIMM@print?5?$CCBlue?5hit?5the?5capturelimit@ 20041a60     g_main.obj
 0002:00004a84       ??_C@_0BC@NGNDEIFJ@Capturelimit?5hit?4?$AA@ 20041a84     g_main.obj
 0002:00004a98       ??_C@_0CD@JENHKKNP@print?5?$CCRed?5hit?5the?5capturelimit?4@ 20041a98     g_main.obj
 0002:00004abc       ??_C@_0CB@FMCEIKLA@print?5?$CC?$CFs?$FO7?5hit?5the?5fraglimit?4?6?$CC@ 20041abc     g_main.obj
 0002:00004ae0       ??_C@_0CB@OIEPEJAM@print?5?$CCBlue?5hit?5the?5fraglimit?4?6?$CC@ 20041ae0     g_main.obj
 0002:00004b04       ??_C@_0P@PJCPOIKO@Fraglimit?5hit?4?$AA@ 20041b04     g_main.obj
 0002:00004b14       ??_C@_0CA@KPFPAKGG@print?5?$CCRed?5hit?5the?5fraglimit?4?6?$CC?$AA@ 20041b14     g_main.obj
 0002:00004b34       ??_C@_0P@EKMAOGJF@Timelimit?5hit?4?$AA@ 20041b34     g_main.obj
 0002:00004b44       ??_C@_0BI@GKJLDCNN@print?5?$CCTimelimit?5hit?4?6?$CC?$AA@ 20041b44     g_main.obj
 0002:00004b5c       ??_C@_08FFAHPNKC@Warmup?3?6?$AA@ 20041b5c     g_main.obj
 0002:00004b68       ??_C@_0BG@NEFGNBIH@print?5?$CCVote?5failed?4?6?$CC?$AA@ 20041b68     g_main.obj
 0002:00004b80       ??_C@_0BG@ICALOBOM@print?5?$CCVote?5passed?4?6?$CC?$AA@ 20041b80     g_main.obj
 0002:00004b98       ??_C@_0CD@EKLBBMMK@print?5?$CC?$CFs?5is?5the?5new?5team?5leader@ 20041b98     g_main.obj
 0002:00004bbc       ??_C@_0CH@IFAGPGDJ@print?5?$CC?$CFs?5is?5not?5on?5the?5team?5any@ 20041bbc     g_main.obj
 0002:00004be4       ??_C@_0BN@PMDPLBOA@print?5?$CC?$CFs?5is?5not?5connected?6?$CC?$AA@ 20041be4     g_main.obj
 0002:00004c04       ??_C@_0BL@FMHAJNKB@print?5?$CCTeam?5vote?5failed?4?6?$CC?$AA@ 20041c04     g_main.obj
 0002:00004c20       ??_C@_0BL@KCNKNMK@print?5?$CCTeam?5vote?5passed?4?6?$CC?$AA@ 20041c20     g_main.obj
 0002:00004c3c       ??_C@_0BA@JGLONBEK@NULL?5ent?9?$DOthink?$AA@ 20041c3c     g_main.obj
 0002:00004c4c       ??_C@_08JBKNBCEM@?$CF4i?3?5?$CFs?6?$AA@ 20041c4c     g_main.obj
 0002:00004c58       ??_C@_0BA@MOHNLIKA@com_buildScript?$AA@ 20041c58     g_main.obj
 0002:00004c68       ??_C@_0CF@MLCIJBNO@?9?9?9?9?9?9?9?9?9?9?9?9?9?9?9?9?9?9?9?9?9?9?9?9?9?9?9?9?9?9?9?9@ 20041c68     g_main.obj
 0002:00004c90       ??_C@_0BG@MOMCCAKP@Not?5logging?5to?5disk?4?6?$AA@ 20041c90     g_main.obj
 0002:00004ca8       ??_C@_0O@DEDEBKNJ@InitGame?3?5?$CFs?6?$AA@ 20041ca8     g_main.obj
 0002:00004cb8       ??_C@_0DO@BDNDJIG@?9?9?9?9?9?9?9?9?9?9?9?9?9?9?9?9?9?9?9?9?9?9?9?9?9?9?9?9?9?9?9?9@ 20041cb8     g_main.obj
 0002:00004cf8       ??_C@_0CE@PLBPIHPI@WARNING?3?5Couldn?8t?5open?5logfile?3?5@ 20041cf8     g_main.obj
 0002:00004d1c       ??_C@_0BF@CCJLMEBG@sound?1player?1fry?4wav?$AA@ 20041d1c     g_main.obj
 0002:00004d34       ??_C@_0O@LOFLFABD@gamedate?3?5?$CFs?6?$AA@ 20041d34     g_main.obj
 0002:00004d44       ??_C@_0O@MKINOKNK@gamename?3?5?$CFs?6?$AA@ 20041d44     g_main.obj
 0002:00004d54       ??_C@_0CF@FDKFKNJ@?9?9?9?9?9?9?9?5Game?5Initialization?5?9?9?9?9@ 20041d54     g_main.obj
 0002:00004d7c       ??_C@_0P@OFNEJLIL@ShutdownGame?3?6?$AA@ 20041d7c     g_main.obj
 0002:00004d8c       ??_C@_0BI@EOKPGBAF@?$DN?$DN?$DN?$DN?5ShutdownGame?5?$DN?$DN?$DN?$DN?6?$AA@ 20041d8c     g_main.obj
 0002:00004da4       ??_C@_0CL@HPAAECKJ@G_Alloc?3?5failed?5on?5allocation?5of@ 20041da4     g_mem.obj
 0002:00004dd0       ??_C@_0BP@CMDJHEKJ@G_Alloc?5of?5?$CFi?5bytes?5?$CI?$CFi?5left?$CJ?6?$AA@ 20041dd0     g_mem.obj
 0002:00004df0       ??_C@_0DC@GFNDCLPP@Game?5memory?5status?3?5?$CFi?5out?5of?5?$CFi@ 20041df0     g_mem.obj
 0002:00004e24       __real@43c80000            20041e24     g_misc.obj
 0002:00004e28       ??_C@_0CO@BGNILIGB@Couldn?8t?5find?5target?5for?5misc_pa@ 20041e28     g_misc.obj
 0002:00004e58       ??_C@_04FBAPEKPH@roll?$AA@ 20041e58     g_misc.obj
 0002:00004e60       __real@3c8efa35            20041e60     g_misc.obj
 0002:00004e64       __real@44fa0000            20041e64     g_missile.obj
 0002:00004e68       ??_C@_06BAPMGMJB@plasma?$AA@ 20041e68     g_missile.obj
 0002:00004e70       ??_C@_07JBPBHDIL@grenade?$AA@ 20041e70     g_missile.obj
 0002:00004e78       ??_C@_03CJHCFFJJ@bfg?$AA@  20041e78     g_missile.obj
 0002:00004e7c       __real@44610000            20041e7c     g_missile.obj
 0002:00004e80       ??_C@_06NHDMJEKK@rocket?$AA@ 20041e80     g_missile.obj
 0002:00004e88       ??_C@_04DGFIONEK@hook?$AA@ 20041e88     g_missile.obj
 0002:00004e90       __real@3fe4cccccccccccd    20041e90     g_missile.obj
 0002:00004e98       __real@408f400000000000    20041e98     g_mover.obj
 0002:00004ea0       ??_C@_0CE@HFNOCNBN@Reached_BinaryMover?3?5bad?5moverSt@ 20041ea0     g_mover.obj
 0002:00004ec4       __real@3e800000            20041ec4     g_mover.obj
 0002:00004ec8       ??_C@_05PEENBMOG@color?$AA@ 20041ec8     g_mover.obj
 0002:00004ed0       ??_C@_05PGFNHLMG@1?51?51?$AA@ 20041ed0     g_mover.obj
 0002:00004ed8       ??_C@_05OEPGNJB@light?$AA@ 20041ed8     g_mover.obj
 0002:00004ee0       ??_C@_05GPLCCBII@noise?$AA@ 20041ee0     g_mover.obj
 0002:00004ee8       ??_C@_0N@FKJMDFJC@door_trigger?$AA@ 20041ee8     g_mover.obj
 0002:00004ef8       ??_C@_03EMOFKE@dmg?$AA@    20041ef8     g_mover.obj
 0002:00004efc       ??_C@_0BP@MPMCKOBA@sound?1movers?1doors?1dr1_end?4wav?$AA@ 20041efc     g_mover.obj
 0002:00004f1c       ??_C@_0CA@KGLPIIML@sound?1movers?1doors?1dr1_strt?4wav?$AA@ 20041f1c     g_mover.obj
 0002:00004f3c       __real@42040000            20041f3c     g_mover.obj
 0002:00004f40       ??_C@_0N@GNEHAGP@plat_trigger?$AA@ 20041f40     g_mover.obj
 0002:00004f50       ??_C@_06LNLHEAAG@height?$AA@ 20041f50     g_mover.obj
 0002:00004f58       ??_C@_05HJCMGBKF@speed?$AA@ 20041f58     g_mover.obj
 0002:00004f60       ??_C@_0BP@FMIAEABD@sound?1movers?1plats?1pt1_end?4wav?$AA@ 20041f60     g_mover.obj
 0002:00004f80       ??_C@_0CA@DPCFJLJP@sound?1movers?1plats?1pt1_strt?4wav?$AA@ 20041f80     g_mover.obj
 0002:00004fa0       ??_C@_0CA@HPFJMDOC@sound?1movers?1switches?1butn2?4wav?$AA@ 20041fa0     g_mover.obj
 0002:00004fc0       ??_C@_0DB@KEBMPPOD@Train?5corner?5at?5?$CFs?5without?5a?5tar@ 20041fc0     g_mover.obj
 0002:00004ff4       ??_C@_0CF@EGOCJBJB@Train?5corner?5at?5?$CFs?5without?5a?5tar@ 20041ff4     g_mover.obj
 0002:0000501c       ??_C@_0M@ONCHNMHP@path_corner?$AA@ 2004201c     g_mover.obj
 0002:00005028       ??_C@_0CJ@BMOHOFCP@func_train?5at?5?$CFs?5with?5an?5unfound@ 20042028     g_mover.obj
 0002:00005054       ??_C@_0CG@DHHNMBFP@path_corner?5with?5no?5targetname?5a@ 20042054     g_mover.obj
 0002:0000507c       ??_C@_0CD@BNKPEMCB@func_train?5without?5a?5target?5at?5?$CF@ 2004207c     g_mover.obj
 0002:000050a0       ??_C@_05CBPKLGJM@phase?$AA@ 200420a0     g_mover.obj
 0002:000050a8       ??_C@_02MLODCJFF@32?$AA@   200420a8     g_mover.obj
 0002:000050b0       __real@3fc45f306446f9b4    200420b0     g_mover.obj
 0002:000050b8       ??_C@_0CC@FGLHJPEN@pushed_p?5?$DO?5?$CGpushed?$FLMAX_GENTITIES@ 200420b8     g_mover.obj
 0002:000050dc       ??_C@_09INHJFLOH@session?$CFi?$AA@ 200420dc     g_session.obj
 0002:000050e8       ??_C@_0BF@GKKABID@?$CFi?5?$CFi?5?$CFi?5?$CFi?5?$CFi?5?$CFi?5?$CFi?$AA@ 200420e8     g_session.obj
 0002:00005100       ??_C@_0CK@FAAHDCAM@Gametype?5changed?0?5clearing?5sessi@ 20042100     g_session.obj
 0002:0000512c       ??_C@_07KMJDECGK@session?$AA@ 2004212c     g_session.obj
 0002:00005134       ??_C@_0P@IPNNKHAH@teamtournament?$AA@ 20042134     g_spawn.obj
 0002:00005144       ??_C@_09KFJDBEJE@harvester?$AA@ 20042144     g_spawn.obj
 0002:00005150       ??_C@_07BNFEBHAE@obelisk?$AA@ 20042150     g_spawn.obj
 0002:00005158       ??_C@_07BEINKNPB@oneflag?$AA@ 20042158     g_spawn.obj
 0002:00005160       ??_C@_03JHHHHEKD@ctf?$AA@  20042160     g_spawn.obj
 0002:00005164       ??_C@_06EJFMBPJF@single?$AA@ 20042164     g_spawn.obj
 0002:0000516c       ??_C@_0L@NCEPCFLK@tournament?$AA@ 2004216c     g_spawn.obj
 0002:00005178       ??_C@_03PAEKGFEI@ffa?$AA@  20042178     g_spawn.obj
 0002:0000517c       ??_C@_0N@PAECNMEH@item_botroam?$AA@ 2004217c     g_spawn.obj
 0002:0000518c       ??_C@_0BD@GGIPJOIB@team_CTF_bluespawn?$AA@ 2004218c     g_spawn.obj
 0002:000051a0       ??_C@_0BC@KIKIBEND@team_CTF_redspawn?$AA@ 200421a0     g_spawn.obj
 0002:000051b4       ??_C@_0BE@COKGGHPD@team_CTF_blueplayer?$AA@ 200421b4     g_spawn.obj
 0002:000051c8       ??_C@_0BD@KLANHAKB@team_CTF_redplayer?$AA@ 200421c8     g_spawn.obj
 0002:000051dc       ??_C@_0P@KKMFIJKM@shooter_plasma?$AA@ 200421dc     g_spawn.obj
 0002:000051ec       ??_C@_0BA@MJCDAGHP@shooter_grenade?$AA@ 200421ec     g_spawn.obj
 0002:000051fc       ??_C@_0P@GNAFHBJH@shooter_rocket?$AA@ 200421fc     g_spawn.obj
 0002:0000520c       ??_C@_0BD@OJADMBDB@misc_portal_camera?$AA@ 2004220c     g_spawn.obj
 0002:00005220       ??_C@_0BE@FCJPPDGO@misc_portal_surface?$AA@ 20042220     g_spawn.obj
 0002:00005234       ??_C@_0L@PMAFMKKM@misc_model?$AA@ 20042234     g_spawn.obj
 0002:00005240       ??_C@_0BF@OMPOACGH@misc_teleporter_dest?$AA@ 20042240     g_spawn.obj
 0002:00005258       ??_C@_0M@NLNGBECJ@target_push?$AA@ 20042258     g_spawn.obj
 0002:00005264       ??_C@_0BA@BFKBOHOP@target_location?$AA@ 20042264     g_spawn.obj
 0002:00005274       ??_C@_0BA@NENIEICJ@target_position?$AA@ 20042274     g_spawn.obj
 0002:00005284       ??_C@_0M@KFDPHLNE@target_kill?$AA@ 20042284     g_spawn.obj
 0002:00005290       ??_C@_0BC@GJLLMIEM@target_teleporter?$AA@ 20042290     g_spawn.obj
 0002:000052a4       ??_C@_0N@DIKJAPJH@target_score?$AA@ 200422a4     g_spawn.obj
 0002:000052b4       ??_C@_0N@LGMMDFPN@target_laser?$AA@ 200422b4     g_spawn.obj
 0002:000052c4       ??_C@_0N@IADDOFND@target_print?$AA@ 200422c4     g_spawn.obj
 0002:000052d4       ??_C@_0P@MNJIBEAO@target_speaker?$AA@ 200422d4     g_spawn.obj
 0002:000052e4       ??_C@_0BH@FJADHEOA@target_remove_powerups?$AA@ 200422e4     g_spawn.obj
 0002:000052fc       ??_C@_0M@KALMALDK@target_give?$AA@ 200422fc     g_spawn.obj
 0002:00005308       ??_C@_0N@JFLGFCMM@trigger_hurt?$AA@ 20042308     g_spawn.obj
 0002:00005318       ??_C@_0BB@COMMHECA@trigger_teleport?$AA@ 20042318     g_spawn.obj
 0002:0000532c       ??_C@_0N@CCJDLJOF@trigger_push?$AA@ 2004232c     g_spawn.obj
 0002:0000533c       ??_C@_0P@KDHOHKJL@trigger_always?$AA@ 2004233c     g_spawn.obj
 0002:0000534c       ??_C@_0L@KLICIANB@func_group?$AA@ 2004234c     g_spawn.obj
 0002:00005358       ??_C@_0L@PGCOCBM@func_train?$AA@ 20042358     g_spawn.obj
 0002:00005364       ??_C@_0O@FPCFJAHB@func_pendulum?$AA@ 20042364     g_spawn.obj
 0002:00005374       ??_C@_0N@BAMIHEIF@func_bobbing?$AA@ 20042374     g_spawn.obj
 0002:00005384       ??_C@_0O@JDFCILJF@func_rotating?$AA@ 20042384     g_spawn.obj
 0002:00005394       ??_C@_0M@OOBMECJN@func_static?$AA@ 20042394     g_spawn.obj
 0002:000053a0       ??_C@_09HCDLIOGG@func_plat?$AA@ 200423a0     g_spawn.obj
 0002:000053ac       ??_C@_09BLMHBGJ@info_camp?$AA@ 200423ac     g_spawn.obj
 0002:000053b8       ??_C@_0N@FHKCBFMD@info_notnull?$AA@ 200423b8     g_spawn.obj
 0002:000053c8       ??_C@_09MBOCECHK@info_null?$AA@ 200423c8     g_spawn.obj
 0002:000053d4       ??_C@_0BC@IHPKIKNE@info_player_start?$AA@ 200423d4     g_spawn.obj
 0002:000053e8       ??_C@_0BE@OHABMMFD@targetShaderNewName?$AA@ 200423e8     g_spawn.obj
 0002:000053fc       ??_C@_0BB@FKLCNMKK@targetShaderName?$AA@ 200423fc     g_spawn.obj
 0002:00005410       ??_C@_06GNEAMJOC@angles?$AA@ 20042410     g_spawn.obj
 0002:00005418       ??_C@_05IOMEMJEC@count?$AA@ 20042418     g_spawn.obj
 0002:00005420       ??_C@_07ONPBMBOP@message?$AA@ 20042420     g_spawn.obj
 0002:00005428       ??_C@_06LNKHAAKC@model2?$AA@ 20042428     g_spawn.obj
 0002:00005430       ??_C@_0CC@JNJOINHG@?$CFs?5doesn?8t?5have?5a?5spawn?5function@ 20042430     g_spawn.obj
 0002:00005454       ??_C@_0BN@EMEGOFNC@G_CallSpawn?3?5NULL?5classname?6?$AA@ 20042454     g_spawn.obj
 0002:00005474       ??_C@_08NJPDEKHO@gametype?$AA@ 20042474     g_spawn.obj
 0002:00005480       ??_C@_06MFKCCKGP@notq3a?$AA@ 20042480     g_spawn.obj
 0002:00005488       ??_C@_07DDCDJNBH@notfree?$AA@ 20042488     g_spawn.obj
 0002:00005490       ??_C@_07CLBNBEAH@notteam?$AA@ 20042490     g_spawn.obj
 0002:00005498       ??_C@_09FDFEENEB@notsingle?$AA@ 20042498     g_spawn.obj
 0002:000054a4       ??_C@_0CE@JHGDANIP@G_AddSpawnVarToken?3?5MAX_SPAWN_CH@ 200424a4     g_spawn.obj
 0002:000054c8       ??_C@_0CB@JFPBODJK@G_ParseSpawnVars?3?5MAX_SPAWN_VARS@ 200424c8     g_spawn.obj
 0002:000054ec       ??_C@_0CN@NMMGIHBC@G_ParseSpawnVars?3?5closing?5brace?5@ 200424ec     g_spawn.obj
 0002:0000551c       ??_C@_0CM@DONEEOIH@G_ParseSpawnVars?3?5EOF?5without?5cl@ 2004251c     g_spawn.obj
 0002:00005548       ??_C@_0CM@CKLLJIGA@G_ParseSpawnVars?3?5found?5?$CFs?5when?5@ 20042548     g_spawn.obj
 0002:00005574       ??_C@_0P@INMNNPOJ@g_enableBreath?$AA@ 20042574     g_spawn.obj
 0002:00005584       ??_C@_0N@PNMKKPBO@enableBreath?$AA@ 20042584     g_spawn.obj
 0002:00005594       ??_C@_0N@CMGOADK@g_enableDust?$AA@ 20042594     g_spawn.obj
 0002:000055a4       ??_C@_0L@FLFKAOCP@enableDust?$AA@ 200425a4     g_spawn.obj
 0002:000055b0       ??_C@_07GFBFDLBM@gravity?$AA@ 200425b0     g_spawn.obj
 0002:000055b8       ??_C@_05LLDJOKNO@music?$AA@ 200425b8     g_spawn.obj
 0002:000055c0       ??_C@_08CCHPPKDI@baseq3?91?$AA@ 200425c0     g_spawn.obj
 0002:000055cc       ??_C@_0DD@EBBCPGHA@SP_worldspawn?3?5The?5first?5entity?5@ 200425cc     g_spawn.obj
 0002:00005600       ??_C@_0L@BIFLFHPF@worldspawn?$AA@ 20042600     g_spawn.obj
 0002:0000560c       ??_C@_0BL@HLOLFMOK@SpawnEntities?3?5no?5entities?$AA@ 2004260c     g_spawn.obj
 0002:00005628       ??_C@_0BI@DIECJMKD@Bad?5filter?5address?3?5?$CFs?6?$AA@ 20042628     g_svcmds.obj
 0002:00005640       ??_C@_0CO@DILFDDOI@g_banIPs?5overflowed?5at?5MAX_CVAR_@ 20042640     g_svcmds.obj
 0002:00005670       ??_C@_01LFCBOECM@?4?$AA@   20042670     g_svcmds.obj
 0002:00005674       ??_C@_01NBENCBCI@?$CK?$AA@ 20042674     g_svcmds.obj
 0002:00005678       ??_C@_0BI@LMFPAHLD@IP?5filter?5list?5is?5full?6?$AA@ 20042678     g_svcmds.obj
 0002:00005690       ??_C@_0BJ@LEBLJMPE@Usage?3?5?5addip?5?$DMip?9mask?$DO?6?$AA@ 20042690     g_svcmds.obj
 0002:000056ac       ??_C@_09HBKBHJKE@Removed?4?6?$AA@ 200426ac     g_svcmds.obj
 0002:000056b8       ??_C@_0BB@DFCHPNBP@Didn?8t?5find?5?$CFs?4?6?$AA@ 200426b8     g_svcmds.obj
 0002:000056cc       ??_C@_0BP@OJMGJOKB@Usage?3?5?5sv?5removeip?5?$DMip?9mask?$DO?6?$AA@ 200426cc     g_svcmds.obj
 0002:000056ec       ??_C@_01EEMJAFIK@?6?$AA@   200426ec     g_svcmds.obj
 0002:000056f0       ??_C@_0BF@HIBFLMFA@?$CF3i?5?5?5?5?5?5?5?5?5?5?5?5?5?5?5?5?5?$AA@ 200426f0     g_svcmds.obj
 0002:00005708       ??_C@_0BF@JEKJFFDI@ET_GRAPPLE?5?5?5?5?5?5?5?5?5?5?$AA@ 20042708     g_svcmds.obj
 0002:00005720       ??_C@_0BF@FONFEMNK@ET_INVISIBLE?5?5?5?5?5?5?5?5?$AA@ 20042720     g_svcmds.obj
 0002:00005738       ??_C@_0BF@KNGJOHIC@ET_TELEPORT_TRIGGER?5?$AA@ 20042738     g_svcmds.obj
 0002:00005750       ??_C@_0BF@JCJGMGAM@ET_PUSH_TRIGGER?5?5?5?5?5?$AA@ 20042750     g_svcmds.obj
 0002:00005768       ??_C@_0BF@JKKJEPNL@ET_SPEAKER?5?5?5?5?5?5?5?5?5?5?$AA@ 20042768     g_svcmds.obj
 0002:00005780       ??_C@_0BF@FABEBACG@ET_PORTAL?5?5?5?5?5?5?5?5?5?5?5?$AA@ 20042780     g_svcmds.obj
 0002:00005798       ??_C@_0BF@DBCLPHFC@ET_BEAM?5?5?5?5?5?5?5?5?5?5?5?5?5?$AA@ 20042798     g_svcmds.obj
 0002:000057b0       ??_C@_0BF@CKCOPBOH@ET_MOVER?5?5?5?5?5?5?5?5?5?5?5?5?$AA@ 200427b0     g_svcmds.obj
 0002:000057c8       ??_C@_0BF@JMOJKPHI@ET_MISSILE?5?5?5?5?5?5?5?5?5?5?$AA@ 200427c8     g_svcmds.obj
 0002:000057e0       ??_C@_0BF@IIDKJKIF@ET_ITEM?5?5?5?5?5?5?5?5?5?5?5?5?5?$AA@ 200427e0     g_svcmds.obj
 0002:000057f8       ??_C@_0BF@GHCCJGLD@ET_PLAYER?5?5?5?5?5?5?5?5?5?5?5?$AA@ 200427f8     g_svcmds.obj
 0002:00005810       ??_C@_0BF@GBIOGILC@ET_GENERAL?5?5?5?5?5?5?5?5?5?5?$AA@ 20042810     g_svcmds.obj
 0002:00005828       ??_C@_04LAMNNBAP@?$CF3i?3?$AA@ 20042828     g_svcmds.obj
 0002:00005830       ??_C@_0BO@DPIFHGAP@User?5?$CFs?5is?5not?5on?5the?5server?6?$AA@ 20042830     g_svcmds.obj
 0002:00005850       ??_C@_0BF@BEBENGBA@Bad?5client?5slot?3?5?$CFi?6?$AA@ 20042850     g_svcmds.obj
 0002:00005868       ??_C@_0BM@KMBENOOM@Client?5?$CFi?5is?5not?5connected?6?$AA@ 20042868     g_svcmds.obj
 0002:00005884       ??_C@_0BD@OKBENEII@print?5?$CCserver?3?5?$CFs?$CC?$AA@ 20042884     g_svcmds.obj
 0002:00005898       ??_C@_09DNOCIDID@g_banIPs?6?$AA@ 20042898     g_svcmds.obj
 0002:000058a4       ??_C@_06DDGIHMAP@listip?$AA@ 200428a4     g_svcmds.obj
 0002:000058ac       ??_C@_08FODIKFHA@removeip?$AA@ 200428ac     g_svcmds.obj
 0002:000058b8       ??_C@_05DNFKLKCD@addip?$AA@ 200428b8     g_svcmds.obj
 0002:000058c0       ??_C@_0N@EKGBLHCI@abort_podium?$AA@ 200428c0     g_svcmds.obj
 0002:000058d0       ??_C@_07OCFGLMLF@botlist?$AA@ 200428d0     g_svcmds.obj
 0002:000058d8       ??_C@_06CJHCPEHG@addbot?$AA@ 200428d8     g_svcmds.obj
 0002:000058e0       ??_C@_0M@OOGGMGEK@game_memory?$AA@ 200428e0     g_svcmds.obj
 0002:000058ec       ??_C@_09NGKIAGHE@forceteam?$AA@ 200428ec     g_svcmds.obj
 0002:000058f8       ??_C@_0L@CLDMIJOM@entitylist?$AA@ 200428f8     g_svcmds.obj
 0002:00005904       ??_C@_05EKJCMADO@delay?$AA@ 20042904     g_target.obj
 0002:0000590c       ??_C@_07PCJFOBJC@cp?5?$CC?$CFs?$CC?$AA@ 2004290c     g_target.obj
 0002:00005914       ??_C@_06MKMJDPPC@?$CFs?4wav?$AA@ 20042914     g_target.obj
 0002:0000591c       ??_C@_04IBLEHOMF@?4wav?$AA@ 2004291c     g_target.obj
 0002:00005924       ??_C@_0CJ@MCNLAIAG@target_speaker?5without?5a?5noise?5k@ 20042924     g_target.obj
 0002:00005950       ??_C@_07FGPCJFED@NOSOUND?$AA@ 20042950     g_target.obj
 0002:00005958       __real@45000000            20042958     g_target.obj
 0002:0000595c       ??_C@_0BO@JBAPADMO@?$CFs?5at?5?$CFs?3?5?$CFs?5is?5a?5bad?5target?6?$AA@ 2004295c     g_target.obj
 0002:0000597c       ??_C@_0CG@NCOEMBAJ@Couldn?8t?5find?5teleporter?5destina@ 2004297c     g_target.obj
 0002:000059a4       ??_C@_0BF@CCKDOAMJ@untargeted?5?$CFs?5at?5?$CFs?6?$AA@ 200429a4     g_target.obj
 0002:000059bc       ??_C@_07CIFAGBMG@unknown?$AA@ 200429bc     g_target.obj
 0002:000059c4       ??_C@_04HEDFJGEJ@FREE?$AA@ 200429c4     g_team.obj
 0002:000059cc       ??_C@_09GNDCBOBP@SPECTATOR?$AA@ 200429cc     g_team.obj
 0002:000059d8       ??_C@_04CNFFLDFF@BLUE?$AA@ 200429d8     g_team.obj
 0002:000059e0       ??_C@_03FNPLCCOA@RED?$AA@  200429e0     g_team.obj
 0002:000059e4       ??_C@_0BB@GAGKBLAF@PrintMsg?5overrun?$AA@ 200429e4     g_team.obj
 0002:000059f8       __real@45fa0000            200429f8     g_team.obj
 0002:000059fc       ??_C@_0CB@KOPONFBB@?$CFs?$FO7?5fragged?5?$CFs?8s?5flag?5carrier?$CB?6@ 200429fc     g_team.obj
 0002:00005a20       ??_C@_0BF@NFGOPKAE@team_CTF_neutralflag?$AA@ 20042a20     g_team.obj
 0002:00005a38       ??_C@_0CP@OBNDLAL@Warning?3?5?5NULL?5passed?5to?5Team_Re@ 20042a38     g_team.obj
 0002:00005a68       ??_C@_0CN@EPFNCNCH@Warning?3?5?5NULL?5passed?5to?5Team_Ta@ 20042a68     g_team.obj
 0002:00005a98       ??_C@_0DA@ICMFPMGB@Warning?3?5?5NULL?5passed?5to?5Team_Ca@ 20042a98     g_team.obj
 0002:00005ac8       ??_C@_0BL@EJNDMGGL@The?5?$CFs?5flag?5has?5returned?$CB?6?$AA@ 20042ac8     g_team.obj
 0002:00005ae4       ??_C@_0BI@KNNACEDO@The?5flag?5has?5returned?$CB?6?$AA@ 20042ae4     g_team.obj
 0002:00005afc       ??_C@_0BM@NKAOENPK@?$CFs?$FO7?5captured?5the?5?$CFs?5flag?$CB?6?$AA@ 20042afc     g_team.obj
 0002:00005b18       ??_C@_0BM@BDFECDMG@?$CFs?$FO7?5returned?5the?5?$CFs?5flag?$CB?6?$AA@ 20042b18     g_team.obj
 0002:00005b34       ??_C@_0BH@PJAKMCBO@?$CFs?$FO7?5got?5the?5?$CFs?5flag?$CB?6?$AA@ 20042b34     g_team.obj
 0002:00005b4c       ??_C@_0CG@PMIHGLOD@Don?8t?5know?5what?5team?5the?5flag?5is@ 20042b4c     g_team.obj
 0002:00005b74       ??_C@_08BKJPOMKC@?$CFc?$CFc?$CFs?$FO7?$AA@ 20042b74     g_team.obj
 0002:00005b80       ??_C@_0M@PHDLOMHJ@tinfo?5?$CFi?5?$CFs?$AA@ 20042b80     g_team.obj
 0002:00005b8c       ??_C@_0BD@FAPFLCHD@?5?$CFi?5?$CFi?5?$CFi?5?$CFi?5?$CFi?5?$CFi?$AA@ 20042b8c     g_team.obj
 0002:00005ba0       ??_C@_0BH@FEKNGHLG@sound?1misc?1windfly?4wav?$AA@ 20042ba0     g_trigger.obj
 0002:00005bb8       ??_C@_0BI@DGLBHPLI@sound?1world?1jumppad?4wav?$AA@ 20042bb8     g_trigger.obj
 0002:00005bd0       ??_C@_0CF@GJKCPHON@func_timer?5at?5?$CFs?5has?5random?5?$DO?$DN?5w@ 20042bd0     g_trigger.obj
 0002:00005bf8       ??_C@_0CF@LENMBBGI@trigger_multiple?5has?5random?5?$DO?$DN?5w@ 20042bf8     g_trigger.obj
 0002:00005c20       ??_C@_03LOHCHBBO@0?45?$AA@ 20042c20     g_trigger.obj
 0002:00005c24       ??_C@_0BI@KPLPFMKN@sound?1world?1electro?4wav?$AA@ 20042c24     g_trigger.obj
 0002:00005c3c       ??_C@_0N@MLGFLFEI@?$CFs?$DN?$CFs?3?$CF5?42f?$EA?$AA@ 20042c3c     g_utils.obj
 0002:00005c4c       ??_C@_0CC@KBENIHEG@G_FindConfigstringIndex?3?5overflo@ 20042c4c     g_utils.obj
 0002:00005c70       ??_C@_0CD@HHFHMIIH@G_PickTarget?3?5target?5?$CFs?5not?5foun@ 20042c70     g_utils.obj
 0002:00005c94       ??_C@_0CK@JOENGKNM@G_PickTarget?5called?5with?5NULL?5ta@ 20042c94     g_utils.obj
 0002:00005cc0       ??_C@_0CI@HMPHOHE@entity?5was?5removed?5while?5using?5t@ 20042cc0     g_utils.obj
 0002:00005ce8       ??_C@_0BO@JIDGNOMJ@WARNING?3?5Entity?5used?5itself?4?6?$AA@ 20042ce8     g_utils.obj
 0002:00005d08       ??_C@_0L@OPPGOKFJ@?$CI?$CFi?5?$CFi?5?$CFi?$CJ?$AA@ 20042d08     g_utils.obj
 0002:00005d14       __real@43870000            20042d14     g_utils.obj
 0002:00005d18       __real@404ca5dc0d03cf25    20042d18     g_utils.obj
 0002:00005d20       ??_C@_07CBNPCFPB@noclass?$AA@ 20042d20     g_utils.obj
 0002:00005d28       ??_C@_0BK@OECJBIJE@G_Spawn?3?5no?5free?5entities?$AA@ 20042d28     g_utils.obj
 0002:00005d44       ??_C@_05FAPHKBON@freed?$AA@ 20042d44     g_utils.obj
 0002:00005d4c       ??_C@_0CM@MOJHPIKM@G_AddEvent?3?5zero?5event?5added?5for@ 20042d4c     g_utils.obj
 0002:00005d78       ??_C@_0L@CPIFJPHE@tempEntity?$AA@ 20042d78     g_utils.obj
 0002:00005d84       __real@46000000            20042d84     g_weapon.obj
 0002:00005d88       __real@3e4ccccd            20042d88     g_weapon.obj
 0002:00005d8c       __real@41600000            20042d8c     g_weapon.obj
 0002:00005d90       __real@48000000            20042d90     g_weapon.obj
 0002:00005d94       __real@462f0000            20042d94     g_weapon.obj
 0002:00005d98       __real@44400000            20042d98     g_weapon.obj
 0002:00005d9c       __real@37800000            20042d9c     q_math.obj
 0002:00005da0       __real@4066c16c16c16c17    20042da0     q_math.obj
 0002:00005da8       ??_C@_0BJ@OLBOPICM@Q_strncpyz?3?5destsize?5?$DM?51?$AA@ 20042da8     q_shared.obj
 0002:00005dc4       ??_C@_0BF@BJHHBLMD@Q_strncpyz?3?5NULL?5src?$AA@ 20042dc4     q_shared.obj
 0002:00005ddc       ??_C@_0BG@EKAPNPCH@Q_strncpyz?3?5NULL?5dest?$AA@ 20042ddc     q_shared.obj
 0002:00005df4       ??_C@_0BN@EFOOAHFL@Q_strcat?3?5already?5overflowed?$AA@ 20042df4     q_shared.obj
 0002:00005e14       ??_C@_0CD@GIPJKOOD@Com_sprintf?3?5overflow?5of?5?$CFi?5in?5?$CF@ 20042e14     q_shared.obj
 0002:00005e38       ??_C@_0CC@GMEFDOKA@Com_sprintf?3?5overflowed?5bigbuffe@ 20042e38     q_shared.obj
 0002:00005e5c       ??_C@_0CG@FLHABLN@Info_ValueForKey?3?5oversize?5infos@ 20042e5c     q_shared.obj
 0002:00005e84       ??_C@_0CE@HMPLGKDK@Info_RemoveKey?3?5oversize?5infostr@ 20042e84     q_shared.obj
 0002:00005ea8       ??_C@_0CD@JIDDAEOO@Can?8t?5use?5keys?5or?5values?5with?5a?5@ 20042ea8     q_shared.obj
 0002:00005ecc       ??_C@_0CL@JCFAGLFD@Can?8t?5use?5keys?5or?5values?5with?5a?5@ 20042ecc     q_shared.obj
 0002:00005ef8       ??_C@_0CD@MGFMEBLE@Can?8t?5use?5keys?5or?5values?5with?5a?5@ 20042ef8     q_shared.obj
 0002:00005f1c       ??_C@_0BN@CAOBGKLE@Info?5string?5length?5exceeded?6?$AA@ 20042f1c     q_shared.obj
 0002:00005f3c       ??_C@_06NELKLDPM@?2?$CFs?2?$CFs?$AA@ 20042f3c     q_shared.obj
 0002:00005f44       ??_C@_0CJ@CEEBDGNA@Info_SetValueForKey?3?5oversize?5in@ 20042f44     q_shared.obj
 0002:00005fc8       __real@0000000000000000    20042fc8     LIBC:cvt.obj
 0002:00005fd0       ??_C@_05KLBDPFGC@e?$CL000?$AA@ 20042fd0     LIBC:cvt.obj
 0002:00005fd8       __real@4150017ec0000000    20042fd8     LIBC:testfdiv.obj
 0002:00005fe0       __real@4147ffff80000000    20042fe0     LIBC:testfdiv.obj
 0002:00005fe8       ??_C@_0BK@NHEOCAHP@IsProcessorFeaturePresent?$AA@ 20042fe8     LIBC:testfdiv.obj
 0002:00006004       ??_C@_08CPNIBGIE@KERNEL32?$AA@ 20043004     LIBC:testfdiv.obj
 0002:00006010       ___newctype                20043010     LIBC:ctype.obj
 0002:00006310       __wctype                   20043310     LIBC:ctype.obj
 0002:00006524       ??_C@_13NOLLCAOD@?$AA?$AA?$AA?$AA@ 20043524     LIBC:a_map.obj
 0002:00006550       ___lookuptable             20043550     LIBC:output.obj
 0002:000065ac       ??_C@_1O@CEDCILHN@?$AA?$CI?$AAn?$AAu?$AAl?$AAl?$AA?$CJ?$AA?$AA@ 200435ac     LIBC:output.obj
 0002:000065bc       ??_C@_06OJHGLDPL@?$CInull?$CJ?$AA@ 200435bc     LIBC:output.obj
 0002:00006630       ??_C@_04MLLJIGOK@atan?$AA@ 20043630     LIBC:libm_error.obj
 0002:00006638       ??_C@_04GFPJNGEK@ceil?$AA@ 20043638     LIBC:libm_error.obj
 0002:00006640       ??_C@_05PBJFFIGL@floor?$AA@ 20043640     LIBC:libm_error.obj
 0002:00006648       ??_C@_04EHEDPDJG@modf?$AA@ 20043648     LIBC:libm_error.obj
 0002:00006650       ??_C@_04HPAFEEIN@exp2?$AA@ 20043650     LIBC:libm_error.obj
 0002:00006658       ??_C@_05EOHGHCHD@exp10?$AA@ 20043658     LIBC:libm_error.obj
 0002:00006660       ??_C@_04KGLCPMCP@log2?$AA@ 20043660     LIBC:libm_error.obj
 0002:00006668       ??_C@_03JGHBODFD@pow?$AA@  20043668     LIBC:libm_error.obj
 0002:0000666c       ??_C@_05HGHHAHAP@log10?$AA@ 2004366c     LIBC:libm_error.obj
 0002:00006674       ??_C@_03KHJOGHMM@exp?$AA@  20043674     LIBC:libm_error.obj
 0002:00006684       ??_C@_0N@FFJGBINN@AuthenticAMD?$AA@ 20043684     LIBC:cpu_disp.obj
 0002:00006694       ??_C@_0P@MIGLKIOC@CorExitProcess?$AA@ 20043694     LIBC:crt0dat.obj
 0002:000066a4       ??_C@_0M@MBOPBNBK@mscoree?4dll?$AA@ 200436a4     LIBC:crt0dat.obj
 0002:000066cc       ??_C@_0P@GGKDKEEG@runtime?5error?5?$AA@ 200436cc     LIBC:crt0msg.obj
 0002:000066dc       ??_C@_02PCIJFNDE@?$AN?6?$AA@ 200436dc     LIBC:crt0msg.obj
 0002:000066e0       ??_C@_0O@MJNIPGOH@TLOSS?5error?$AN?6?$AA@ 200436e0     LIBC:crt0msg.obj
 0002:000066f0       ??_C@_0N@BONNPDHF@SING?5error?$AN?6?$AA@ 200436f0     LIBC:crt0msg.obj
 0002:00006700       ??_C@_0P@MBDAJNE@DOMAIN?5error?$AN?6?$AA@ 20043700     LIBC:crt0msg.obj
 0002:00006710       ??_C@_0KC@BDDGGBEJ@R6029?$AN?6?9?5This?5application?5cannot@ 20043710     LIBC:crt0msg.obj
 0002:000067b4       ??_C@_0CF@KJDAIALP@R6028?$AN?6?9?5unable?5to?5initialize?5he@ 200437b4     LIBC:crt0msg.obj
 0002:000067dc       ??_C@_0DF@GAKBPDFP@R6027?$AN?6?9?5not?5enough?5space?5for?5lo@ 200437dc     LIBC:crt0msg.obj
 0002:00006814       ??_C@_0DF@IBLNNAIG@R6026?$AN?6?9?5not?5enough?5space?5for?5st@ 20043814     LIBC:crt0msg.obj
 0002:0000684c       ??_C@_0CG@IOHKGFNJ@R6025?$AN?6?9?5pure?5virtual?5function?5c@ 2004384c     LIBC:crt0msg.obj
 0002:00006874       ??_C@_0DF@JIJJFJDC@R6024?$AN?6?9?5not?5enough?5space?5for?5_o@ 20043874     LIBC:crt0msg.obj
 0002:000068ac       ??_C@_0CJ@EGEJHFME@R6019?$AN?6?9?5unable?5to?5open?5console?5@ 200438ac     LIBC:crt0msg.obj
 0002:000068d8       ??_C@_0CB@GNHNIELH@R6018?$AN?6?9?5unexpected?5heap?5error?$AN?6@ 200438d8     LIBC:crt0msg.obj
 0002:000068fc       ??_C@_0CN@FOLDKNG@R6017?$AN?6?9?5unexpected?5multithread?5@ 200438fc     LIBC:crt0msg.obj
 0002:0000692c       ??_C@_0CM@FAHFJNHO@R6016?$AN?6?9?5not?5enough?5space?5for?5th@ 2004392c     LIBC:crt0msg.obj
 0002:00006958       ??_C@_0JG@LBKMGKLD@?$AN?6This?5application?5has?5requested@ 20043958     LIBC:crt0msg.obj
 0002:000069f0       ??_C@_0CM@FLCNIPKK@R6009?$AN?6?9?5not?5enough?5space?5for?5en@ 200439f0     LIBC:crt0msg.obj
 0002:00006a1c       ??_C@_0CK@KMMJOAPP@R6008?$AN?6?9?5not?5enough?5space?5for?5ar@ 20043a1c     LIBC:crt0msg.obj
 0002:00006a48       ??_C@_0CF@HOHMHDEK@R6002?$AN?6?9?5floating?5point?5not?5load@ 20043a48     LIBC:crt0msg.obj
 0002:00006a70       ??_C@_0CF@GOGNBNAK@Microsoft?5Visual?5C?$CL?$CL?5Runtime?5Lib@ 20043a70     LIBC:crt0msg.obj
 0002:00006a98       ??_C@_02PHMGELLB@?6?6?$AA@ 20043a98     LIBC:crt0msg.obj
 0002:00006a9c       ??_C@_0BK@OFGJDLJJ@Runtime?5Error?$CB?6?6Program?3?5?$AA@ 20043a9c     LIBC:crt0msg.obj
 0002:00006ab8       ??_C@_03KHICJKCI@?4?4?4?$AA@ 20043ab8     LIBC:crt0msg.obj
 0002:00006abc       ??_C@_0BH@DNAGHKFM@?$DMprogram?5name?5unknown?$DO?$AA@ 20043abc     LIBC:crt0msg.obj
 0002:00006b04       ??_C@_0L@KDOEJCKC@_nextafter?$AA@ 20043b04     LIBC:fpexcept.obj
 0002:00006b10       ??_C@_05JGDBENOH@_logb?$AA@ 20043b10     LIBC:fpexcept.obj
 0002:00006b18       ??_C@_03ONILCKOB@_yn?$AA@  20043b18     LIBC:fpexcept.obj
 0002:00006b1c       ??_C@_03NAKIGLHK@_y1?$AA@  20043b1c     LIBC:fpexcept.obj
 0002:00006b20       ??_C@_03MJLDFKDL@_y0?$AA@  20043b20     LIBC:fpexcept.obj
 0002:00006b24       ??_C@_05GKKHEGJL@frexp?$AA@ 20043b24     LIBC:fpexcept.obj
 0002:00006b2c       ??_C@_04KEPJIHGP@fmod?$AA@ 20043b2c     LIBC:fpexcept.obj
 0002:00006b34       ??_C@_06MEIMCGCF@_hypot?$AA@ 20043b34     LIBC:fpexcept.obj
 0002:00006b3c       ??_C@_05KBKMEMPO@_cabs?$AA@ 20043b3c     LIBC:fpexcept.obj
 0002:00006b44       ??_C@_05CEJMAHNP@ldexp?$AA@ 20043b44     LIBC:fpexcept.obj
 0002:00006b4c       ??_C@_04ODHECPBC@fabs?$AA@ 20043b4c     LIBC:fpexcept.obj
 0002:00006b54       ??_C@_03IIINPABG@tan?$AA@  20043b54     LIBC:fpexcept.obj
 0002:00006b58       ??_C@_03LALBNOCG@cos?$AA@  20043b58     LIBC:fpexcept.obj
 0002:00006b5c       ??_C@_03BLEJJJBH@sin?$AA@  20043b5c     LIBC:fpexcept.obj
 0002:00006b60       ??_C@_04EIAKFFMI@sqrt?$AA@ 20043b60     LIBC:fpexcept.obj
 0002:00006b68       ??_C@_05KNGEOGJB@atan2?$AA@ 20043b68     LIBC:fpexcept.obj
 0002:00006b70       ??_C@_04PDIFKINK@acos?$AA@ 20043b70     LIBC:fpexcept.obj
 0002:00006b78       ??_C@_04FIHNOPOL@asin?$AA@ 20043b78     LIBC:fpexcept.obj
 0002:00006b80       ??_C@_04FJHINJAO@tanh?$AA@ 20043b80     LIBC:fpexcept.obj
 0002:00006b88       ??_C@_04HPJJNFIM@cosh?$AA@ 20043b88     LIBC:fpexcept.obj
 0002:00006b90       ??_C@_04COOMCNPB@sinh?$AA@ 20043b90     LIBC:fpexcept.obj
 0002:00006b98       ??_C@_0BI@DFKBFLJE@GetProcessWindowStation?$AA@ 20043b98     LIBC:crtmbox.obj
 0002:00006bb0       ??_C@_0BK@CIDNPOGP@GetUserObjectInformationA?$AA@ 20043bb0     LIBC:crtmbox.obj
 0002:00006bcc       ??_C@_0BD@HHGDFDBJ@GetLastActivePopup?$AA@ 20043bcc     LIBC:crtmbox.obj
 0002:00006be0       ??_C@_0BA@HNOPNCHB@GetActiveWindow?$AA@ 20043be0     LIBC:crtmbox.obj
 0002:00006bf0       ??_C@_0M@CHKKJDAI@MessageBoxA?$AA@ 20043bf0     LIBC:crtmbox.obj
 0002:00006bfc       ??_C@_0L@GMPLCCII@user32?4dll?$AA@ 20043bfc     LIBC:crtmbox.obj
 0002:00006c08       ??_C@_06IMKFLFPG@1?$CDQNAN?$AA@ 20043c08     LIBC:x10fout.obj
 0002:00006c10       ??_C@_05DNEBIAHO@1?$CDINF?$AA@ 20043c10     LIBC:x10fout.obj
 0002:00006c18       ??_C@_05PHHOCPM@1?$CDIND?$AA@ 20043c18     LIBC:x10fout.obj
 0002:00006c20       ??_C@_06PGGFOGJG@1?$CDSNAN?$AA@ 20043c20     LIBC:x10fout.obj
 0002:00006c28       ??_C@_09KLGCKDOD@Program?3?5?$AA@ 20043c28     LIBC:secfail.obj
 0002:00006c38       ??_C@_0KA@JEHFIFGP@A?5buffer?5overrun?5has?5been?5detect@ 20043c38     LIBC:secfail.obj
 0002:00006cd8       ??_C@_0BJ@MDEKIEOJ@Buffer?5overrun?5detected?$CB?$AA@ 20043cd8     LIBC:secfail.obj
 0002:00006cf8       ??_C@_0LB@BPLHHLFD@A?5security?5error?5of?5unknown?5caus@ 20043cf8     LIBC:secfail.obj
 0002:00006dac       ??_C@_0CD@GMKACBEK@Unknown?5security?5failure?5detecte@ 20043dac     LIBC:secfail.obj
 0002:00006de0       __load_config_used         20043de0     LIBC:loadcfg.obj
 0002:00006e30       ___safe_se_handler_table   20043e30     <linker-defined>
 0002:00006e38       ___rtc_iaa                 20043e38     LIBC:initsect.obj
 0002:00006e3c       ___rtc_izz                 20043e3c     LIBC:initsect.obj
 0002:00006e40       ___rtc_taa                 20043e40     LIBC:initsect.obj
 0002:00006e44       ___rtc_tzz                 20043e44     LIBC:initsect.obj
 0002:00006e48       __IMPORT_DESCRIPTOR_KERNEL32 20043e48     kernel32:KERNEL32.dll
 0002:00006e5c       __NULL_IMPORT_DESCRIPTOR   20043e5c     kernel32:KERNEL32.dll
 0003:00000000       ___xc_a                    20045000     LIBC:crt0init.obj
 0003:00000008       ___xc_z                    20045008     LIBC:crt0init.obj
 0003:0000000c       ___xi_a                    2004500c     LIBC:crt0init.obj
 0003:00000020       ___xi_z                    20045020     LIBC:crt0init.obj
 0003:00000024       ___xp_a                    20045024     LIBC:crt0init.obj
 0003:0000002c       ___xp_z                    2004502c     LIBC:crt0init.obj
 0003:00000030       ___xt_a                    20045030     LIBC:crt0init.obj
 0003:00000034       ___xt_z                    20045034     LIBC:crt0init.obj
 0003:00000070       _voiceCommands             20045070     ai_vcmd.obj
 0003:000000e8       _bg_itemlist               200450e8     bg_misc.obj
 0003:0000086c       _bg_numItems               2004586c     bg_misc.obj
 0003:00000870       _eventnames                20045870     bg_misc.obj
 0003:000009a0       _pm_stopspeed              200459a0     bg_pmove.obj
 0003:000009a4       _pm_duckScale              200459a4     bg_pmove.obj
 0003:000009a8       _pm_swimScale              200459a8     bg_pmove.obj
 0003:000009ac       _pm_wadeScale              200459ac     bg_pmove.obj
 0003:000009b0       _pm_accelerate             200459b0     bg_pmove.obj
 0003:000009b4       _pm_airaccelerate          200459b4     bg_pmove.obj
 0003:000009b8       _pm_wateraccelerate        200459b8     bg_pmove.obj
 0003:000009bc       _pm_flyaccelerate          200459bc     bg_pmove.obj
 0003:000009c0       _pm_friction               200459c0     bg_pmove.obj
 0003:000009c4       _pm_waterfriction          200459c4     bg_pmove.obj
 0003:000009c8       _pm_flightfriction         200459c8     bg_pmove.obj
 0003:000009cc       _pm_spectatorfriction      200459cc     bg_pmove.obj
 0003:00000a58       _modNames                  20045a58     g_combat.obj
 0003:00000fc8       _fields                    20045fc8     g_spawn.obj
 0003:00001118       _spawns                    20046118     g_spawn.obj
 0003:00001308       _axisDefault               20046308     q_math.obj
 0003:0000132c       _colorBlack                2004632c     q_math.obj
 0003:0000133c       _colorRed                  2004633c     q_math.obj
 0003:0000134c       _colorGreen                2004634c     q_math.obj
 0003:0000135c       _colorBlue                 2004635c     q_math.obj
 0003:0000136c       _colorYellow               2004636c     q_math.obj
 0003:0000137c       _colorMagenta              2004637c     q_math.obj
 0003:0000138c       _colorCyan                 2004638c     q_math.obj
 0003:0000139c       _colorWhite                2004639c     q_math.obj
 0003:000013ac       _colorLtGrey               200463ac     q_math.obj
 0003:000013bc       _colorMdGrey               200463bc     q_math.obj
 0003:000013cc       _colorDkGrey               200463cc     q_math.obj
 0003:000013e0       _g_color_table             200463e0     q_math.obj
 0003:00001460       _bytedirs                  20046460     q_math.obj
 0003:00001bfc       __fltused                  20046bfc     LIBC:fpinit.obj
 0003:00001c00       __ldused                   20046c00     LIBC:fpinit.obj
 0003:00001c04       __FPinit                   20046c04     LIBC:fpinit.obj
 0003:00001c08       __FPmtinit                 20046c08     LIBC:fpinit.obj
 0003:00001c0c       __FPmtterm                 20046c0c     LIBC:fpinit.obj
 0003:00001c10       __aexit_rtn                20046c10     LIBC:dllcrt0.obj
 0003:00001c20       __cfltcvt_tab              20046c20     LIBC:cmiscdat.obj
 0003:00001c40       __pctype                   20046c40     LIBC:ctype.obj
 0003:00001c44       __pwctype                  20046c44     LIBC:ctype.obj
 0003:00001c48       ___mb_cur_max              20046c48     LIBC:nlsdata1.obj
 0003:00001c4c       ___decimal_point           20046c4c     LIBC:nlsdata1.obj
 0003:00001c50       ___decimal_point_length    20046c50     LIBC:nlsdata1.obj
 0003:00001c54       ___lc_clike                20046c54     LIBC:nlsdata2.obj
 0003:00001c58       ___nullstring              20046c58     LIBC:output.obj
 0003:00001c5c       ___wnullstring             20046c5c     LIBC:output.obj
 0003:00001c60       __pmatherr                 20046c60     LIBC:libm_error.obj
 0003:00001c68       ___badioinfo               20046c68     LIBC:ioinit.obj
 0003:00001c70       __amblksiz                 20046c70     LIBC:heapinit.obj
 0003:00001c78       __XcptActTab               20046c78     LIBC:winxfltr.obj
 0003:00001cf0       __First_FPE_Indx           20046cf0     LIBC:winxfltr.obj
 0003:00001cf4       __Num_FPE                  20046cf4     LIBC:winxfltr.obj
 0003:00001cf8       __XcptActTabCount          20046cf8     LIBC:winxfltr.obj
 0003:00001cfc       __fpecode                  20046cfc     LIBC:winxfltr.obj
 0003:00001ec0       ___security_cookie         20046ec0     LIBC:seccook.obj
 0003:00001ec8       __iob                      20046ec8     LIBC:_file.obj
 0003:00002150       __matherr_flag             20047150     LIBC:matherr.obj
 0003:00002248       __d_inf                    20047248     LIBC:util.obj
 0003:00002250       __d_ind                    20047250     LIBC:util.obj
 0003:00002258       __d_max                    20047258     LIBC:util.obj
 0003:00002260       __d_min                    20047260     LIBC:util.obj
 0003:00002268       __d_mzero                  20047268     LIBC:util.obj
 0003:00002290       __NLG_Destination          20047290     LIBC:exsup.obj
 0003:00002408       __pow10pos                 20047408     LIBC:constpow.obj
 0003:00002568       __pow10neg                 20047568     LIBC:constpow.obj
 0003:00002808       _c_pmove                   20047808     bg_pmove.obj
 0003:00047e18       _remapCount                2008ce18     g_utils.obj
 0003:00047e8c       _vec3_origin               2008ce8c     q_math.obj
 0003:0005e0a8       ___fastflag                200a30a8     LIBC:fpinit.obj
 0003:0005e0ac       __adjust_fdiv              200a30ac     LIBC:fpinit.obj
 0003:0005e0b4       __aenvptr                  200a30b4     LIBC:dllcrt0.obj
 0003:0005e0b8       __wenvptr                  200a30b8     LIBC:dllcrt0.obj
 0003:0005e0bc       ___error_mode              200a30bc     LIBC:dllcrt0.obj
 0003:0005e0c0       ___app_type                200a30c0     LIBC:dllcrt0.obj
 0003:0005e0f4       ___lc_handle               200a30f4     LIBC:nlsdata2.obj
 0003:0005e10c       ___lc_codepage             200a310c     LIBC:nlsdata2.obj
 0003:0005e110       ___lc_collate_cp           200a3110     LIBC:nlsdata2.obj
 0003:0005e114       _errno                     200a3114     LIBC:crt0dat.obj
 0003:0005e118       __doserrno                 200a3118     LIBC:crt0dat.obj
 0003:0005e11c       __umaskval                 200a311c     LIBC:crt0dat.obj
 0003:0005e120       __osplatform               200a3120     LIBC:crt0dat.obj
 0003:0005e124       __osver                    200a3124     LIBC:crt0dat.obj
 0003:0005e128       __winver                   200a3128     LIBC:crt0dat.obj
 0003:0005e12c       __winmajor                 200a312c     LIBC:crt0dat.obj
 0003:0005e130       __winminor                 200a3130     LIBC:crt0dat.obj
 0003:0005e134       ___argc                    200a3134     LIBC:crt0dat.obj
 0003:0005e138       ___argv                    200a3138     LIBC:crt0dat.obj
 0003:0005e13c       ___wargv                   200a313c     LIBC:crt0dat.obj
 0003:0005e140       __environ                  200a3140     LIBC:crt0dat.obj
 0003:0005e144       ___initenv                 200a3144     LIBC:crt0dat.obj
 0003:0005e148       __wenviron                 200a3148     LIBC:crt0dat.obj
 0003:0005e14c       ___winitenv                200a314c     LIBC:crt0dat.obj
 0003:0005e150       __pgmptr                   200a3150     LIBC:crt0dat.obj
 0003:0005e154       __wpgmptr                  200a3154     LIBC:crt0dat.obj
 0003:0005e158       __exitflag                 200a3158     LIBC:crt0dat.obj
 0003:0005e15c       __C_Termination_Done       200a315c     LIBC:crt0dat.obj
 0003:0005e160       __C_Exit_Done              200a3160     LIBC:crt0dat.obj
 0003:0005e274       __pxcptinfoptrs            200a3274     LIBC:winxfltr.obj
 0003:0005e278       __adbgmsg                  200a3278     LIBC:crt0msg.obj
 0003:0005e2b0       __cflush                   200a32b0     LIBC:_file.obj
 0003:0005e31c       ?_pnhHeap@@3P6AHI@ZA       200a331c     LIBC:handler.obj
 0003:0005e320       __newmode                  200a3320     LIBC:_newmode.obj
 0003:0005e340       _remappedShaders           200a3340     <common>
 0003:00062540       _teamgame                  200a7540     <common>
 0003:00062580       _pushed                    200a7580     <common>
 0003:0006a580       _pushed_p                  200af580     <common>
 0003:0006a5a0       _g_password                200af5a0     <common>
 0003:0006a6c0       _g_smoothClients           200af6c0     <common>
 0003:0006a7e0       _g_friendlyFire            200af7e0     <common>
 0003:0006a900       _g_podiumDist              200af900     <common>
 0003:0006aa20       _g_gravity                 200afa20     <common>
 0003:0006ab40       _g_filterBan               200afb40     <common>
 0003:0006ac60       _g_entities                200afc60     <common>
 0003:00134c60       _g_restarted               20179c60     <common>
 0003:00134d80       _g_quadfactor              20179d80     <common>
 0003:00134ea0       _g_debugMove               20179ea0     <common>
 0003:00134fc0       _g_weaponTeamRespawn       20179fc0     <common>
 0003:001350e0       _g_fraglimit               2017a0e0     <common>
 0003:00135200       _g_dmflags                 2017a200     <common>
 0003:00135320       _g_maxclients              2017a320     <common>
 0003:00135440       _pmove_msec                2017a440     <common>
 0003:00135560       _g_synchronousClients      2017a560     <common>
 0003:00135680       _g_knockback               2017a680     <common>
 0003:001357a0       _g_warmup                  2017a7a0     <common>
 0003:001358c0       _g_weaponRespawn           2017a8c0     <common>
 0003:001359e0       _g_allowVote               2017a9e0     <common>
 0003:00135b00       _g_debugAlloc              2017ab00     <common>
 0003:00135c20       _g_dedicated               2017ac20     <common>
 0003:00135d40       _g_rankings                2017ad40     <common>
 0003:00135e60       _g_timelimit               2017ae60     <common>
 0003:00135f80       _g_needpass                2017af80     <common>
 0003:001360a0       _g_blood                   2017b0a0     <common>
 0003:001361c0       _g_listEntity              2017b1c0     <common>
 0003:001362e0       _g_inactivity              2017b2e0     <common>
 0003:00136400       _g_cheats                  2017b400     <common>
 0003:00136520       _g_maxGameClients          2017b520     <common>
 0003:00136640       _g_speed                   2017b640     <common>
 0003:00136760       _g_log                     2017b760     <common>
 0003:00136880       _g_teamForceBalance        2017b880     <common>
 0003:001369a0       _g_banIPs                  2017b9a0     <common>
 0003:00136ac0       _g_gametype                2017bac0     <common>
 0003:00136be0       _g_capturelimit            2017bbe0     <common>
 0003:00136d00       _pmove_fixed               2017bd00     <common>
 0003:00136e20       _g_doWarmup                2017be20     <common>
 0003:00136f40       _g_logSync                 2017bf40     <common>
 0003:00137060       _g_teamAutoJoin            2017c060     <common>
 0003:00137180       _g_podiumDrop              2017c180     <common>
 0003:001372a0       _g_motd                    2017c2a0     <common>
 0003:001373c0       _g_debugDamage             2017c3c0     <common>
 0003:001374e0       _g_clients                 2017c4e0     <common>
 0003:001436e0       _g_forcerespawn            201886e0     <common>
 0003:00143800       _level                     20188800     <common>
 0003:00145c00       _itemRegistered            2018ac00     <common>
 0003:00146000       _bot_minplayers            2018b000     <common>
 0003:00146110       _g_numArenas               2018b110     <common>
 0003:00146114       _podium1                   2018b114     <common>
 0003:00146118       _podium3                   2018b118     <common>
 0003:0014611c       _podium2                   2018b11c     <common>
 0003:00146120       _pml                       2018b120     <common>
 0003:001461ac       _pm                        2018b1ac     <common>
 0003:001461c0       _ctftaskpreferences        2018b1c0     <common>
 0003:00146bc0       _bot_interbreedcycle       2018bbc0     <common>
 0003:00146ce0       _bot_saveroutingcache      2018bce0     <common>
 0003:00146e00       _bot_interbreedbots        2018be00     <common>
 0003:00146f20       _bot_memorydump            2018bf20     <common>
 0003:00147030       _bot_interbreed            2018c030     <common>
 0003:00147034       _floattime                 2018c034     <common>
 0003:00147040       _botstates                 2018c040     <common>
 0003:00147140       _bot_interbreedchar        2018c140     <common>
 0003:00147260       _bot_developer             2018c260     <common>
 0003:00147380       _bot_report                2018c380     <common>
 0003:001474a0       _bot_interbreedwrite       2018c4a0     <common>
 0003:001475c0       _bot_testsolid             2018c5c0     <common>
 0003:001476d0       _regularupdate_time        2018c6d0     <common>
 0003:001476d4       _numbots                   2018c6d4     <common>
 0003:001476e0       _bot_testclusters          2018c6e0     <common>
 0003:001477f0       _bot_interbreedmatchcount  2018c7f0     <common>
 0003:00147800       _bot_pause                 2018c800     <common>
 0003:00147920       _bot_thinktime             2018c920     <common>
 0003:00147a40       _blue_altroutegoals        2018ca40     <common>
 0003:00147d40       _bot_nochat                2018cd40     <common>
 0003:00147e60       _bot_challenge             2018ce60     <common>
 0003:00147f80       _bot_rocketjump            2018cf80     <common>
 0003:001480a0       _ctf_redflag               2018d0a0     <common>
 0003:001480d8       _botai_freewaypoints       2018d0d8     <common>
 0003:001480e0       _bot_testrchat             2018d0e0     <common>
 0003:00148200       _bot_grapple               2018d200     <common>
 0003:00148310       _altroutegoals_setup       2018d310     <common>
 0003:00148320       _lastteleport_origin       2018d320     <common>
 0003:0014832c       _lastteleport_time         2018d32c     <common>
 0003:00148330       _blue_numaltroutegoals     2018d330     <common>
 0003:00148340       _bot_predictobstacles      2018d340     <common>
 0003:00148450       _maxclients                2018d450     <common>
 0003:00148460       _g_spSkill                 2018d460     <common>
 0003:00148580       _red_altroutegoals         2018d580     <common>
 0003:00148880       _bot_fastchat              2018d880     <common>
 0003:001489a0       _ctf_blueflag              2018d9a0     <common>
 0003:001489d8       _max_bspmodelindex         2018d9d8     <common>
 0003:001489dc       _red_numaltroutegoals      2018d9dc     <common>
 0003:001489e0       _gametype                  2018d9e0     <common>
 0003:00148a00       _botai_waypoints           2018da00     <common>
 0003:0014bc00       _numnodeswitches           20190c00     <common>
 0003:0014bc20       _nodeswitch                20190c20     <common>
 0003:0014d8e0       _notleader                 201928e0     <common>
 0003:0014d9e0       ___sbh_pHeaderDefer        201929e0     <common>
 0003:0014d9e4       ___sbh_cntHeaderList       201929e4     <common>
 0003:0014d9e8       ___sbh_pHeaderList         201929e8     <common>
 0003:0014d9ec       ___sbh_threshold           201929ec     <common>
 0003:0014d9f0       ___sbh_pHeaderScan         201929f0     <common>
 0003:0014d9f4       ___sbh_sizeHeaderList      201929f4     <common>
 0003:0014d9f8       ___sbh_indGroupDefer       201929f8     <common>
 0003:0014d9fc       ___piob                    201929fc     <common>
 0003:0014da00       __bufin                    20192a00     <common>
 0003:0014ea00       __nstream                  20193a00     <common>
 0003:0014ea04       ___mblcid                  20193a04     <common>
 0003:0014ea08       ___ismbcodepage            20193a08     <common>
 0003:0014ea20       __mbctype                  20193a20     <common>
 0003:0014eb24       ___mbcodepage              20193b24     <common>
 0003:0014eb30       ___mbulinfo                20193b30     <common>
 0003:0014eb40       __mbcasemap                20193b40     <common>
 0003:0014ec40       __crtheap                  20193c40     <common>
 0003:0014ec44       ___active_heap             20193c44     <common>
 0003:0014ec48       __nhandle                  20193c48     <common>
 0003:0014ec60       ___pioinfo                 20193c60     <common>
 0003:0014ed60       ___env_initialized         20193d60     <common>
 0003:0014ed64       ___onexitend               20193d64     <common>
 0003:0014ed68       ___onexitbegin             20193d68     <common>
 0003:0014ed6c       ___mbctype_initialized     20193d6c     <common>
 0003:0014ed70       ___use_sse2_mathfcns       20193d70     <common>
 0003:0014ed74       ___sse2_available          20193d74     <common>
 0003:0014ed78       __acmdln                   20193d78     <common>
 0003:0014ed7c       __pRawDllMain              20193d7c     <common>

 entry point at        0001:0003311e

 Static symbols

 0001:00005690       _VectorCompare             20006690 f   ai_dmnet.obj
 0001:000057c0       _VectorLengthSquared       200067c0 f   ai_dmnet.obj
 0001:000057c0       _VectorLengthSquared       200067c0 f   ai_dmnet.obj
 0001:00016e10       _PM_StartTorsoAnim         20017e10 f   bg_pmove.obj
 0001:00016e30       _PM_ContinueLegsAnim       20017e30 f   bg_pmove.obj
 0001:00016e70       _PM_ForceLegsAnim          20017e70 f   bg_pmove.obj
 0001:00016f10       _PM_Friction               20017f10 f   bg_pmove.obj
 0001:00017040       _PM_Accelerate             20018040 f   bg_pmove.obj
 0001:000170c0       _PM_CmdScale               200180c0 f   bg_pmove.obj
 0001:00017150       _PM_SetMovementDir         20018150 f   bg_pmove.obj
 0001:00017220       _PM_CheckJump              20018220 f   bg_pmove.obj
 0001:000172e0       _PM_CheckWaterJump         200182e0 f   bg_pmove.obj
 0001:00017440       _PM_WaterJumpMove          20018440 f   bg_pmove.obj
 0001:00017490       _PM_WaterMove              20018490 f   bg_pmove.obj
 0001:000176b0       _PM_FlyMove                200186b0 f   bg_pmove.obj
 0001:000177c0       _PM_AirMove                200187c0 f   bg_pmove.obj
 0001:00017940       _PM_GrappleMove            20018940 f   bg_pmove.obj
 0001:00017a70       _PM_WalkMove               20018a70 f   bg_pmove.obj
 0001:00017e00       _PM_DeadMove               20018e00 f   bg_pmove.obj
 0001:00017ec0       _PM_NoclipMove             20018ec0 f   bg_pmove.obj
 0001:000180c0       _PM_FootstepForSurface     200190c0 f   bg_pmove.obj
 0001:000180e0       _PM_CrashLand              200190e0 f   bg_pmove.obj
 0001:000182e0       _PM_CorrectAllSolid        200192e0 f   bg_pmove.obj
 0001:000184a0       _PM_GroundTraceMissed      200194a0 f   bg_pmove.obj
 0001:000185b0       _PM_GroundTrace            200195b0 f   bg_pmove.obj
 0001:00018820       _PM_SetWaterLevel          20019820 f   bg_pmove.obj
 0001:00018940       _PM_CheckDuck              20019940 f   bg_pmove.obj
 0001:00018b60       _PM_Footsteps              20019b60 f   bg_pmove.obj
 0001:00018d70       _PM_WaterEvents            20019d70 f   bg_pmove.obj
 0001:00018e10       _PM_BeginWeaponChange      20019e10 f   bg_pmove.obj
 0001:00018e80       _PM_FinishWeaponChange     20019e80 f   bg_pmove.obj
 0001:00018ef0       _PM_TorsoAnimation         20019ef0 f   bg_pmove.obj
 0001:00018f70       _PM_Weapon                 20019f70 f   bg_pmove.obj
 0001:00019210       _PM_Animate                2001a210 f   bg_pmove.obj
 0001:00019260       _PM_DropTimers             2001a260 f   bg_pmove.obj
 0001:0001b7a0       _SpawnModelOnVictoryPad    2001c7a0 f   g_arenas.obj
 0001:0001ba60       _CelebrateStop             2001ca60 f   g_arenas.obj
 0001:0001ba90       _CelebrateStart            2001ca90 f   g_arenas.obj
 0001:0001bae0       _PodiumPlacementThink      2001cae0 f   g_arenas.obj
 0001:0001bf10       _SpawnPodium               2001cf10 f   g_arenas.obj
 0001:0001c390       _G_LoadArenasFromFile      2001d390 f   g_bot.obj
 0001:0001c460       _G_LoadArenas              2001d460 f   g_bot.obj
 0001:0001c600       _PlayerIntroSound          2001d600 f   g_bot.obj
 0001:0001cc80       _AddBotToSpawnQueue        2001dc80 f   g_bot.obj
 0001:0001cfc0       _G_SpawnBots               2001dfc0 f   g_bot.obj
 0001:0001d100       _G_LoadBotsFromFile        2001e100 f   g_bot.obj
 0001:0001d1d0       _G_LoadBots                2001e1d0 f   g_bot.obj
 0001:0001d4c0       _G_AddBot                  2001e4c0 f   g_bot.obj
 0001:0001e310       _ClientCleanName           2001f310 f   g_client.obj
 0001:00020540       _G_SayTo                   20021540 f   g_cmds.obj
 0001:00020860       _Cmd_Tell_f                20021860 f   g_cmds.obj
 0001:00020930       _G_VoiceTo                 20021930 f   g_cmds.obj
 0001:00020a80       _Cmd_VoiceTell_f           20021a80 f   g_cmds.obj
 0001:00020b50       _Cmd_VoiceTaunt_f          20021b50 f   g_cmds.obj
 0001:00026cd0       _InitShooter_Finish        20027cd0 f   g_misc.obj
 0001:000284a0       _Touch_DoorTriggerSpectator 200294a0 f   g_mover.obj
 0001:0002ac40       _StringToFilter            2002bc40 f   g_svcmds.obj
 0001:0002acf0       _UpdateIPBans              2002bcf0 f   g_svcmds.obj
 0001:0002aed0       _AddIP                     2002bed0 f   g_svcmds.obj
 0001:0002d270       _target_location_linkup    2002e270 f   g_target.obj
 0001:0002d380       _VectorLength              2002e380 f   g_team.obj
 0001:0002d380       _VectorLength              2002e380 f   g_team.obj
 0001:0002e900       _SortClients               2002f900 f   g_team.obj
 0001:00032a10       _$$$00001                  20033a10 f   LIBC:strchr.obj
 0001:00032d20       _shortsort                 20033d20 f   LIBC:qsort.obj
 0001:000333ff       __shift                    200343ff f   LIBC:cvt.obj
 0001:00033909       __hextodec                 20034909 f   LIBC:input.obj
 0001:0003393b       __inc                      2003493b f   LIBC:input.obj
 0001:00034c8a       _write_char                20035c8a f   LIBC:output.obj
 0001:00034cbd       _write_multi_char          20035cbd f   LIBC:output.obj
 0001:00034ce1       _write_string              20035ce1 f   LIBC:output.obj
 0001:0003579e       _has_osfxsr_set            2003679e f   LIBC:cpu_disp.obj
 0001:00035a0e       _doexit                    20036a0e f   LIBC:crt0dat.obj
 0001:00035d84       _parse_cmdline             20036d84 f   LIBC:stdargv.obj
 0001:00036529       $$$00003                   20037529 f   LIBC:exsup3.obj
 0001:00036893       _CPtoLCID                  20037893 f   LIBC:mbctype.obj
 0001:000368c2       _setSBCS                   200378c2 f   LIBC:mbctype.obj
 0001:000368eb       _setSBUpLow                200378eb f   LIBC:mbctype.obj
 0001:00037329       __abstract_cw              20038329 f   LIBC:ieee87.obj
 0001:000373bb       __hw_cw                    200383bb f   LIBC:ieee87.obj
 0001:00037918       _report_failure            20038918 f   LIBC:secchk.obj
 0001:00039c00       $$$00001                   2003ac00 f   LIBC:exsup.obj
 0001:00039c20       __unwind_handler           2003ac20 f   LIBC:exsup.obj
 0001:00039c20       $$$00003                   2003ac20 f   LIBC:exsup.obj
 0001:00039c42       $$$00005                   2003ac42 f   LIBC:exsup.obj
 0001:00039caa       $$$00007                   2003acaa f   LIBC:exsup.obj
 0001:00039cee       $$$00011                   2003acee f   LIBC:exsup.obj
 0001:0003ade4       _flsall                    2003bde4 f   LIBC:fflush.obj
